:020000040800F2
:1000000080B100209D010008253A0108A5240108BF
:10001000493701089535000875D401080000000033
:10002000000000000000000000000000416701081F
:10003000D56C00080000000021430108717101081F
:10004000B7010008B7010008B7010008B7010008B0
:10005000B7010008B7010008D96C0008B701000813
:10006000B7010008E56C0008F16C0008B701000852
:100070003567000845670008B7010008B7010008A8
:10008000B7010008B7010008B7010008B701000870
:1000900099350008A9350008B7010008FD6C000873
:1000A00065720108B7010008B7010008B701000830
:1000B000B7010008B7010008B7010008B701000840
:1000C000B7010008B7010008B7010008B701000830
:1000D000B701000889A20108B7010008B7010008AC
:1000E000B7010008B7010008B7010008B701000810
:1000F000B7010008B7010008B701000855670008FC
:10010000B7010008B7010008B7010008B7010008EF
:10011000B7010008B7010008B701000875720108AF
:10012000B701000865670008756700088567000863
:10013000B7010008B7010008B7010008B7010008BF
:10014000B9350008C9350008B7010008953A01081B
:1001500095670008A5670008B5670008A5A2010813
:10016000B7010008B7010008B7010008B70100088F
:10017000B7010008B7010008B7010008000000003F
:10018000B7010008B7010008DFF80CD000F0C4FB8D
:1001900000480047C1D7010880B1002006488047C9
:1001A00006480047FEE7FEE7FEE7FEE7FEE7FEE75C
:1001B000FEE7FEE7FEE7FEE7457201088901000859
:1001C0002DE9F05F0546002092469B46884606468C
:1001D000814640241BE0284641464746224600F01F
:1001E0002DFA53465A46C01A914110D3114618466B
:1001F000224600F014FA2D1A67EB01084F462246FA
:100200000120002100F00BFA17EB00094E41201EDF
:10021000A4F10104DFDC484631462A464346BDE8E6
:10022000F09F00000649074A0868504343F239022C
:10023000104408604008704701490860704700009A
:10024000000000206D4EC64140EA01039B0703D029
:1002500009E008C9121F08C0042AFAD203E011F805
:10026000013B00F8013B521EF9D27047D2B201E0C7
:1002700000F8012B491EFBD270470022F6E710B5AB
:1002800013460A4604461946FFF7F0FF204610BD04
:1002900010B5044604E00B7800F8013B03B1491C9B
:1002A000521EF8D2204610BD421C10F8011B002936
:1002B000FBD1801A704710B5002200E0521C835C0D
:1002C0008C5CA34201D1002BF8D1D8B2E1B2401A24
:1002D00010BD034611F8012B00F8012B002AF9D1BB
:1002E0001846704730B505460020034600E05B1C09
:1002F000934205D2EC5CC85C201A01D1002CF6D1E7
:1003000030BD2DE9FE4F804681EA0300C00F0C4648
:10031000009021F0004123F00045B8EB0200A94114
:1003200005D24046214690461C460B46024623F025
:100330000040104347D0270DC7F30A00C3F30A510A
:100340000290401A019040286BDAC3F3130040F486
:10035000801B0098924620B10023D2EB030A63EB86
:100360000B0B01985946C0F14002504600F057F976
:1003700006460D4650465946019A00F06FF910EBBB
:1003800008006141002487EA115284EAE7731A43A6
:1003900040D0009A62B3019A012A4FEA075215DC55
:1003A000001B61EB02014FF0004202EA0752CDE967
:1003B0000042001C41F5801132462B4600F0A6F9A0
:1003C00003B0BDE8F08F40462146F9E7001B61EB22
:1003D0000201001C41F5801300185B412018A2F5B2
:1003E000001747EB030140EAD570B6196D4111E0E3
:1003F0006D084FEA360645EAC0754FEA0752001B02
:1004000061EB0201001C41F5801149084FEA300000
:100410000019514132462B4603B0BDE8F04F00F0C1
:1004200066B90098012240000023D0EB020263EB82
:10043000E073009821464FEAE074B8EB000061EBEE
:100440000401E9E783F000435BE781F0004158E7EE
:100450002DE9FE4F81EA030404F0004421F000413D
:1004600000944FF0000B23F0004350EA01045ED0EB
:1004700052EA03045BD0C3F30A54C1F30A552C4477
:10048000A4F2F3340194A0FB0254C1F3130141F42C
:100490008011C3F3130343F4801301FB024400FBF8
:1004A000034E840A970A44EA815447EA8357A4FB1F
:1004B000076802958D0A05FB07854FEA932C04FB1C
:1004C0000C542705029D4FEA065847EA1637B5EB4C
:1004D00008056EEB070C870E920E47EA811742EA79
:1004E0008312A7FB0201B6EB0B0164EB00042B0D9A
:1004F00043EA0C335E1844EB1C50DA465146E7FBE6
:100500000201C5F313044FEA0B3343EA14534FEAD5
:100510000432019C43EA0603A4F10C040294009CFB
:10052000CDE900B400F0F2F803B0BDE8F08F002090
:100530000146F9E70EB5C10F80EAE0700844CA072A
:10054000002140F233438DE80E000A460B4600F0CE
:10055000DDF803B000BD70B5C1F30A5201F00045EB
:100560000024C1F3130140F2FF3341F480119A4299
:1005700001DA002070BD40F233439A42A2F23342C6
:1005800003DC524200F05AF800E090402C43F1D0D6
:10059000404270BD00F0004230F000400AD0C10D72
:1005A00001F56071C0F3160042EA0151C20840072C
:1005B0001143704700200146704701F0004330B4FA
:1005C00021F0004150EA010206D00A0DA2F5607246
:1005D000C1F31301002A02DC30BC00207047440F35
:1005E00044EAC104C100E01830BC00EBC25000F086
:1005F00047B830B50B46014600202022012409E00F
:1006000021FA02F59D4205D303FA02F5491B04FACB
:1006100002F52844151EA2F10102F1DC30BD202AAA
:1006200004DB203A00FA02F1002070479140C2F149
:10063000200320FA03F3194390407047202A04DB7B
:10064000203A21FA02F00021704721FA02F3D0404B
:10065000C2F120029140084319467047202A06DB68
:10066000CB17203A41FA02F043EAE07306E041FA80
:1006700002F3D040C2F1200291400843194670476E
:100680000029A8BF7047401C490008BF20F00100A6
:10069000704710B4B0FA80FC00FA0CF050EA010484
:1006A00004BF10BC704749B1CCF1200421FA04F416
:1006B00011FA0CF118BF012121430843A3EB0C01EF
:1006C000CB1D4FEA00614FEA102042BF002010BC52
:1006D000704700EBC35010440029A4BF10BC704702
:1006E000401C490008BF20F0010010BC704710B545
:1006F000141E73F1000408DA401C41F10001921845
:100700005B411A4301D120F0010010BD2DE9F04DED
:1007100092469B4611B1B1FA81F202E0B0FA80F242
:1007200020329046FFF77BFF04460F4640EA0A005E
:1007300041EA0B0153465A46084313D0114653EA87
:10074000010019D0C8F140025046FFF777FF054677
:100750000E46504659464246FFF761FF084305D012
:10076000012004E020463946BDE8F08D0020054315
:1007700046EAE0762C4337430A986305E40AA0EB87
:1007800008000022FD0A44EA47540A3002D500203E
:100790000146E9E7010510196941DDE9084500193D
:1007A0006941BDE8F04DA2E72DE9F04D81EA03046F
:1007B00004F0004B21F0004514464FF0000A23F0EE
:1007C000004150EA050220D054EA01021DD0C5F3D1
:1007D0000A570246C5F31303C1F31300C1F30A56C7
:1007E00040F4801543F48013A7EB0608101BD6468F
:1007F00008F2FD3873EB050002D308F1010801E0AF
:1008000092185B41B8F1000F03DA00200146BDE801
:10081000F08D00204FF48011064684460EE0171B31
:1008200073EB050705D3121B63EB050306434CEA84
:10083000010C49084FEA300092185B4150EA010769
:10084000EDD152EA030012D082EA040083EA0501E6
:10085000084305D0101BAB4106D20122002306E05D
:1008600000224FF0004302E06FF0010253101AEB38
:1008700006004CEB085110EB0A0041EB0B01BDE800
:10088000F04DFFF734BFC1F30A52C1F3130140F238
:10089000FF3341F480119A4202DA0020014670478A
:1008A00040F233439A42A2F2334202DC5242FFF753
:1008B000C5BEFFF7B4BE000030B5041E71F10004E0
:1008C00004DB4FF00044404264EB0101141E73F15D
:1008D000000405DB1C464FF00043524263EB040367
:1008E0008B4208BF824230BD30B5041E71F1000456
:1008F00004DB4FF00044404264EB0101141E73F12D
:10090000000405DB1C464FF00043524263EB040336
:10091000994208BF904230BD064C074D06E0E068A2
:1009200040F0010394E8070098471034AC42F6D336
:10093000FFF72EFC845E0208A45E02080EB540F2AA
:10094000334102910021CDE900110A460B46FFF721
:10095000DDFE03B000BD70B58D1810F8014B14F02A
:10096000030201D110F8012B231106D110F8013B2D
:1009700003E010F8016B01F8016B521EF9D1ABB125
:1009800010F8012B04F00C048A1A0C2C03D0A2EBF3
:1009900084129B1C08E010F8014BA2EB0422F8E73C
:1009A00012F8014B01F8014B5B1EF9D5A942D4D3D3
:1009B000002070BD80B582B0019042F20030C4F2D8
:1009C000010000900099486820F440304860019888
:1009D0004268009948681043486001980168486877
:1009E00020F480704860019801680269486840EA14
:1009F0000220486001980168486820F04070486013
:100A0000019801688268486810434860019801684D
:100A1000886820F40060886001980168C26888686E
:100A2000104388600198806A0121C0F600718842F5
:100A300019D0FFE701980168886820F0706088602D
:100A400001980168826A886810438860019801688B
:100A5000886820F04050886001980168C26A886800
:100A6000104388600CE001980168886820F070608D
:100A7000886001980168886820F040508860FFE72E
:100A800001980168886820F0020088600198027E61
:100A90000168886840EA42008860019890F8200068
:100AA00060B3FFE70198406A30B1FFE70198406A00
:100AB000082801D8FFE708E045F28E00C0F60200E2
:100AC00040F2A6711CF0D6FDFFE701980168486866
:100AD00040F40060486001980168486820F4604074
:100AE000486001980168426A4EF20000CFF6FF703C
:100AF00000EB423248681043486006E00198016804
:100B0000486820F400604860FFE701980168C86AFF
:100B100020F47000C86201980168C2690020CFF615
:100B2000F07000EB0252C86A1043C8620198016875
:100B3000886820F400708860019890F8302001687F
:100B4000886840EA4220886001980168886820F43B
:100B500080608860019801684269886840EA822064
:100B6000886002B080BD000080B58AB0089007910F
:100B7000089820B9FFE7FF208DF827009BE0079831
:100B800020B9FFE7FF208DF8270094E0079890ED4B
:100B9000000A90ED013A90ED021A90ED032A20EE42
:100BA000030A21EE021A30EE010A30EE000A8DED42
:100BB000060A079890ED010A90ED021A20EE000A4D
:100BC00021EE011A30EE010A30EE001AB7EE000AEB
:100BD0008DED010A30EE410A8DED050A9DED060A04
:100BE000DDED050A21F080FE9DED011A089880EDEB
:100BF000010A079890ED000A90ED013A90ED024A43
:100C000090ED032A20EE040A22EE032A30EE420A77
:100C100030EE000A8DED040A9DED040AB0EEC00A24
:100C2000B4EE410AF1EE10FA0ADBFFE7DDED040A4B
:100C30009FED230A1CF032FD089880ED020A07E0C0
:100C40009DED040A21F04CFB089880ED020AFFE7B5
:100C5000079890ED000A90ED011A90ED022A90EDB0
:100C6000033A20EE030A21EE021A30EE010A30EEBA
:100C7000000A8DED030A079890ED020A90ED031A21
:100C800020EE000A21EE011A30EE010A30EE001AC1
:100C9000B7EE000A30EE410A8DED020A9DED030A1F
:100CA000DDED020A21F020FE089880ED000A002008
:100CB0008DF82700FFE79DF927000AB080BD00BF2F
:100CC000DB0FC93F80B58CB00A9009918DED080A01
:100CD0000A9820B9FFE7FF208DF82F0029E19DED4C
:100CE000081AB7EE000A80EE010A0A9880ED040A9D
:100CF0000A994FF07E5008600A99002048600A99CE
:100D000088600A99C8600998002800F00E81FFE702
:100D10000998016800914068FFF73CFC0246009882
:100D200001920A46019942EC101B8DED020BFFF770
:100D300031FC9DED020B41EC110B21F0D5FC8DED4A
:100D4000040B9DF8170080F080008DF817000498C0
:100D50000599FFF732FC0790099890ED000AB5EE6F
:100D6000400AF1EE10FA2BD1FFE7099890ED010A45
:100D7000B5EE400AF1EE10FA22D1FFE7099890EDA6
:100D8000020AB5EE400AF1EE10FA19D1FFE70A990E
:100D900040F2C560C3F64D7008600A9944F62D20F4
:100DA000C3F60D4048600A994AF25640CBF63930F6
:100DB00088600A9944F2AD70C3F61970C860B3E058
:100DC0009DED070A9FED5D1AB4EE410AF1EE10FAAF
:100DD00008DBFFE79DED070AB5EE400AF1EE10FAD9
:100DE00019DDFFE70A9945F66E10C3F67F700860BB
:100DF0000A9945F20C30C3F6B01048600A9948F6DB
:100E0000AB00CBF6BB3088600A9949F28550C3F637
:100E10009750C86087E09DED070A9FED491AB4EE30
:100E2000410AF1EE10FA0ADBFFE79DED070A9FED9C
:100E3000431AB4EE410AF1EE10FA19DDFFE70A9900
:100E400040F2C560C3F64D7008600A9944F62D2043
:100E5000C3F60D4048600A994AF25640CBF6393045
:100E600088600A9944F2AD70C3F61970C86059E001
:100E70009DED070A9FED331AB4EE410AF1EE10FA28
:100E80000ADBFFE79DED070A9FED2D1AB4EE410A3C
:100E9000F1EE10FA19DDFFE70A9940F2C560C3F6DA
:100EA0004D7008600A9944F62D20C3F60D40486045
:100EB0000A994AF25640CBF6393088600A9944F2D2
:100EC000AD70C3F61970C8602BE09DED070A9FED69
:100ED0001D1AB4EE410AF1EE10FA08DBFFE79DEDB2
:100EE000070AB5EE400AF1EE10FA19DDFFE70A999C
:100EF00040F2C560C3F64D7008600A9944F62D2093
:100F0000C3F60D4048600A994AF25640CBF6393094
:100F100088600A9944F2AD70C3F61970C860FFE7A3
:100F2000FFE7FFE7FFE7FFE7FFE700208DF82F006F
:100F3000FFE79DF92F000CB080BD00BFDB0FC93F5C
:100F4000DB0F49400000B44281B0009000990020BE
:100F500088604860086001B07047000080B52DEDE2
:100F6000048BB2B030902F912E922D93309828B9E7
:100F7000FFE7FF208DF8C70000F0F7BD2F9828B9D4
:100F8000FFE7FF208DF8C70000F0EFBD2E9828B9CD
:100F9000FFE7FF208DF8C70000F0E7BD40F28411A5
:100FA000C2F200014EF69E70C3F6275008602D98DD
:100FB00048B9FFE730982F992E9A00F0DDFD8DF8A3
:100FC000C70000F0D2BD2D98006809902D984068A8
:100FD00008902D98806807909DED090AB5EE400AAB
:100FE000F1EE10FA19D1FFE79DED080AB5EE400ABF
:100FF000F1EE10FA11D1FFE79DED070AB5EE400AB8
:10100000F1EE10FA09D1FFE730982F992E9A00F0EF
:10101000B3FD8DF8C70000F0A8BD2F9800680690BA
:101020002F98406805902F98806804902E9800684B
:1010300003902E98406802902E9880680190309816
:101040009DED033A90ED010A90ED022A90ED031A0E
:1010500020EE430A9DED023A22EE032A30EE420AC8
:101060009DED012A21EE021A30EE410AB6EE001A79
:1010700020EE010A8DED270A30989DED034A90ED90
:10108000000A90ED023A90ED032A20EE040A9DED4D
:10109000014A23EE043A30EE030A9DED023A22EEB5
:1010A000032A30EE420A20EE010A8DED260A30981E
:1010B0009DED024A90ED000A90ED013A90ED032A71
:1010C00020EE040A9DED014A23EE043A30EE430A75
:1010D0009DED033A22EE032A30EE020A20EE010AC9
:1010E0008DED250A30989DED014A90ED000A90EDB6
:1010F000013A90ED022A20EE040A9DED024A23EE09
:10110000043A30EE030A9DED033A22EE032A30EE54
:10111000420A20EE010A8DED240A9DED060AB5EE85
:10112000400AF1EE10FA11D1FFE79DED050AB5EE88
:10113000400AF1EE10FA09D1FFE79DED040AB5EE81
:10114000400AF1EE10FA00F09984FFE79DED060ADF
:1011500020EE000A9DED051A21EE011A30EE010A7B
:101160009DED041A21EE011A30EE010A11F020FA69
:101170008DED2C0A9DED2C1A9DED060A20EE010A3C
:101180008DED060A9DED2C1A9DED050A20EE010A53
:101190008DED050A9DED2C1A9DED040A20EE010A45
:1011A0008DED040A9DED090A20EE000A9DED081A56
:1011B00021EE011A30EE010A9DED071A21EE011A07
:1011C00030EE010A11F0F4F98DED2C0A9DED2C1A88
:1011D0009DED090A20EE010A8DED090A9DED2C1AFC
:1011E0009DED080A20EE010A8DED080A9DED2C1AEE
:1011F0009DED070A20EE010A8DED070A309890ED6B
:10120000000A30EE000A9DED091A20EE010A8DED6C
:10121000210A309890ED000A30EE000A9DED081A80
:1012200020EE010A8DED200A309890ED000A30EE94
:10123000000A9DED071A20EE010A8DED1F0A309875
:1012400090ED010A30EE000A9DED091A20EE010A28
:101250008DED1E0A309890ED000A30EE000A8DEDFB
:10126000190A309890ED010A30EE000A8DED180A47
:10127000309890ED020A30EE000A8DED170A309892
:1012800090ED030A30EE000A8DED160A309890EDCD
:10129000000A90ED021A30EE000A20EE010A8DEDF0
:1012A000150A309890ED020A90ED031A30EE000A0C
:1012B00020EE010A8DED140A309890ED000A20EE20
:1012C000000A8DED130A309890ED000A90ED011A96
:1012D00020EE010A8DED120A309890ED000A90ED93
:1012E000021A20EE010A8DED110A309890ED000AE5
:1012F00090ED031A20EE010A8DED100A309890ED62
:10130000010A20EE000A8DED0F0A309890ED010AD7
:1013100090ED021A20EE010A8DED0E0A309890ED44
:10132000010A90ED031A20EE010A8DED0D0A3098A6
:1013300090ED020A20EE000A8DED0C0A309890ED37
:10134000020A90ED031A20EE010A8DED0B0A309887
:1013500090ED030A20EE000A8DED0A0A9DED091AB0
:101360009DED130A21EE000A9DED202A309890EDA4
:10137000025A90ED033A22EE032A30EE420A9DED26
:101380001F2A22EE052A30EE020A9DED0F2A21EED9
:10139000022A30EE020A9DED182A9DED084A22EE3F
:1013A000044A24EE054A30EE040A9DED074A22EE77
:1013B000042A22EE032A30EE020A9DED0C2A21EEC9
:1013C000022A30EE420A9DED0A2A21EE021A30EE80
:1013D000410A8DED230A9DED210A309890ED015AC6
:1013E00090ED024A90ED033A20EE030A9DED081AB3
:1013F0009DED132A21EE022A30EE020A9DED1F2AEE
:1014000022EE052A30EE420A9DED1E2A22EE042A23
:1014100030EE020A9DED0F2A21EE022A30EE420A3A
:101420009DED0C2A21EE022A30EE020A9DED172ACC
:101430009DED074A22EE042A22EE032A30EE020A2C
:101440009DED0A2A21EE021A30EE410A8DED220AA4
:101450009DED230A20EE000A9DED221A21EE011ACD
:1014600030EE010A11F0A4F8B7EE006A86EE000A29
:101470008DED1D0A9DED210A309890ED012A90ED29
:10148000021A90ED033A20EE011A9DED200A20EE9B
:10149000020A30EE412A9DED071A9DED130A21EE56
:1014A000000A30EE022A9DED1E0A20EE030A30EEFD
:1014B000020A9DED0F2A21EE022A30EE420A9DED2E
:1014C000172A9DED084A22EE042A22EE032A30EE66
:1014D000020A9DED0C2A21EE022A30EE420A9DED11
:1014E0000A2A21EE021A30EE010A8DED1C0A9DED4A
:1014F0001D0A30EE000A8DED1B0A9DED1C0A30EE30
:10150000000A8DED1A0A9DED170ADDED0D0A30EE89
:10151000A02A9DED151A31EE422A9DED061A31EEF4
:10152000021A20EE010A9DED181ADDED123A33EE93
:10153000A32A9DED143A32EE032A9DED053A32EED0
:10154000432A21EE021A70EE014A9DED1C3A3098B2
:1015500090ED011A90ED020AD0ED032A63EE001A15
:101560009DED1D2A9DED0C7AB6EE004A8DED004AE8
:1015700077EE445A9DED0A5A35EE255A62EE055A29
:101580009DED115A75EE606A63EE266A75EEA66AE5
:10159000DDED095A75EEA65A61EEA51A71EEA41A90
:1015A00062EE222A23EE011A31EE621ADDED0E2AD6
:1015B000DDED104A72EEE42A62EE222ADDED0B4ADE
:1015C00073EEA43A63EE233A72EEA32ADDED083AF5
:1015D00072EEE32A21EE221A31EE211A22EE000ADF
:1015E00035EE205A22EE052A9DED0F5A34EE455A6B
:1015F00035EE475A23EE053A32EE032A9DED073ABF
:1016000032EE432A20EE020A30EE010A8DED2B0A5B
:101610009DED160ADDED0D2A32EEA21A9DED152A7A
:1016200031EE421A9DED062A31EE421A20EE010AF1
:101630009DED191ADDED126A36EEA62A9DED143ADB
:1016400032EE032A9DED053A32EE432A21EE021ACC
:1016500030EE011A3098D0ED005AD0ED014AD0EDAD
:10166000023A90ED032AB1EE000A24EE803A9DED95
:101670000F7A37EE075A75EE461ADDED0C0A30EE9A
:10168000A05A75EE211A9DED045A35EE215A23EE2B
:10169000053A31EE031A9DED1C5A65EE027A9DED76
:1016A0001D3A74EE601A9DED0A8A71EEC81A23EE97
:1016B000218ADDED111A32EEE19A25EE099A38EE13
:1016C000098A9DED099A38EE498A67EE887A31EEEB
:1016D000271A63EE233A65EE255A73EEA53ADDED3F
:1016E0000E5ADDED107A75EEE75A63EE255ADDED00
:1016F0000B7A76EEA76A65EE266A75EEA65ADDEDE0
:10170000086A75EEE65A63EEA53A31EE231A23EE27
:10171000022ADDED1A3A63EEA43A32EE632A71EE44
:10172000A21A23EE213A34EE477A37EE607A25EE9C
:10173000075A33EE053A9DED075A33EE453A22EE4D
:10174000032A31EE021A8DED2A1A9DED191ADDEDEC
:101750000D0A30EEA03A9DED152A32EE433A9DED8A
:10176000062A32EE032A21EE021A9DED162ADDED3D
:10177000124A34EEA43A9DED145A33EE053A9DED2B
:10178000055A33EE453A22EE032A31EE022A30980A
:1017900090ED001AD0ED011AD0ED022AD0ED033AF7
:1017A00022EE800A9DED0F5A35EE053A33EE467A69
:1017B0009DED0C6A36EE063A33EE077A9DED043A5B
:1017C00033EE073A20EE030A70EE025A9DED1B0A33
:1017D00020EE620A9DED1C3A23EE012A30EE420A09
:1017E0009DED1D2A34EE467ADDED0A6A37EE667A03
:1017F00062EE076A9DED117A70EEC77A63EE277A82
:1018000076EEA76ADDED097A76EEE76A20EE260A23
:1018100030EE250A62EE211A63EE233A71EEA31A26
:10182000DDED0E3ADDED105A73EEE53A62EE233A45
:10183000DDED0B5A74EEA54A63EE244A73EEA43A2A
:10184000DDED084A73EEE43A61EEA31A30EE210AA8
:1018500022EE011ADDED1A1A61EEA21A31EE611ABA
:1018600037EE207A22EE072A34EE455A35EE465AF4
:1018700023EE053A32EE032A9DED073A32EE432A73
:1018800021EE021A30EE010A8DED290A9DED180AAB
:101890009DED0D7A37EE071A9DED152A31EE421AAD
:1018A0009DED062A31EE421A20EE010A9DED171A2F
:1018B000DDED122A32EEA22A9DED143A32EE032A11
:1018C0009DED053A32EE432A21EE021A70EE013AFE
:1018D0009DED1B1A3098D0ED001A90ED010AD0ED65
:1018E000020A90ED032A21EE022A9DED1C3A23EE16
:1018F000001A31EE421A9DED1D2A9DED0C5A34EE70
:10190000456ADDED0A4A36EE646A62EE064A9DEDEE
:10191000116A77EE465A63EE255A74EEA54ADDED5C
:10192000095A74EEE54A21EE241A31EE231A62EECA
:10193000211A63EE200A70EEE10ADDED0E1ADDEDEC
:10194000103A71EEE31A62EE211ADDED0B3A72EEF7
:10195000A32A63EE222A71EEA21ADDED082A71EEA7
:10196000E21A60EEA10A31EE201A22EE000A36EEEB
:10197000076A22EE062A9DED0F6A34EE464A34EEDF
:10198000454A23EE043A32EE032A9DED073A32EE41
:10199000432A20EE020A30EE010A8DED280A9DED61
:1019A0002B0A20EE000A9DED2A1A21EE011A30EED4
:1019B000010A9DED291A21EE011A30EE010A9DED72
:1019C000281A21EE011A30EE010A10F0F1FD8DED1A
:1019D0002C0A9DED2C1A9DED2B0A20EE010A8DEDAF
:1019E0002B0A9DED2C1A9DED2A0A20EE010A8DEDA1
:1019F0002A0A9DED2C1A9DED290A20EE010A8DED93
:101A0000290A9DED2C1A9DED280A20EE010A8DED84
:101A1000280A40F28410C2F2000090ED000A9DED09
:101A20002B1A20EE011A9DED270A30EE410A8DEDAA
:101A3000270A90ED000A9DED2A1A20EE011A9DED6D
:101A4000260A30EE410A8DED260A90ED000A9DED42
:101A5000291A20EE011A9DED250A30EE410A8DED7E
:101A6000250A90ED000A9DED281A20EE011A9DED41
:101A7000240A30EE410A8DED240AFFE79DED271A76
:101A8000309890ED000A90ED042A21EE021A30EE13
:101A9000010A80ED000A9DED261A309890ED010AAA
:101AA00090ED042A21EE021A30EE010A80ED010ABF
:101AB0009DED251A309890ED020A90ED042A21EE52
:101AC000021A30EE010A80ED020A9DED241A3098C8
:101AD00090ED030A90ED042A21EE021A30EE010A7D
:101AE00080ED030A309890ED000A90ED013A90EDF8
:101AF000022A90ED031A20EE000A23EE033A30EE9C
:101B0000030A22EE022A30EE020A21EE011A30EE1A
:101B1000010A10F04DFD8DED2C0A9DED2C1A309828
:101B200090ED000A20EE010A80ED000A9DED2C1ACE
:101B3000309890ED010A20EE010A80ED010A9DED3A
:101B40002C1A309890ED020A20EE010A80ED020A6C
:101B50009DED2C1A309890ED030A20EE010A80EDDD
:101B6000030A00208DF8C700FFE79DF9C70032B0D7
:101B7000BDEC048B80BD000080B5A0B01E901D910F
:101B80001C921E9820B9FFE7FF208DF87F00D3E25A
:101B90001D9820B9FFE7FF208DF87F00CCE21C984C
:101BA00020B9FFE7FF208DF87F00C5E240F28411E5
:101BB000C2F2000142F60230C3F6075008601D98D9
:101BC00000681B901D9840681A901D9880681990B5
:101BD0001C98006818901C98406817901C988068A2
:101BE00016901E989DED183A90ED010A90ED022A8C
:101BF00090ED031A20EE430A9DED173A22EE032AD8
:101C000030EE420A9DED162A21EE021A30EE410A0C
:101C1000B6EE001A20EE010A8DED100A1E989DED19
:101C2000184A90ED000A90ED023A90ED032A20EE5A
:101C3000040A9DED164A23EE043A30EE030A9DEDA8
:101C4000173A22EE032A30EE420A20EE010A8DED09
:101C50000F0A1E989DED174A90ED000A90ED013A8B
:101C600090ED032A20EE040A9DED164A23EE043A75
:101C700030EE430A9DED183A22EE032A30EE020AB6
:101C800020EE010A8DED0E0A1E989DED164A90ED8C
:101C9000000A90ED013A90ED022A20EE040A9DED33
:101CA000174A23EE043A30EE030A9DED183A22EE6D
:101CB000032A30EE420A20EE010A8DED0D0A9DED59
:101CC0001B0AB5EE400AF1EE10FA11D1FFE79DEDC7
:101CD0001A0AB5EE400AF1EE10FA09D1FFE79DEDC0
:101CE000190AB5EE400AF1EE10FA00F0AE81FFE7F6
:101CF0009DED1B0A20EE000A9DED1A1A21EE011A35
:101D000030EE010A9DED191A21EE011A30EE010A9A
:101D100010F04EFC8DED150A9DED151A9DED1B0A78
:101D200020EE010A8DED1B0A9DED151A9DED1A0A94
:101D300020EE010A8DED1A0A9DED151A9DED190A86
:101D400020EE010A8DED190A1E9890ED000A30EE82
:101D5000000A8DED0C0A1E9890ED010A30EE000A83
:101D60008DED0B0A1E9890ED020A30EE000A8DED03
:101D70000A0A1E9890ED030A30EE000A8DED090A5A
:101D80001E9890ED000AB1EE003A20EE030A8DEDA8
:101D9000080A1E9890ED010A20EE030A8DED070A4D
:101DA0001E9890ED020A20EE030A8DED060A1E9899
:101DB00090ED010AB2EE001A20EE010A8DED050A3F
:101DC0001E9890ED020A20EE010A8DED040A1E987D
:101DD00090ED000A20EE000A8DED030A1E9890EDAA
:101DE000010A20EE000A8DED020A1E9890ED020A0B
:101DF00020EE000A8DED010A1E9890ED030A20EEF8
:101E0000000A8DED000A9DED081A9DED010A21EEF4
:101E1000000A9DED0A2A9DED1B4A22EE042A30EEAF
:101E2000020A9DED022A21EE021A30EE010A9DED12
:101E30000B1A9DED1A2A21EE021A30EE410A8DEDA1
:101E4000140A9DED071A9DED000A21EE000A9DED92
:101E5000092A9DED1B4A22EE042A30EE420A9DED2E
:101E6000032A22EE032A1E9890ED014A22EE042A4C
:101E700030EE020A9DED0C2A9DED1A4A22EE042A4C
:101E800030EE420A30EE410A9DED052A9DED024AF0
:101E900022EE044A30EE040A9DED014A22EE042AA5
:101EA00030EE020A9DED192A21EE021A30EE010AE7
:101EB0008DED130A9DED030A20EE030A1E9890EDA6
:101EC000021A20EE010A9DED0C1A9DED1B2A21EE4F
:101ED000021A30EE010A9DED061A9DED002A21EE50
:101EE000022A30EE020A9DED092A9DED1A4A22EEE1
:101EF000042A30EE420A30EE410A9DED042A9DED9F
:101F0000024A22EE044A30EE040A9DED014A22EE16
:101F1000042A30EE020A9DED192A21EE021A30EE53
:101F2000010A8DED120A9DED020A20EE030A1E98A9
:101F300090ED032A20EE020A9DED0B1A9DED1B4A3F
:101F400021EE041A30EE410A9DED011A21EE031A2A
:101F500021EE021A30EE010A9DED0A1A9DED1A2AB1
:101F600021EE021A30EE410A8DED110A9DED140AA0
:101F700020EE000A9DED131A21EE011A30EE010A3F
:101F80009DED121A21EE011A30EE010A9DED111A93
:101F900021EE011A30EE010A10F00AFB8DED150A50
:101FA0009DED151A9DED140A20EE010A8DED140A1F
:101FB0009DED151A9DED130A20EE010A8DED130A11
:101FC0009DED151A9DED120A20EE010A8DED120A03
:101FD0009DED151A9DED110A20EE010A8DED110AF5
:101FE00040F28410C2F2000090ED000A9DED141A38
:101FF00020EE011A9DED100A30EE410A8DED100A17
:1020000090ED000A9DED131A20EE011A9DED0F0AC6
:1020100030EE410A8DED0F0A90ED000A9DED121A87
:1020200020EE011A9DED0E0A30EE410A8DED0E0AEA
:1020300090ED000A9DED111A20EE011A9DED0D0A9A
:1020400030EE410A8DED0D0AFFE79DED101A1E9846
:1020500090ED000A90ED042A21EE021A30EE010AFA
:1020600080ED000A9DED0F1A1E9890ED010A90ED8B
:10207000042A21EE021A30EE010A80ED010A9DEDDC
:102080000E1A1E9890ED020A90ED042A21EE021A13
:1020900030EE010A80ED020A9DED0D1A1E9890EDBA
:1020A000030A90ED042A21EE021A30EE010A80EDB7
:1020B000030A1E9890ED000A90ED013A90ED022A75
:1020C00090ED031A20EE000A23EE033A30EE030AE5
:1020D00022EE022A30EE020A21EE011A30EE010A47
:1020E00010F066FA8DED150A9DED151A1E9890ED0B
:1020F000000A20EE010A80ED000A9DED151A1E98D7
:1021000090ED010A20EE010A80ED010A9DED151AFD
:102110001E9890ED020A20EE010A80ED020A9DED64
:10212000151A1E9890ED030A20EE010A80ED030AAD
:1021300000208DF87F00FFE79DF97F0020B080BD73
:1021400084B002900191029820B9FFE7FE208DF83B
:102150000F001CE0019820B9FFE7FE208DF80F006A
:1021600015E0029900200090C1F81B0088614861C9
:102170000861C860886048600199886148610861A9
:10218000C8608860486008608DF80F00FFE79DF91F
:102190000F0004B07047000080B582B00090009836
:1021A00020B9FFE7FE208DF807002AE042F2A06088
:1021B000C2F200000078C00720B1FFE7FD208DF8D3
:1021C00007001EE01BF016FF43F23C31C2F2000193
:1021D000086020B9FFE7FE208DF8070011E042F209
:1021E0008542C0F600020220032101F037F942F2D5
:1021F000A061C2F200010120087000208DF80700E4
:10220000FFE79DF9070002B080BD000080B582B0F5
:10221000019000910199C42081F826000199DDF810
:1022200000C0DCF80000DCF80420DCF80830DCF842
:102230000CC0C1F833C0C1F82F30C1F82B20C1F851
:1022400027000199002081F83700019890F84A0092
:10225000012808D1FFE7019991F8370040F001000B
:1022600081F837001DE0019890F84A00022808D153
:10227000FFE7019991F8370040F0020081F837003C
:102280000EE0019890F84A00032808D1FFE7019971
:1022900091F8370040F0040081F83700FFE7FFE7CE
:1022A000FFE70198273021214FF6FF7202F0FCF979
:1022B0000199A1F84800002002B080BD80B582B02D
:1022C000019000910199A820C8770198203004213D
:1022D0004FF6FF7202F0E8F901998884002002B0FD
:1022E00080BD000080B584B0029001910298043056
:1022F0001B2102F0F5F908B9FFE724E00298806895
:102300000199486002984068019908600298C06885
:10231000019988600298007CC0F3C000019908769A
:102320000298D0F811000199C8600298D0F8150001
:10233000019908610298D0F81900019948610020BC
:102340008DF80F000AE041F28C41C2F200010868EA
:1023500001300860FF208DF80F00FFE79DF90F00A6
:1023600004B080BD80B582B00090022001F016F864
:10237000009904311B220FF037FF20B9FFE700203E
:102380008DF8070003E0FF208DF80700FFE79DF9B7
:10239000070002B080BD000080B584B002908DF8C7
:1023A00007109DF80700C00790B1FFE7022000F07A
:1023B000F5FF02991F312B220FF0A6FF20B9FFE78E
:1023C00000208DF80F0015E0FF208DF80F0011E0C0
:1023D000022000F0E3FF0299263124220FF094FF3F
:1023E00020B9FFE700208DF80F0003E0FF208DF8F3
:1023F0000F00FFE79DF90F0004B080BD80B54FF4DA
:102400008040012100221BF067FDA0F58040B0FA5A
:1024100080F0400980BD000084B08DED030ACDED51
:10242000020A9DED030A9DED021AB1EE411AB4EEC7
:10243000410AF1EE10FA07DAFFE79DED020AB1EE6C
:10244000400A8DED010A18E09DED030A9DED021A88
:10245000B4EE410AF1EE10FA05DDFFE79DED020A48
:102460008DED000A04E09DED030A8DED000AFFE703
:102470009DED000A8DED010AFFE79DED010A04B014
:102480007047000080B543F23C30C2F200000068A3
:102490004FF480411BF0CEFC80BD000080B543F2BC
:1024A0002C30C2F20000006802211BF0C3FC80BD8A
:1024B00080B582B040F66C42C2F20002002001906A
:1024C0001221132300F06EFA019802B080BD0000C3
:1024D00080B5082001214FF0FF321BF0FDFC80BDCC
:1024E00081B000909FED010A01B070470000C84321
:1024F00080B543F22C30C2F20000006801211BF0CD
:1025000099FC80BD82B00190019890ED000A0020F6
:102510009FED141AB4EE410AF1EE10FA00901BDAA6
:10252000FFE7019890ED010A00209FED0E1AB4EE2E
:10253000410AF1EE10FA00900EDAFFE7019890EDF3
:10254000020A9FED081A0020B4EE410AF1EE10FADB
:10255000B8BF01200090FFE7009800F0010002B032
:10256000704700BF8FC2F53C80B540F66C40C2F2A8
:102570000000C21D01200221062300F013FA0020F2
:1025800080BD000080B5042001214FF0FF321BF018
:10259000A3FC80BD80B58CB00A9009910A9820B93F
:1025A000FFE7FE208DF82F00B5E0099820B9FFE77E
:1025B000FE208DF82F00AEE042F29C60C2F20000D7
:1025C0000078C00720B1FFE7FD208DF82F00A2E0C2
:1025D0001BF010FD43F22C31C2F20001086020B95B
:1025E000FFE7FE208DF82F0095E009980A99C86151
:1025F000002008907E21B622069200F087FA069A03
:102600000120142100F082FA1E20079000F01CFB2C
:102610000799089800F00CFA0899084600F008FAA3
:102620001E2804D0FFE7FC208DF82F0073E0012066
:10263000002100F0FDF90F2804D0FFE7FC208DF801
:102640002F0068E01020039000F0A6FB20200490EB
:1026500000F0A2FB42F62D12C0F600020121029109
:10266000084600F079FE039842F29D41C0F6000151
:1026700000F006FC049842F2F141C0F6000100F0BF
:10268000FFFB002005904021AA2200F03FFA029AA9
:102690000598412100F03AFA05985321082200F0EC
:1026A00035FA059858210422019200F02FFA019A78
:1026B00005987D2100F02AFA322000F0C5FA029A2E
:1026C0000F21104600F022FA02980399032200F02D
:1026D0001DFA0298059A162100F018FA029A18219C
:1026E000104600F013FA02981521802200F00EFA2D
:1026F0000A2000F0A9FA0299039842F29C62C2F201
:102700000002117000F082FB049800F07FFB059836
:102710008DF82F00FFE79DF92F000CB080BD000061
:1027200084B00290029820B9FFE7FE208DF80F00D8
:102730006AE040F66C41C2F20001B1F80100ADF868
:102740000600B1F80300ADF80400B1F80500ADF8DB
:102750000200BDF9060000EE100AB8EEC00A0298A9
:1027600080ED000ABDF9040000EE100AB8EEC00AC0
:10277000029880ED010ABDF9020000EE100AB8EEE1
:10278000C00A029880ED020A029890ED000A9FEDBF
:10279000201A80EE010A80ED000A029890ED010AED
:1027A00080EE010A80ED010A029890ED020A80EEA7
:1027B000010A80ED020A487C897CC00040EA511081
:1027C000ADF80000BDF90000B0F5806F07DBFFE752
:1027D000BDF80000A0F50060ADF80000FFE7BDF90E
:1027E000000000EE100AB8EEC00AB4EE001A20EEA7
:1027F000010AB3EE071A30EE010A029880ED060ACC
:1028000000208DF80F00FFE79DF90F0004B070471E
:1028100000A0AA4584B00290029820B9FFE7FE20EC
:102820008DF80F007AE040F66C40C2F20000B0F87C
:102830000710ADF80610B0F80910ADF80410B0F8A4
:102840000B00ADF80200BDF9060000EE100AB8EE6C
:10285000C00A029880ED030ABDF9040000EE100AD8
:10286000B8EEC00A029880ED040ABDF9020000EE3D
:10287000100AB8EEC00A029880ED050A029890EDA1
:10288000030A9FED281A80EE010A80ED030A0298E0
:1028900090ED040A80EE010A80ED040A029890EDA2
:1028A000050A80EE010A80ED050A029890ED030A00
:1028B0009FED1D1A20EE010A80ED030A029890EDAB
:1028C000040A20EE010A80ED040A029890ED050A40
:1028D00020EE010A80ED050A0298C16991ED001A07
:1028E00090ED030A30EE410A80ED030A0298C169B7
:1028F00091ED011A90ED040A30EE410A80ED040AD0
:102900000298C16991ED021A90ED050A30EE410A74
:1029100080ED050AFE208DF80F00FFE79DF90F00FE
:1029200004B070476F12034235FA8E3C80B5002028
:10293000C4F20200102108F003FD80B9FFE7002077
:10294000C4F202001021012208F024FD43F22C30D1
:10295000C2F20000006808211BF06CFAFFE740F2A9
:102960000040C4F20200012108F0EAFC88B9FFE748
:1029700040F20040C4F202000122114608F00AFDB4
:1029800043F22C30C2F20000006804211BF052FA1E
:10299000FFE780BD80B5032001214FF0FF321BF01F
:1029A0009BFA80BD80B586B08DF817008DF81610A3
:1029B00004928DF80F30049808B9FFE736E09DF8CF
:1029C00017000146029120B1FFE70298012808D0C4
:1029D00010E00020C4F202001021002208F0DAFC0E
:1029E00008E040F20040C4F202000121002208F099
:1029F000D1FCFFE79DF8160040F0800040F67F41D3
:102A0000C2F20001009108700120019000F084FCE6
:102A10000099019A14230BF0FBFE019800F07CFC56
:102A200004999DF80F200BF0B5FDFFE706B080BDBF
:102A300080B586B08DF816008DF81510012000F0D5
:102A400003F99DF816000146049120B1FFE70498B0
:102A5000012808D010E00020C4F20200102100225A
:102A600008F098FC08E040F20040C4F202000121A6
:102A7000002208F08FFCFFE79DF8150040F0800071
:102A800040F67F41C2F200010191087001200090E0
:102A900000F042FC009A0199142302930BF0B8FE57
:102AA000009800F039FC0199029B02220BF05AFCBD
:102AB0009DF816000146039120B1FFE70398012815
:102AC0000FD01EE00020C4F202001021012208F005
:102AD00061FC40F67F40C2F2000040788DF817009C
:102AE0000FE040F20040C4F202000122114608F05B
:102AF00051FC40F67F40C2F2000000788DF81700CC
:102B0000FFE79DF8170006B080BD000080B584B0D7
:102B10008DF80F008DF80E108DF80D209DF80E0029
:102B200000F07F0040F67F41C2F2000108709DF87E
:102B30000D004870012000F087F89DF80F00014655
:102B4000029120B1FFE70298012808D010E0002090
:102B5000C4F202001021002208F01CFC08E040F240
:102B60000040C4F202000121002208F013FCFFE73C
:102B7000012000F0D1FB40F67F41C2F200010222A9
:102B800014230BF045FE9DF80F000146019120B182
:102B9000FFE70198012808D010E00020C4F20200ED
:102BA0001021012208F0F6FB08E040F20040C4F2D8
:102BB00002000122114608F0EDFBFFE704B080BDE2
:102BC00083B08DF807009DF807000146009150B1D1
:102BD000FFE7009801280CD1FFE741F62820C2F258
:102BE0000000029008E041F60020C2F200000290CE
:102BF00002E000200290FFE7029803B07047000057
:102C000082B08DF806008DF805100092009820B96A
:102C1000FFE7FE208DF8070011E000989DF80610F0
:102C200040F2A853C2F20003342211FB02319DF896
:102C3000052041F8220000208DF80700FFE79DF9EC
:102C4000070002B07047000080B586B004901AF00B
:102C500079FE01464FF47A70B0FBF1F003900498CE
:102C60000399B0FBF1F002901AF02EFE0146481CC9
:102C7000019198B1FFE70198022820D3FFE701985E
:102C800002280FD0FFE701980338022806D3FFE798
:102C900001986FF00041884215D1FFE7FF208DF8C1
:102CA000170014E0029818B1FFE70298009002E0C4
:102CB00001200090FFE700981AF0C0FD03E004989F
:102CC00007F0D2FDFFE700208DF81700FFE79DF920
:102CD000170006B080BD000080B588B00790079847
:102CE000E0B1FFE707980B2818D8FFE70798049092
:102CF00000200290022006900120059007F014FFAA
:102D0000FFE7322004F0B0FA08B1FFE7F9E702A8C4
:102D100001A907F0CBFD07F079FEFFE708B080BD01
:102D200080B584B003900291019202980399019AB0
:102D3000FDF78AFA04B080BD80B584B0039002919B
:102D4000019207F0F1FEFFE70198C0B1FFE7FFE74E
:102D5000322004F089FA08B1FFE7F9E703990298F5
:102D600002780023184607F05BFE039801300390B9
:102D7000029801300290019801380190E4E707F0D1
:102D800045FE04B080BD000080B582B0019001987E
:102D90001CF016FF02B080BD80B582B0ADF8040013
:102DA000BDF804000138014600911F2822D800997F
:102DB000DFE801F0182020202020201C20202020E7
:102DC0002020201020202020202020202020202013
:102DD000202020140A2008F005FF0FE0172008F03B
:102DE00001FF0BE0062008F0FDFE07E0092008F0D7
:102DF000F9FE03E0FF208DF8070003E000208DF8C6
:102E00000700FFE79DF9070002B080BD80B582B0E2
:102E1000ADF80400BDF804000138014600911F28F8
:102E200022D80099DFE801F0182020202020201C63
:102E300020202020202020102020202020202020A2
:102E400020202020202020140A2008F0E3FE0FE09C
:102E5000172008F0DFFE0BE0062008F0DBFE07E09D
:102E6000092008F0D7FE03E0FF208DF8070003E0FB
:102E700000208DF80700FFE79DF9070002B080BD34
:102E800083B0ADF808000191019820B9FFE7FE205A
:102E90008DF80B0025E000208DF80300FFE79DF87A
:102EA00003000F2819DCFFE7BDF808009DF80310A8
:102EB000C840C00750B1FFE701989DF8032040F2D9
:102EC0002C61C2F2000141F8220006E0FFE79DF804
:102ED000030001308DF80300E1E700208DF80B00BE
:102EE000FFE79DF90B0003B07047000080B588B084
:102EF000082004900120059000200690079041F6DC
:102F0000B810C2F2000004A904F062FE18B1FFE795
:102F100003F0FAFEFFE741F6B810C2F2000001909C
:102F200005F090FA0198052105F0F6F9019804F0F2
:102F3000AFFF03909DED030AB8EE400A40F29C50AB
:102F4000C2F2000090ED001A20EE010A9FED041A73
:102F500020EE010A8DED020A9DED020A08B080BD47
:102F60005D74214180B588B0102004900120059047
:102F700000200690079041F67010C2F2000004A9EC
:102F800004F026FE18B1FFE703F0BEFEFFE741F6AE
:102F90007010C2F20000019005F054FA019805216A
:102FA00005F0BAF9019804F073FF03909DED030A50
:102FB000B8EE400A40F29C50C2F2000090ED001AB8
:102FC00020EE010A8DED020A9DED020A9FED061A20
:102FD00030EE010A9FED051A20EE010AB3EE091A40
:102FE00030EE010A08B080BD5C8F42BF0000C843CC
:102FF00080B588B006AA0392024603988DF81E2079
:103000008DF81D1080ED000A90ED000AB7EE001A51
:10301000B4EE410AF1EE10FA04DDFFE7FF208DF86F
:103020001F0097E0039890ED000A9FED4C1A20EEE8
:10303000010ABDEEC00A10EE100AADF812009DF8AC
:103040001E0001460291F0B1FFE70298012804D06A
:10305000FFE7029802280BD020E0BDF8120042F2F0
:10306000BC41C2F200010968C8630820059015E060
:10307000BDF8120042F2BC41C2F200010968886347
:10308000042005900AE0BDF8120042F2BC41C2F2F1
:1030900000010968486300200590FFE79DF81D00C6
:1030A0000146019140B1FFE70198012814D0FFE7E4
:1030B0000198022820D049E0059942F2BC40C2F2B2
:1030C00000000DF0D5FF059A42F2B461C2F2000192
:1030D00008681043086039E0059942F2BC40C2F22A
:1030E00000000EF0A7F9059A42F2B461C2F20001A5
:1030F00008689043086029E042F2B460C2F2000020
:1031000000680599084210D0FFE7059942F2BC40DB
:10311000C2F200000EF08EF9059A42F2B461C2F2DA
:1031200000010868904308600FE0059942F2BC4036
:10313000C2F200000DF09CFF059A42F2B461C2F2A7
:103140000001086810430860FFE7FFE700208DF8E2
:103150001F00FFE79DF91F0008B080BD00FF7F47FB
:1031600080B582B0019001981CF006FA02B080BDD3
:1031700080B586B004A90291014602988DF8161018
:1031800080ED000A90ED000AB7EE001AB4EE410A95
:10319000F1EE10FA04DDFFE7FF208DF817006AE07A
:1031A000029890ED000AB5EE400AF1EE10FA03DA4B
:1031B000FFE700200490FFE79DF81600014601910B
:1031C00020B1FFE70198012815D029E0029890ED81
:1031D000000A42F2E430C2F20000006890ED0B1ADF
:1031E000B8EE411A20EE010ABDEEC00A10EE100A38
:1031F000ADF80E0014E0029890ED000A42F29C3007
:10320000C2F20000006890ED0B1AB8EE411A20EEF1
:10321000010ABDEEC00A10EE100AADF80E00FFE77D
:10322000BDF80E0001281DDBFFE79DF816000146E2
:10323000009120B1FFE70098012809D011E0BDF806
:103240000E0042F2E431C2F200010968486308E06E
:10325000BDF80E0042F29C31C2F2000109684863D9
:10326000FFE704E09DF8160000F02CF8FFE70020CF
:103270008DF81700FFE79DF9170006B080BD00002C
:1032800080B582B08DF807009DF8070001460091D7
:1032900020B1FFE70098012808D00FE042F2E430A7
:1032A000C2F2000000210DF0E3FE07E042F29C3084
:1032B000C2F2000000210DF0DBFEFFE7002002B0AB
:1032C00080BD000080B584B08DF80F009DF80F0020
:1032D0000146029120B1FFE70298012808D00FE0D3
:1032E00042F2E430C2F2000000210EF0A3F807E041
:1032F00042F29C30C2F2000000210EF09BF8FFE782
:1033000041F20040C4F2020040210022019208F084
:1033100041F8019804B080BD83B08DF807009DF896
:1033200007000146009120B1FFE70098012806D070
:103330000BE042F24430C2F20000029008E042F298
:10334000EC20C2F20000029002E000200290FFE7B1
:10335000029803B07047000082B08DF806008DF827
:1033600005100092009820B9FFE7FE208DF80700B5
:1033700010E000989DF8062040F2F061C2F20001D2
:1033800001EB42119DF8052041F8220000208DF844
:103390000700FFE79DF9070002B0704783B08DF882
:1033A00007009DF807000146009140B1FFE7009833
:1033B00001280AD0FFE7009802280CD011E042F261
:1033C000D850C2F2000002900EE042F21C60C2F23D
:1033D0000000029008E042F29450C2F20000029015
:1033E00002E000200290FFE7029803B0704700005F
:1033F00080B582B00190019800680068C00600287E
:103400002AD5FFE7FFE700200090019800680068D8
:10341000009001980068406800900098FFE70198CC
:1034200016F016F800EBC00140F27070C2F2000016
:1034300000EB8100006A70B1FFE7019816F008F810
:1034400000EBC00140F27070C2F2000000EB81009E
:10345000006A8047FFE7FFE702B080BD82B08DF8C9
:1034600006008DF805100092009820B9FFE7FE20B5
:103470008DF8070012E000989DF8061001EBC102DC
:1034800040F27071C2F2000101EB82019DF805204B
:1034900041F8220000208DF80700FFE79DF90700A2
:1034A00002B0704783B080B585B009930892079148
:1034B00003900020ADF8060007A80290039A029B33
:1034C00049F29450C2F2000040F2FF311EF0C2FEF9
:1034D000ADF80600BDF8060001280CDBFFE7BDF8DB
:1034E000061049F29450C2F2000000F02FF80020BC
:1034F0008DF8130003E0FE208DF81300FFE79DF91F
:10350000130005B0BDE8804003B0704749F2145085
:10351000C2F200000078704780B582B00090009839
:1035200020B9FFE7FE208DF807000BE0009841F27C
:10353000E441C2F20001086000F076FC00208DF842
:103540000700FFE79DF9070002B080BD80B582B09B
:103550000190ADF8021000208DF80100FFE70198FE
:10356000BDF8021000F086FC48B1FFE79DF80100AD
:1035700001308DF801000A20FFF766FB00E005E04E
:10358000FFE79DF801000328E9DBFFE7002002B018
:1035900080BD0000FFE7FEE780B541F60020C2F2E3
:1035A000000005F073FC80BD80B541F60020C2F23A
:1035B000000005F06BFC80BD80B541F62820C2F20A
:1035C000000005F063FC80BD80B541F62820C2F202
:1035D000000005F05BFC80BD80B582B0002001904A
:1035E000FFF7EEFA019942F65842C2F20002009249
:1035F00002F11C0305F040FB0099019B41F2E840F9
:10360000C2F200000068D0F8D8001A461AF030FB69
:1036100002B080BD80B582B001200090FFF7D0FAE3
:10362000009942F67C42C2F20002019202F11C03B0
:1036300005F022FB019941F2E840C2F20000006867
:10364000D0F8D80000231A461AF012FB02B080BD51
:1036500083B0029001918DED000A0299002008715B
:1036600000980199086003B07047000080B588B0E9
:10367000079006910798006805909DED050A9FED5B
:10368000181A20EE010ABDEEC00A10EE100AADF8BD
:10369000120042F6A041C2F2000101914FF4047001
:1036A0000860002003908860C860082008619DF8C9
:1036B0001320084600F8182F0290BDF81200487633
:1036C0000698D0F8C400C078FFF77AFA0199029AF8
:1036D000069BD43305F00EF8039808B080BD00BFF8
:1036E0000000C84282B0019000910098008800EE6E
:1036F000100AB8EEC00A9FED151A80EE010A019873
:1037000080ED000A0098408800EE100AB8EEC00A6A
:1037100080EE010A019880ED010A0098808800EE91
:10372000100AB8EEC00A80EE010A019880ED020A84
:103730000098C08800EE100AB8EEC00A80EE010AB8
:10374000019880ED030A02B0704700BF0000C84234
:1037500083B001900091019820B9FFE700208DF817
:103760000B000AE00198006800990840401AB0FA7E
:1037700080F040098DF80B00FFE79DF80B0003B0C7
:103780007047000083B001900091019820B9FFE7D5
:10379000FE208DF80B0008E0009A0199086890431C
:1037A000086000208DF80B00FFE79DF90B0003B0C7
:1037B0007047000082B000900098006846F6000153
:1037C000C4F20001884204D1FFE701208DF8070010
:1037D00010E00098006846F20041C4F200018842FF
:1037E00004D1FFE700208DF8070003E003208DF8E7
:1037F0000700FFE79DF8070002B0704780B592B060
:1038000010900F91109820B9FFE7FE208DF8470027
:103810007DE042F29D60C2F200000078C00720B156
:10382000FFE7FD208DF8470071E01AF0E3FB43F25B
:103830003031C2F20001086020B9FFE7FE208DF8A8
:10384000470064E020202421002204921AF090F91D
:103850001099C1F8D8000F981099C1F8C40005A8B4
:1038600002902821FCF709FD04980A900590069023
:103870000B90012103910C91079008900D910E215E
:1038800001910E910990FFF79BF9029905F056F806
:103890000498FFF795F906F003F9049843F2D9521A
:1038A000C0F600020621FFF7ABF90498FFF788F98C
:1038B000022104F0E3FE019903980A910990FFF7B1
:1038C0007FF9029905F03AF80398FFF779F906F0C5
:1038D000E7F8039843F21562C0F600020821FFF7EB
:1038E0008FF90398FFF76CF9102104F0C7FE0399D4
:1038F0000498109A41F2E843C2F200031A6042F2BF
:103900009D62C2F2000211708DF84700FFE79DF939
:10391000470012B080BD000080B590B08DF83E0029
:103920000E910D920E9820B9FFE7FE208DF83F0012
:1039300022E19DF83E000146079158B1FFE7079844
:103940000138022869D3FFE7079803380228C0F03E
:10395000A9800CE10E9890ED000A9FED891A20EEE7
:10396000010ABDEEC00A10EE100AADF832000E9842
:1039700090ED010A20EE010ABDEEC00A10EE100A19
:10398000ADF830000E9890ED020A20EE010ABDEE6F
:10399000C00A10EE100AADF82E000E9890ED030A42
:1039A00020EE010ABDEEC00A10EE100AADF82C00A0
:1039B00042F6A041C2F2000105914FF40070086088
:1039C00000208860C860082008619DF83320084600
:1039D00000F8182F0690BDF8320048769DF83100A7
:1039E0008876BDF83000C8769DF82F000877BDF8BE
:1039F0002E0048779DF82D008877BDF82C00C877F9
:103A00000D98D0F8C4000078FFF7DAF80599069A07
:103A10000D9BC83304F06EFEAAE00E9890ED040AE8
:103A20009FED591A20EE010ABDEEC00A10EE100AF1
:103A3000ADF82A000E9890ED050A20EE010ABDEEC1
:103A4000C00A10EE100AADF8280042F6A041C2F2FA
:103A50000001039140F2FF20086000208860C860E8
:103A600008220A619DF82B300A4602F8183F04929A
:103A7000BDF82A204A769DF829208A76BDF82820AC
:103A8000CA76087748778877C8770D98D0F8C40049
:103A90004078FFF795F80399049A0D9BCC3304F016
:103AA00029FE65E00E9890ED070A9FED351A20EE8D
:103AB000010ABDEEC00A10EE100AADF826000E98FD
:103AC00090ED080A20EE010ABDEEC00A10EE100AC1
:103AD000ADF824000E9890ED090A20EE010ABDEE23
:103AE000C00A10EE100AADF822000E9890ED0A0AF6
:103AF0009FED241A20EE010ABDEEC00A10EE100A56
:103B0000ADF8200042F6A041C2F20001019140F25E
:103B1000FF10086000208860C860082008619DF8D8
:103B20002720084600F8182F0290BDF82600487696
:103B30009DF825008876BDF82400C8769DF82300FE
:103B40000877BDF8220048779DF821008877BDF8F6
:103B50002000C8770D98D0F8C4008078FFF730F8BF
:103B60000199029A0D9BD03304F0C4FD00E0FFE7F9
:103B700000208DF83F00FFE79DF93F0010B080BDA9
:103B80000000804600401C460060EA4683B0029078
:103B9000019101980178407840EA0120ADF80200D7
:103BA00001980179407940EA0120ADF80000BDF8A4
:103BB000020000EE100AB8EEC00A9FED191A80EE5E
:103BC000010A9FED181A20EE010A029880ED000A02
:103BD00001988178C07840EA012000B200EE100A16
:103BE000B8EEC00A029880ED010ABDF9000000EBB2
:103BF0008000800000EE100AB8EEC00A9FED0A1A9D
:103C000080EE010A029880ED020A0198807900EEA8
:103C1000100AB8EE400A029880ED030A03B070471C
:103C200000000046DB0FC9400000804680B586B02A
:103C300004900391049820B9FFE7FE208DF8170047
:103C400089E0039820B9FFE7FE208DF8170082E095
:103C5000039800680190A0F20120042817D3FFE721
:103C60000198A0F20520042828D3FFE70198A0F2CC
:103C7000092002283AD3FFE7019840F21121884237
:103C80004CD0FFE70198B0F5207F53D05EE0039859
:103C90000068A0F2012002900498029900EB011044
:103CA000043003991C31FFF771FF0299012000FADB
:103CB00001F2049908681043086048E0039800681E
:103CC000A0F2052002900298811D012000FA01F265
:103CD00004990868104308600498029900EB0110E9
:103CE000643003991C31FFF751FF30E003980068FE
:103CF000A0F2092002900298011D012000FA01F2B1
:103D000004990868104308600498029900EB0110B8
:103D1000443003991C31FFF739FF18E00499086813
:103D200040F4007008600498AC3003991C31FFF730
:103D3000D9FC0CE00499086840F48060086004989D
:103D4000BC3003991C3100F00BF800E0FFE70020C5
:103D50008DF81700FFE79DF9170006B080BD000041
:103D600082B0019000910098017842788078000438
:103D700040EA0220084400EE100AB8EEC00A9FEDA7
:103D80000A1A80EE010A019880ED000A0098C078B6
:103D90000199087100990879497940EA012001994F
:103DA000C88002B0704700BF00007A4484B08DF82C
:103DB0000F000291ADF806209DF80F00014600911A
:103DC00023281DD80099DFE801F012131415161BE3
:103DD0001B1B1B1B1B1B1B1B1B1B1B1B1B1B1B1B33
:103DE0001B1B1B1B1B1B1B1B1B1B1718191A08E07B
:103DF00007E006E005E004E003E002E001E000E0A7
:103E0000FFE7002004B070470020704780B541F202
:103E1000A060C2F2000049F21451C2F2000116F093
:103E200045FC002080BD000080B541F2A060C2F2D8
:103E3000000016F0F5FB002080BD000080B582B0C8
:103E40000190009141F2E440C2F2000000680121BB
:103E500019F0F0FF002002B080BD000083B0029096
:103E600001918DF8032000208DF802009DF90200D9
:103E700003B0704780B586B00490ADF80E100020F6
:103E80008DF80D0041F2A060C2F20000D0F8BC0233
:103E900002900298D0F8140220B1FFE701208DF8BB
:103EA000170013E00499BDF80E2041F2A060C2F2A1
:103EB0000000019016F014FC019816F0FFFC8DF83C
:103EC0000D009DF80D008DF81700FFE79DF8170015
:103ED00006B080BD80B588B0069005918DF813209E
:103EE00005989DF8131000F08DF88DF812000598D4
:103EF0009DF8131000F078F88DF811009DF812006D
:103F000010280DD1FFE70698007F00F001008DF822
:103F100010000598807A00F001008DF80F0025E070
:103F20009DF8120011280DD1FFE70698407F00F0A0
:103F300001008DF810000598C07A00F001008DF89E
:103F40000F0012E00698C08B9DF81210C84000F0D8
:103F500001008DF81000059840889DF81210C840A7
:103F600000F001008DF80F00FFE7FFE79DF811005A
:103F70000146029140B1FFE70298012817D0FFE700
:103F80000298022824D02AE09DF810100020C907CA
:103F9000019031B1FFE79DF80F0080F00100019022
:103FA000FFE7019800F001008DF81F0017E09DF871
:103FB00010100020C907009021B9FFE79DF80F00FD
:103FC0000090FFE7009800F001008DF81F0006E068
:103FD0009DF8100000F001008DF81F00FFE79DF82C
:103FE0001F0008B080BD000082B001908DF8031062
:103FF000019800699DF8031000EB4100007A02B0BF
:104000007047000082B001908DF80310019800699C
:104010009DF8031000EB4100407A02B070470000A9
:1040200081B000900098407800F0010001B0704726
:1040300083B001900091019820B9FFE7FF208DF82F
:104040000B000FE0009820B9FFE7FF208DF80B0070
:1040500008E00199002008700099019A11618DF81B
:104060000B00FFE79DF90B0003B0704783B0019090
:104070008DF803109DF80300102807D1FFE7019881
:10408000007F00F001008DF80B0015E09DF80300A3
:10409000112807D1FFE70198407F00F001008DF85B
:1040A0000B0009E00198C08B9DF80310C84000F098
:1040B00001008DF80B00FFE79DF80B0003B070477F
:1040C00084B0029001918DED000A029820B9FFE7BB
:1040D000FF208DF80F0025E0019820B9FFE7FF20B1
:1040E0008DF80F001EE0029800680199886202981E
:1040F00040680199C8620298007EC00748B1FFE796
:104100000199022081F834000199012081F83600DC
:1041100004E00199012081F83400FFE700208DF8C8
:104120000F00FFE79DF90F0004B0704780B584B021
:10413000029001918DED000A029820B9FFE7FF205F
:104140008DF80F0056E0019820B9FFE7FF208DF8A9
:104150000F004FE002980421FFF788FF80B1FFE7CE
:1041600002980521FFF782FF50B1FFE70298062170
:10417000FFF77CFF20B1FFE7019901200870FFE7FE
:1041800002980421FFF772FF80B1FFE70298052132
:10419000FFF76CFF50B1FFE702980721FFF766FFBA
:1041A00020B1FFE7019900200870FFE70298407DE9
:1041B00020B1FFE70298007D20B9FFE7019800F0E9
:1041C00023FA13E001980078C00738B1FFE702989E
:1041D00001999DED000A00F011F806E0029801999E
:1041E0009DED000A00F08CF9FFE7FFE700208DF855
:1041F0000F00FFE79DF90F0004B080BD80B584B0CB
:10420000039002918DED010A0299012081F82400AA
:104210000398B0F9160000EE100AB8EEC00A9DED42
:10422000011A20EE010A0298016991ED001A20EEB0
:10423000010A80ED0A0A0398B0F91800404200EE26
:10424000100AB8EEC00A9DED011A20EE010A02988C
:10425000016991ED001A20EE010A80ED0B0A029827
:104260000022C26102988261029880F83820039887
:104270000299FFF72FFE58B1FFE70298016991ED0F
:10428000091A90ED070A30EE010A80ED070AFFE7F0
:10429000039802990122FFF71DFE58B1FFE702982B
:1042A000016991ED091A90ED070A30EE410A80ED9F
:1042B000070AFFE7039802990222FFF70BFE58B1A5
:1042C000FFE70298016991ED091A90ED060A30EEB8
:1042D000410A80ED060AFFE7039802990322FFF7DF
:1042E000F9FD58B1FFE70298016991ED091A90EDC7
:1042F000060A30EE010A80ED060AFFE703980299EC
:104300000422FFF7E7FDA8B1FFE70298016991EDEC
:104310000A1A90ED060A20EE010A80ED060A0298BC
:10432000016991ED0A1A90ED070A20EE010A80ED6D
:10433000070AFFE7039802990522FFF7CBFDA8B112
:10434000FFE70298016991ED0B1A90ED060A20EE45
:10435000010A80ED060A0298016991ED0B1A90EDB1
:10436000070A20EE010A80ED070AFFE70398029989
:104370000622FFF7AFFD48B1FFE70299022081F85E
:1043800034000299012081F8360008E002990220E9
:1043900081F834000299002081F83600FFE7039885
:1043A00002990722FFF796FDB0B1FFE7029991F855
:1043B0003500013081F83500029991F835004AF650
:1043C000AB22CAF6AA22A0FB0232520802EB42023A
:1043D000801A81F83500FFE7039802990B22FFF756
:1043E00079FD38B1FFE7029904200875029902208F
:1043F0004875FFE7039802990A22FFF76BFD40B169
:10440000FFE7029991F837200120904381F83700A7
:10441000FFE7039802990822FFF75CFD20B3FFE74E
:104420000298007B02280BD1FFE702983930042163
:1044300000F0F8F80299002048700299087312E021
:104440000298007B012801D1FFE70BE00298393088
:10445000032100F0E7F80299022008730299012075
:104460004870FFE7FFE7FFE7039802990922FFF78B
:1044700031FDD8B1FFE70298007B01280BD1FFE79F
:10448000029900204870029908730298393002217D
:1044900000F0C8F809E00298012101730298417008
:1044A0000298393000F0BEF8FFE703E002990020DF
:1044B0004870FFE7039802990C22FFF70BFD28B123
:1044C000FFE70299012081F83800FFE7039802997D
:1044D0000D22FFF7FFFC20B1FFE7029902200875CB
:1044E000FFE70398C08B029948800299039AD2F89B
:1044F0001600D2F81A208A60486004B080BD00001F
:1045000085B0049003918DED020A0498407D014628
:104510000191032817D80199DFE801F011020A067A
:104520000399012008750EE00399022008750AE03E
:1045300003990420087503990020487503E0039946
:1045400000200875FFE70498007D014600910328CC
:1045500031D80099DFE801F02702170A03990120FA
:1045600081F82400039981F8340024E003990120A4
:1045700081F824000399002081F836000399022075
:1045800081F8340017E00399012081F82400039A90
:10459000022182F83410039A002182F83510039921
:1045A00081F8360007E00399002081F82400039980
:1045B00081F83400FFE70498006803998861049843
:1045C00040680399C861049890ED020A9DED021AB3
:1045D00020EE010A0398016991ED011A20EE010A0B
:1045E00080ED0A0A049890ED030A9DED021A20EE70
:1045F000010A0398016991ED011A20EE010A80ED8C
:104600000B0A05B07047000081B0009000990020AF
:104610000875009981F82400009981F8340001B0F0
:104620007047000083B001908DF80310019820B905
:10463000FFE7FF208DF80B001BE00198C0780228EF
:1046400006DCFFE70198C078B0F1FF3F04DCFFE72C
:10465000FF208DF80B000CE09DF803000199CA784B
:1046600088540199C8780130C87000208DF80B007B
:10467000FFE79DF90B0003B07047000081B0ADF873
:1046800002008DF80110BDF802109DF801004840AD
:10469000C2B244F6E010C0F6020030F8120080EA20
:1046A000112001B07047000080B584B003900291E2
:1046B000ADF80620FFE70298411E029158B1FFE7CE
:1046C000BDF8060003994A1C03920978FFF7D6FF4C
:1046D000ADF80600EFE7BDF8060004B080BD0000AD
:1046E00080B584B0029001910198012804D8FFE7B9
:1046F00000208DF80F001BE00298019902394FF657
:10470000FF72FFF7D1FFADF80200BDF80200029A78
:10471000019901F001031A4421F00101114431F81B
:10472000021C401AB0FA80F040098DF80F00FFE734
:104730009DF80F0004B080BD83B0029001918DF808
:104740000320FFE70198411E019178B1FFE79DF832
:10475000030002994A1C02920978414044F6E03075
:10476000C0F60200405C8DF80300EBE79DF8030003
:1047700003B0704780B584B0029001910198012880
:1047800004D8FFE700208DF80F0015E0029801998A
:104790000139FF22FFF7D0FF8DF803009DF80300D9
:1047A000029A0199114411F8011C401AB0FA80F0E4
:1047B00040098DF80F00FFE79DF80F0004B080BDA1
:1047C00085B002A900910146009880ED010AC0ED74
:1047D000000A8DF8071090ED010AB5EE400AF1EEDF
:1047E00010FA03D1FFE7002004906DE09DF8070068
:1047F000C007A0B3FFE7009890ED010AB2EE0E1AD1
:10480000B4EE410AF1EE10FA06D1FFE74FF20000D4
:10481000C4F29150049057E0009890ED010AB3EE75
:10482000021AB4EE410AF1EE10FA06D1FFE748F29F
:104830000000C4F2A250049046E0009890ED010AF6
:10484000B3EE0E1AB4EE410AF1EE10FA06D1FFE70C
:104850004BF20000C4F2E550049035E022E00098ED
:1048600090ED010AB2EE041AB4EE410AF1EE10FA2C
:1048700006D1FFE741F20000C4F28B50049023E020
:10488000009890ED010AB3EE001AB4EE410AF1EE81
:1048900010FA06D1FFE744F20000C4F2B5500490CC
:1048A00012E0FFE7009890ED010A9FED0A1A20EE52
:1048B000010A90ED001A9FED082A21EE021A80EEFF
:1048C000010A80ED020AFFE7009890ED020A05B0A8
:1048D000704700BF00007042DB0FC94080B584B054
:1048E00003900291019202980078012805D0FFE719
:1048F00002988068019908600CE0029890ED010A26
:10490000D0ED020A90ED031A0FF03CFD019880ED06
:10491000000AFFE70399012008710398D0ED020A0D
:1049200090ED030AB2EE081A00F0BAF8039880ED91
:10493000000A04B080BD000082B00190009101988F
:10494000006800990860019800790099087102B028
:104950007047000084B08DED030A9DED030A20EE40
:10496000000A8DED010A9DED010A9DED031A20EE6E
:10497000010A8DED000A9DED030A9FED3E1AB4EE8B
:10498000410AF1EE10FA03DAFFE70020029053E04B
:104990009DED030A9FED381AB4EE410AF1EE10FACC
:1049A0001DDAFFE79DED000A9FED391A20EE010A9E
:1049B0009DED011A9FED372A21EE021A30EE010A11
:1049C0009DED031A9FED342A21EE021A30EE010A02
:1049D0009FED321A30EE010A8DED020A2BE09DEDBB
:1049E000030A9FED261AB4EE410AF1EE10FA1DDA21
:1049F000FFE79DED000A9FED221A20EE010A9DEDD2
:104A0000011A9FED202A21EE021A30EE010A9DEDD7
:104A1000031A9FED1D2A21EE021A30EE010A9FEDC6
:104A20001B1A30EE010A8DED020A03E04FF07E50B2
:104A30000290FFE7FFE7FFE79DED020AB5EE400AAF
:104A4000F1EE10FA03DAFFE7002002900EE09DED90
:104A5000020AB7EE001AB4EE410AF1EE10FA04DDD4
:104A6000FFE74FF07E500290FFE7FFE79DED020A5F
:104A700004B0704700009C413333AF410000CC418B
:104A800061E0B93C46B6D3BF295C21423333A4C3AD
:104A90001399B93BFB5CADBEE17AD84014AE34C289
:104AA00084B08DED030ACDED020A8DED011A9DED66
:104AB000030A9DED012A30EE420A9DED021A31EE05
:104AC000421A80EE010A8DED000A9DED000AB5EE56
:104AD000400AF1EE10FA03DAFFE7002000900EE042
:104AE0009DED000AB7EE001AB4EE410AF1EE10FA9D
:104AF00004DDFFE74FF07E500090FFE7FFE79DEDFC
:104B0000000A04B07047000080B588B08DED070A38
:104B1000CDED060A05909DED050AB8EE400A10EEAF
:104B2000100AFBF737FD41EC100B9FED2B1B53ECEC
:104B3000112B51EC100BFBF78BFC41EC100B51ECE3
:104B4000100BFBF73AFD00EE100A1EF0CDF99FEDB9
:104B5000261A20EE010A10EE100AFBF71BFD41ECAD
:104B6000100B51EC100B9FED1E0B52EC103BD20FB3
:104B700062F3DF7141EC100B8DED020B0798FBF730
:104B800009FD9DED021B41EC100B51EC110B53EC98
:104B9000102BFBF7B6FB41EC100B51EC100BFBF7A5
:104BA0000CFD04909DED040A9FED101AB4EE410A2D
:104BB000F1EE10FA05DDFFE79DED060A8DED010A25
:104BC00004E09DED040A8DED010AFFE79DED010A69
:104BD00008B080BD00BF00BFFCA9F1D24D62503FBC
:104BE0000000000000000000CDCC4C3ECDCC4C3F7E
:104BF00080B58EB007AB05930C900B910A920C9880
:104C000020B9FFE7FE208DF8370067E10B9820B947
:104C1000FFE7FE208DF8370060E10A990C980268E2
:104C2000891A00EE101AB8EE400A9FEDAE1A80EE17
:104C3000010A80ED010A0A980C9908600C980B99FA
:104C400009780A9A00F02EFB0C98007C014604912A
:104C500000B3FFE7049801280DD0FFE7049802385D
:104C6000032817D3FFE7049805280AD0FFE7049824
:104C700006280FD04CE00C99002048610C998861FF
:104C800046E00B9840680C9948610B9840680C9975
:104C900088613DE005980C9991ED080AC96891ED8D
:104CA000001A30EE410A80ED020A90ED020A1DF072
:104CB000D7FF059880ED010A90ED020A1EF014F965
:104CC000059880ED000A90ED010A0B9991ED011A0B
:104CD00091ED022A20EE010A90ED001A21EE021A4F
:104CE00030EE410A0C9981ED050A90ED000A0B990E
:104CF00091ED011A91ED022A20EE010A90ED011AC0
:104D000021EE021A30EE010A0C9880ED060AFFE748
:104D10000C98007C01460391062848D80399DFE8E7
:104D200001F00404081A300408000C990020C8613E
:104D30003DE00C9901F13800CA6892ED000AD1ED0E
:104D4000011AD1ED080A9FED6B1A0FF07DF80C984F
:104D500080ED070A2BE00C9901F13800CA6892ED4A
:104D6000000A9FED631A30EE010AD1ED011AD1ED70
:104D7000080A9FED601A0FF067F80C9880ED070A9B
:104D800015E00C9890ED0B0A8DED020A0A989FED44
:104D9000560ADFED560AFFF7B7FEB0EE401A9DED5A
:104DA000020A20EE010A0C9880ED070AFFE70C9B2F
:104DB00003F1120003F114011A6B93F911309FED06
:104DC0004E0A0EF0C5FC00208DF81B00FFE79DF891
:104DD0001B000C9991F9111088427BDAFFE70C98BF
:104DE000416A406F9DF81B2000EB421001EB8201ED
:104DF00091ED000A0DF018FC0C98406A9DF81B100C
:104E000000EB810080ED000A0C98007C01460191C6
:104E1000E0B3FFE701980138052804D3FFE70198C4
:104E2000062821D03AE00C99486B9DF81B30C3EB63
:104E3000031200EB82000A6B02EB830292ED000A80
:104E40004A6A02EB8302D2ED000AD1ED011A9FED0E
:104E5000291A0EF0F9FF0C98C06F9DF81B1000EB9B
:104E6000810080ED000A19E00C989DF81B10026B80
:104E7000C06F02EB810292ED000A9FED201A80EED6
:104E8000010A00EB810080ED000A07E00C98C16F79
:104E90009DF81B20002041F82200FFE70C999DF8A7
:104EA0001B20886FC96F00EB421001EB820191ED6E
:104EB000000A0DF0B9FB0C98C06F9DF81B1000EBB9
:104EC000810080ED000AFFE79DF81B0001308DF89E
:104ED0001B007CE700208DF83700FFE79DF93700C5
:104EE0000EB080BD00007A449A99193FCDCC4C3F5A
:104EF000AB611C3F0000000000C0DA4500A00C467A
:104F000083B00290019100208DF80300FFE79DF827
:104F10000300029991F91110884210DAFFE7029814
:104F2000C06F9DF8032050F82200019941F822003B
:104F3000FFE79DF8030001308DF80300E7E703B0B9
:104F40007047000082B0019000910198007C0099A8
:104F50000870019890ED080AC06890ED001A30EED4
:104F6000410A009880ED010A02B0704780B58AB00E
:104F700005AB03930346039808930791069280EDCF
:104F8000000A089820B9FFE7FE208DF827001CE1F1
:104F9000079808998860089900200874069808996D
:104FA000C860079890F84C00C00728B1FFE7089840
:104FB000C06800F0DBFAFFE70898806800780146D7
:104FC0000291062832D80299DFE801F0040B12188A
:104FD0001F2C250008990420487400208DF8130028
:104FE00024E008990420487401208DF813001DE086
:104FF0000899022048748DF8130017E008990420DE
:10500000487403208DF8130010E0089904204874B8
:105010008DF813000AE008990120487405208DF8E6
:10502000130003E0FC208DF82700CEE0089890F9EB
:1050300011008000FEF794F8089948620898406AC9
:1050400008B9FFE7A5E0089890F911008000FEF785
:1050500087F8089988620898806A08B9FFE798E09D
:10506000089890F911008000FEF77AF80899086313
:105070000898006B08B9FFE78BE0089890F91100D9
:10508000C0EB00108000FEF76BF8089948630898A1
:10509000406B08B9FFE77CE0089890F911008000A8
:1050A000FEF75EF80899C8670898C06F08B9FFE76F
:1050B0006FE0089890F911004001FEF751F8089947
:1050C00048670898406F08B9FFE762E0089890F9D0
:1050D00011004001FEF744F8089988670898806F2E
:1050E00008B9FFE755E000208DF81200FFE79DF8B2
:1050F0001200089991F91110884233DAFFE7039AF8
:1051000008988168406B9DF81230C3EB031300EBE5
:10511000830092ED000A0A1D00210FF00DF8039A9A
:1051200008988168406F9DF8123000EB431092EDB3
:10513000000AD1ED110A0DF0D3FA039A089881689C
:10514000806F9DF8123000EB431092ED000AD1ED14
:10515000120A0DF0C5FAFFE79DF8120001308DF834
:105160001200C4E7039A089901F1380092ED000A91
:10517000896801F12402002101910EF0DDFF0898F9
:1051800012309DF813100EF035FC01988DF82700B1
:105190001BE00898406AFDF7F7FD0898006BFDF7E3
:1051A000F3FD0898406BFDF7EFFD0898C06FFDF721
:1051B000EBFD0898406FFDF7E7FD0898806FFDF75D
:1051C000E3FDFE208DF82700FFE79DF927000AB0D8
:1051D00080BD000080B584B0039002910192002050
:1051E000009001980078012805D0FFE70020C4F264
:1051F000FA40009042E002980079012833D1FFE79D
:10520000029890ED000A9FED231AB4EE410AF1EEE8
:1052100010FA28DDFFE7029890ED000AB7EE001AB9
:10522000B4EE410AF1EE10FA05DDFFE70020CBF6FF
:105230008070009016E0019890ED010A029890EDC0
:10524000001A9FED152A31EE021A9FED142A81EE05
:10525000021A9FED132A21EE021A30EE010A8DED9B
:10526000000AFFE709E0019890ED010AD0ED020A7B
:105270000FF038F98DED000AFFE7FFE79DED000A1A
:10528000039A516AD06F92F911200FF0B7F80020FD
:1052900004B080BD9A99993E9A9999BE3333333FB1
:1052A0000000C84280B586B004908DF80F100292BD
:1052B000049820B9FFE7FE208DF8170066E09DF8FE
:1052C0000F000499097C884204D1FFE700208DF883
:1052D00017005BE09DF80F0004281CD1FFE704983D
:1052E000007C042817D0FFE70298FAF7A5FFFAF729
:1052F00099FF00EBD07121F00101411A0120002932
:1053000018BF4FF0FF3000EE100AB8EEC00A049844
:1053100080ED0B0AFFE700208DF80700FFE79DF8FE
:105320000700049991F91110884227DAFFE70498E1
:10533000406B9DF80710C1EB011100EB81000EF0EE
:10534000C7FF0498406F9DF8071000EB41109FEDD8
:10535000110A8DED000A0DF061FA9DED000A049826
:10536000806F9DF8071000EB41100DF057FAFFE732
:105370009DF8070001308DF80700D0E79DF80F0079
:105380000499087400208DF81700FFE79DF91700B5
:1053900006B080BD0000000084B002900191029828
:1053A00020B9FFE7FE208DF80F0048E0019820B9F2
:1053B000FFE7FE208DF80F0041E00298806890F82A
:1053C0004C00C00758B1FFE7019890ED111A9FED0E
:1053D0001E0A30EE410A029880ED080A04E00198A6
:1053E000406C02990862FFE700208DF80300FFE798
:1053F0009DF80300029991F9111088421BDAFFE72A
:1054000001989DF8032000EB021080680299496A18
:1054100041F8220001989DF8032000EB0210C068BB
:105420000299896A41F82200FFE79DF803000130E4
:105430008DF80300DCE700208DF80F00FFE79DF9F1
:105440000F0004B0704700BFDB0FC94084B0039069
:105450008DED020ACDED010A039890ED000A9DED55
:10546000021A30EE010A8DED000A9DED010AB5EE3B
:10547000400AF1EE10FA26DDFFE79DED000A9DEDF2
:10548000011AB4EE410AF1EE10FA09DBFFE79DEDD7
:10549000011A9DED000A30EE410A8DED000A11E07F
:1054A0009DED000AB5EE400AF1EE10FA09DAFFE7C9
:1054B0009DED011A9DED000A30EE010A8DED000A06
:1054C000FFE7FFE7FFE700980399086004B0704723
:1054D00085B08DED040ACDED030A8DED021A9DED28
:1054E000040A9DED031A30EE410A8DED010A9DED8F
:1054F000020AB5EE400AF1EE10FA32DDFFE79DED4B
:10550000020AB0EE001A80EE010A8DED000A9DED50
:10551000010A9DED001AB4EE410AF1EE10FA09DD20
:10552000FFE79DED021A9DED010A30EE410A8DED77
:10553000010A15E09DED010A9DED001AB1EE411A38
:10554000B4EE410AF1EE10FA09DAFFE79DED021A16
:105550009DED010A30EE010A8DED010AFFE7FFE73C
:10556000FFE79DED010A05B07047000081B0009093
:10557000009890ED001A9FED040A30EE410A80ED8C
:10558000000A01B0704700BFDB0FC94083B0029032
:105590008DED010ACDED000A029890ED000A9DED17
:1055A000001AB4EE410AF1EE10FA04DDFFE70098AC
:1055B00002990860FFE7029890ED000A9DED011A3C
:1055C000B4EE410AF1EE10FA04DAFFE7019802990D
:1055D0000860FFE703B0704780B5B4B032903191F6
:1055E0003092329818B9FFE700203390FDE13198EE
:1055F000013831900020ADF84E0040F21060C2F248
:105600000000007801461291072800F2C881129923
:10561000DFE811F008001A002C0097003601610144
:10562000A301B4013298319945F66132C0F6020205
:105630001CF0E2FD40F21061C2F200010878013076
:10564000087001203390D0E13298319945F68F22CD
:10565000C0F602021CF0D0FD40F21061C2F200015F
:1056600008780130087001203390BEE143F27410D5
:10567000C2F200001190C06818F0ACFD1198806B68
:1056800014A90022052318F013FAC0B1FFE73298DD
:10569000319945F66122C0F602021CF0ADFD40F2E0
:1056A0001061C2F200010720087043F27410C2F2C8
:1056B0000000C06818F06EFD0120339095E143F2C0
:1056C0007410C2F20000C06818F064FD14A8FCF762
:1056D00019FF90B1FFE73298319945F63732C0F69D
:1056E00002021CF089FD40F21061C2F2000108784C
:1056F000013008700120339077E140F21160C2F26E
:105700000000017801310170007802280FDCFFE70A
:105710003298319945F6AD22C0F602021CF06CFDBC
:1057200040F21061C2F200010120087006E040F270
:105730001061C2F2000107200870FFE701203390DA
:1057400053E13298319945F68232C0F602021CF0DC
:1057500053FD17A8109000F01BFF1098002129910D
:105760002A912B9100F0D2FFFFE7BDF84E00B0F573
:105770007A7F4BDAFFE743F27410C2F20000806BCD
:1057800014A90F910022052318F092F901460F98F1
:10579000B1FA81F149098DF84D10FCF7B3FE8DF88F
:1057A0004C009DF84D00C00778B3FFE79DF84C0012
:1057B000C00750B3FFE79DED141A40F21460C2F227
:1057C000000090ED000A30EE010A80ED000A9DED28
:1057D000151A40F21860C2F2000090ED000A30EE97
:1057E000010A80ED000A9DED161A40F21C60C2F21B
:1057F000000090ED000A30EE010A80ED000ABDF8CD
:105800004E000130ADF84E00FFE7AEE7BDF84E00A8
:1058100000EE100AB8EE401A40F21460C2F2000026
:1058200090ED000A80EE010A80ED000ABDF84E00FE
:1058300000EE100AB8EE401A40F21860C2F2000002
:1058400090ED000A80EE010A80ED000ABDF84E00DE
:1058500000EE100AB8EE401A40F21C60C2F20000DE
:1058600090ED000A80EE010A80ED000A40F210611E
:10587000C2F2000108780130087001203390B4E0D2
:105880003298319945F60932C0F602021CF0B4FC98
:1058900017A80E9000F07CFE0E9840F21461C2F240
:1058A00000010968299140F21861C2F200010968FB
:1058B0002A9140F21C61C2F2000109682B9100F0AC
:1058C00025FF40F21061C2F2000108780130087033
:1058D0000120339089E032980C9031980D9040F27D
:1058E0001460C2F200000068FAF754FE41EC100B9D
:1058F0008DED0A0B40F21860C2F200000068FAF762
:1059000049FE41EC100B8DED080B40F21C60C2F219
:1059100000000068FAF73EFE9DED081B9DED0A0BA6
:1059200002460C980B460D9943EC122B6A4682ED09
:10593000042B82ED021B82ED000B45F6C532C0F64A
:1059400002021CF059FC40F21061C2F2000108781A
:10595000013008700120339047E03298319945F6C4
:10596000F622C0F602021CF047FC40F21061C2F2BF
:105970000001082008700120339036E032983199F8
:1059800045F67A22C0F602021CF036FC40F21061A5
:10599000C2F20001082008700120339025E040F297
:1059A0001461C2F2000100200790086040F2186103
:1059B000C2F20001086040F21C61C2F200010860FE
:1059C00040F21161C2F2000108703298319945F637
:1059D0009542C0F602021CF00FFC079840F21061DD
:1059E000C2F2000108703390FFE7339834B080BDF5
:1059F00080B5B0B02E902D912C922E9818B9FFE75B
:105A000000202F9060E22D9801382D902C980121D4
:105A10002BAA01F081FC28902C9802212AAA01F0DF
:105A20007BFC27902C98032129AA01F075FC269075
:105A300028982B9A45F29B31C0F60201FAF752FCE6
:105A4000A0B9FFE72E982D9945F6E152C0F6020263
:105A500045F26863C0F602031CF0CEFB40F2206101
:105A6000C2F20001002008702F902DE228982B9A96
:105A700045F6FF51C0F60201FAF734FC00285BD16D
:105A8000FFE7279818B9FFE7269808B1FFE70BE270
:105A900040F22060C2F20000007801460A9120B175
:105AA000FFE70A98012810D045E02E982D9945F679
:105AB0001452C0F602021CF09FFB40F22061C2F2B9
:105AC0000001012008702F90FEE10DA809906421CB
:105AD000FAF7D3FB45F25440C0F60200089000F0FC
:105AE0009DFD189045F25740C0F60200069000F068
:105AF000D7FD069A014609981791142107911CF0C9
:105B00007BFB0799089A099814301CF075FB0998DB
:105B100000F0FCFD2E982D9945F6D042C0F6020209
:105B20001CF06AFB40F22061C2F200010220087002
:105B300001202F90C8E19DE128982B9A45F610612D
:105B4000C0F60201FAF7CEFB002840F0CF80FFE755
:105B5000279818B1FFE7269808B1FFE7A4E1279836
:105B60002A9A45F60A61C0F60201FAF7BBFB002843
:105B700057D1FFE700F088FD0C9040F22060C2F2A0
:105B8000000000780146059120B1FFE70598012843
:105B900010D045E02E982D9945F67F52C0F60202AE
:105BA0001CF02AFB40F22061C2F2000101200870C3
:105BB0002F9089E10C9840F22161C2F2000109782E
:105BC00050F83100E0B1FFE72E982D990C9A40F281
:105BD0002163C2F2000304931B7852F8333045F678
:105BE000DD52C0F602021CF007FB04990878013070
:105BF000087040F22061C2F20001012008700CE040
:105C000040F22161C2F200010020087040F22061E0
:105C1000C2F2000102200870FFE701202F9053E13B
:105C200063E027982A9A45F60461C0F60201FAF764
:105C300059FB002857D1FFE700F02CFD0B9040F2F4
:105C40002060C2F2000000780146039120B1FFE716
:105C50000398012810D045E02E982D9945F69652CC
:105C6000C0F602021CF0C8FA40F22061C2F2000144
:105C7000012008702F9027E10B9840F22161C2F2B9
:105C80000001097850F83100E0B1FFE72E982D9916
:105C90000B9A40F22163C2F2000302931B7852F880
:105CA000333045F6DD52C0F602021CF0A5FA029927
:105CB00008780130087040F22061C2F20001012032
:105CC00008700CE040F22161C2F20001002008706F
:105CD00040F22061C2F2000102200870FFE70120BB
:105CE0002F90F1E000E0DFE0FFE7C2E028982B9A78
:105CF00045F6EA51C0F60201FAF7F4FA002840F03E
:105D0000B780FFE7279818B1FFE7269808B9FFE7A3
:105D1000CAE027982A9A45F60461C0F60201FAF70C
:105D2000E1FA00283ED1FFE740F22060C2F2000015
:105D30000078B0BBFFE70DA800F02AFC269800F021
:105D4000AFFC88B9FFE72E982D9945F6D842C0F6EA
:105D500002021CF051FA40F22061C2F2000102205E
:105D6000087001202F90AFE02E982D9945F69842AB
:105D7000C0F602021CF040FA269B45F6E152C0F63E
:105D800002020DA8019014211CF036FA019800F0CF
:105D9000BDFC40F22061C2F20001012008702F908A
:105DA00092E04BE027982A9A45F60A61C0F6020174
:105DB000FAF798FA00283FD1FFE740F22060C2F2DC
:105DC00000000078B8BBFFE70DA800F0E1FB2698C3
:105DD00000F024FC88B9FFE72E982D9945F667520C
:105DE000C0F602021CF008FA40F22061C2F2000183
:105DF0000220087001202F9066E02E982D9945F61C
:105E00009842C0F602021CF0F7F90DA80090143079
:105E1000269B45F6E152C0F6020214211CF0ECF973
:105E2000009800F073FC40F22061C2F200010120F2
:105E300008702F9048E000E036E0FFE740F2206075
:105E4000C2F200000078012811D1FFE72E982D99A9
:105E500045F63A52C0F602021CF0CEF940F220613B
:105E6000C2F200010220087001202F902CE0FFE711
:105E7000FFE7FFE7FFE740F22060C2F20000007892
:105E8000022810D1FFE72E982D9945F29632C0F6E0
:105E900002021CF0B1F940F22061C2F200010020C0
:105EA00008702F9010E0FFE72E982D9945F60222FA
:105EB000C0F602021CF0A0F940F22061C2F200011B
:105EC000002008702F90FFE72F9830B080BD0000B1
:105ED00080B588B0069005910492069818B9FFE73E
:105EE000002007908DE005980138059042F21120BE
:105EF000ADF80E00BDF80E00ADF80C009DF80E00D8
:105F00009DF80F1040EA0120ADF80A0040F222602F
:105F1000C2F20000007801460191032861D801997E
:105F2000DFE801F00214283C0698059945F6824204
:105F3000C0F602021CF060F940F22261C2F20001D8
:105F4000087801300870012007905AE006980599FA
:105F5000BDF80C3045F65542C0F602021CF04CF973
:105F600040F22261C2F2000108780130087001207D
:105F7000079046E006980599BDF80A3045F6284294
:105F8000C0F602021CF038F940F22261C2F20001B0
:105F90000878013008700120079032E0BDF80C004D
:105FA000BDF80A10884209D1FFE70698059945F621
:105FB0001042C0F602021CF01FF908E0069805998D
:105FC00045F60342C0F602021CF016F9FFE740F264
:105FD0002261C2F2000108780130087001200790A8
:105FE0000FE00698059945F69542C0F602021CF0AE
:105FF00003F940F22261C2F200010020087007900C
:10600000FFE7079808B080BD80B5DEB05C905B917B
:106010005A925C9818B9FFE700205D90C9E05B9840
:1060200001385B9040F22360C2F200000078014624
:106030000991042800F2AD800999DFE801F00324FA
:10604000778899000AA800F0A3FA5C9807905B98FB
:1060500008902298FAF79EFA024607980B4608998C
:1060600043EC102B6A4682ED000B45F6F332C0F686
:1060700002021CF0C1F840F22361C2F200010120CB
:1060800008705D9095E043F27410C2F20000069033
:10609000C06818F09FF80698006F23A900220A2311
:1060A00017F006FD80B1FFE743F27410C2F2000062
:1060B000C06818F06FF840F22361C2F200010320BB
:1060C000087001205D9074E00AA8039000F060FA67
:1060D00043F27410C2F20000C06818F05BF8039835
:1060E0003899229100F012FB039800F051FA5C9865
:1060F00004905B9805902298FAF74CFA02460498AF
:106100000B46059943EC102B6A4682ED000B45F6D1
:10611000C342C0F602021CF06FF840F22361C2F2E3
:1061200000010220087001205D9042E05C985B99BC
:1061300045F63A52C0F602021CF05EF840F22361C6
:10614000C2F200010520087001205D9031E05C98EA
:106150005B9945F63222C0F602021CF04DF840F27F
:106160002361C2F200010520087001205D9020E04B
:106170005C985B9945F6F042C0F602021CF03CF8D0
:1061800040F22361C2F200010520087001205D90F9
:106190000FE05C985B9945F69542C0F602021CF050
:1061A0002BF840F22361C2F20001002008705D90DC
:1061B000FFE75D985EB080BD80B5E6B06490639106
:1061C0006292649818B9FFE700206590C2E0639876
:1061D0000138639040F22460C2F20000007801466A
:1061E000119148B1FFE71198012817D0FFE71198E6
:1061F000022800F08E809DE06498639945F69C32F9
:10620000C0F602021BF0F8FF40F22461C2F2000166
:10621000087801300870012065909BE012A800F01A
:10622000B7F943F27410C2F200001090C06817F082
:10623000D1FF1098006F2BA90022052317F038FC1E
:10624000C0B1FFE76498639945F64622C0F60202A2
:106250001BF0D2FF40F22461C2F20001022008705C
:1062600043F27410C2F20000C06817F093FF0120DF
:1062700065906FE043F27410C2F20000C06817F03E
:1062800089FF3C9827904098289012A800F03EFA89
:1062900064980E9063980F902798289906912999F1
:1062A0000891FAF777F90246069807920A46079985
:1062B00042EC101B8DED0C0BFAF76CF902460898B6
:1062C00009920A46099942EC101B8DED0A0BFAF768
:1062D00061F99DED0A1B9DED0C0B02460E980B46D5
:1062E0000F9943EC122B6A4682ED042B82ED021BC0
:1062F00082ED000B45F6A342C0F602021BF07CFFC4
:1063000040F22461C2F20001032008700120659070
:1063100020E06498639945F67A22C0F602021BF0E9
:106320006BFF40F22461C2F20001032008700120DB
:1063300065900FE06498639945F69542C0F60202B5
:106340001BF05AFF40F22461C2F2000100200870E5
:106350006590FFE7659866B080BD000080B596B097
:10636000149013911292149818B9FFE70020159019
:106370000AE113980138139040F22560C2F2000040
:10638000007801460A91092800F2EE800A99DFE8B8
:1063900001F00517243643557385BCCE1498139A23
:1063A00045F26571C0F60201F9F772FF40F225610E
:1063B000C2F2000108780130087001201590E3E076
:1063C000149819F0DBFF40F22561C2F20001087851
:1063D0000130087001201590D6E01498139A45F604
:1063E000F401C0F60201F9F753FF40F22561C2F251
:1063F000000108780130087001201590C4E014985D
:1064000019F02AFF40F22561C2F20001087801303C
:10641000087001201590B7E01498139A45F2F471B2
:10642000C0F60201F9F734FF40F22561C2F2000123
:1064300008780130087001201590A5E00BA819F02C
:1064400027FC149813990B9AC2F5C04C6B46C3F8FD
:1064500004C01A6045F6DF32C0F602024FF4C043B2
:106460001BF0CAFE40F22561C2F20001087801303B
:1064700008700120159087E01498139A45F675016D
:10648000C0F60201F9F704FF40F22561C2F20001F3
:106490000878013008700120159075E01498089074
:1064A0001398099043F27410C2F20000D0F8AC10B7
:1064B0000491D0F8B400FAF76DF8024604980592FA
:1064C0000A46059942EC101B8DED060BFAF762F8AF
:1064D0009DED060B024608980B46099943EC112BDB
:1064E0006A4682ED021B82ED000B45F6EB32C0F6E8
:1064F00002021BF081FE40F22561C2F20001087821
:1065000001300870012015903EE01498139A45F66A
:106510008111C0F60201F9F7BBFE40F22561C2F21B
:106520000001087801300870012015902CE01498C3
:10653000139943F27412C2F2000202F1CC03EC464A
:10654000CCF8003002F1B80345F61F42C0F6020253
:106550001BF052FE40F22561C2F2000108780130C2
:106560000870012015900FE01498139945F6954294
:10657000C0F602021BF040FE40F22561C2F20001AB
:10658000002008701590FFE7159816B080BD000038
:1065900080B582B0019001990020C0F60E006422FF
:1065A000FCF7BEFB0198143000F038F80199C8627E
:1065B000019800F075F8019988620198806A38B9ED
:1065C000FFE7019940F28810C2F200008862FFE7FD
:1065D0000198C06A38B9FFE7019944F61810C0F66F
:1065E0000200C862FFE70198806A013038B9FFE70E
:1065F000019940F28810C2F200008862FFE701981A
:10660000C06A013038B9FFE7019944F61810C0F6A6
:106610000200C862FFE702B080BD000080B584B010
:106620000290029818B9FFE70020039029E00020AB
:106630000190FFE7019944F67C60C0F6020050F833
:106640003100D8B1FFE7019944F67C60C0F6020042
:1066500050F831000299F9F72EFE50B9FFE7019981
:1066600044F67C60C0F6020000EBC1004068039075
:1066700007E0FFE7019801300190DBE7002003907D
:10668000FFE7039804B080BD44F67C60C0F60200CA
:106690007047000044F69460C0F6020070470000A6
:1066A00080B584B00290029818B9FFE700200390EB
:1066B00029E000200190FFE7019944F69460C0F6BC
:1066C000020050F83100D8B1FFE7019944F6946018
:1066D000C0F6020050F831000299F9F7ECFD50B90C
:1066E000FFE7019944F69460C0F6020000EBC10098
:1066F0004068039007E0FFE7019801300190DBE775
:1067000000200390FFE7039804B080BD80B582B0FD
:10671000019017F03FF90B20FCF7DEFA01990020F9
:10672000C0F60E006422FCF707FB17F089F902B0EF
:1067300080BD000080B541F69840C2F2000003F031
:10674000F5FB80BD80B541F6B820C2F2000003F031
:10675000EDFB80BD80B541F65820C2F2000003F089
:10676000E5FB80BD80B541F6F840C2F2000003F0C1
:10677000DDFB80BD80B541F61830C2F2000003F0A9
:10678000D5FB80BD80B541F67830C2F2000003F041
:10679000CDFB80BD80B541F6D830C2F2000003F0D9
:1067A000C5FB80BD80B541F65850C2F2000003F031
:1067B000BDFB80BD80B541F63840C2F2000003F059
:1067C000B5FB80BD82B001900198007810384AF680
:1067D000AB21CAF6AA21A0FB011000090090009984
:1067E00044F21870C0F60200405C0199C865009838
:1067F000042807D3FFE701990868042262F309001F
:10680000886506E00199086840F2FF329043886588
:10681000FFE70198806D02B07047000086B00590D8
:1068200000208DF813000598806A03900598806910
:1068300010BBFFE70398029003281BD80299DFE8FA
:1068400001F0020D0218059890F82F00C00720B142
:10685000FFE701208DF81300FFE70CE00598C06A00
:10686000B0F1C07F04D1FFE701208DF81300FFE7EE
:1068700001E000E0FFE745E005988069B0F5005FC2
:1068800025D1FFE70398019003281ED80199DFE87E
:1068900001F00206021101208DF8130016E00598A0
:1068A00090F82F00C00720B1FFE701208DF81300FA
:1068B000FFE70BE00598C06AB0F1C07F04D1FFE7A5
:1068C00001208DF81300FFE700E0FFE719E00398CF
:1068D0000090032804D3FFE70098032804D00EE0BB
:1068E00001208DF813000BE0059890F82F00C007E9
:1068F00020B1FFE701208DF81300FFE700E0FFE77C
:10690000FFE7FFE79DF8130006B0704784B00390DF
:1069100002910192009303980168086820F4802096
:1069200008600098039909684860039880684028C7
:1069300009D1FFE7019803990968886002980399D3
:106940000968C86008E0029803990968886001989E
:1069500003990968C860FFE704B0704782B00090EF
:10696000009820B9FFE701208DF8070074E0009837
:1069700000886FF3DF20B0F5B67F09D3FFE70098FA
:1069800000886FF3DF2040F29561884204D3FFE76F
:1069900001208DF807005FE000980068C0F3CA206E
:1069A000B0F5B67F09D3FFE700980068C0F3CA20AE
:1069B00040F29561884204D3FFE701208DF807007B
:1069C0004AE0009881880068800D40EA81206FF3DA
:1069D000DF20B0F5B67F0DD3FFE70098818800680F
:1069E000800D40EA81206FF3DF2040F295618842FC
:1069F00004D3FFE701208DF807002DE00098808880
:106A0000C0F34A00B0F5B67F09D3FFE7009880884D
:106A1000C0F34A0040F29561884204D3FFE70120A9
:106A20008DF8070018E0009881880020B0EB913FB6
:106A300004D1FFE701208DF807000DE00098808861
:106A4000000B800720B9FFE701208DF8070003E065
:106A500000208DF80700FFE79DF8070002B070479F
:106A600080B584B002900191029820B9FFE7FE2022
:106A70008DF80F000EE0019820B9FFE7FE208DF899
:106A80000F0007E001982421F9F7F7FB00208DF8AB
:106A90000F00FFE79DF90F0004B080BD80B584B002
:106AA0000290029820B9FFE7FE208DF80F002BE03E
:106AB00042F29E60C2F200000078C00720B1FFE7FA
:106AC000FD208DF80F001FE017F094FA43F23431E7
:106AD000C2F20001086020B9FFE7FE208DF80F0028
:106AE00012E046F67542C0F6000200200190032134
:106AF000FCF7B4FC019842F29E62C2F2000201214E
:106B000011708DF80F00FFE79DF90F0004B080BDF4
:106B100080B584B002900191029820B9FFE7FE2071
:106B20008DF80F009FE00298FFF718FF20B1FFE7F4
:106B3000FF208DF80F0096E001982421F9F79DFBC6
:106B4000FFE70020C4F2A5400090029800886FF390
:106B5000DF2000EE100AB8EE400A9FED451A30EE35
:106B6000410A30EE000A9DED002A80EE020A0198EB
:106B700080ED020A02980068C0F3CA2000EE100AF5
:106B8000B8EE400A30EE410A30EE000A9DED002AD0
:106B900080EE020A019880ED030A0298818800685D
:106BA000800D40EA81206FF3DF2000EE100AB8EE7E
:106BB000400A30EE410A30EE000A9DED002A80EED8
:106BC000020A019880ED000A02988088C0F34A000A
:106BD00000EE100AB8EE400A30EE410A30EE000A2C
:106BE0009DED002A80EE020A019880ED010A0298CC
:106BF0008088800B0199487502988088C0F3013025
:106C0000019908750298C0880199C8820298008984
:106C10000199088302984089019948830298007B72
:106C2000002818BF0120019908770298407B0028AE
:106C300018BF0120019948770298C0890199C8833B
:106C40000298008A00EE100AB8EE400A30EE410ABF
:106C50009DED001A80EE010A019880ED040A0020E3
:106C60008DF80F00FFE79DF90F0004B080BD00BF55
:106C70000000804480B543F23430C2F20000006866
:106C8000802117F0D7F880BD80B582B00090002039
:106C9000FCF784FB009912220BF0A6FA20B9FFE75B
:106CA00000208DF8070003E0FF208DF80700FFE7C4
:106CB0009DF9070002B080BD80B582B00190019AB5
:106CC0008020012117F008F98038B0FA80F04009DF
:106CD00002B080BD7047000080B5012003F084FF42
:106CE00080BD000080B5082003F07EFF80BD00005D
:106CF00080B5102003F078FF80BD000080B5202013
:106D000003F072FF80BD0000FFE700BFFDE7000059
:106D100080B584B003908DF80B100020019003988B
:106D200060B3FFE70398012828D0FFE70398022803
:106D300024D0FFE70398032820D0FFE70398042816
:106D40001CD0FFE70398052818D0FFE70398062812
:106D500014D0FFE70398072810D0FFE7039808280E
:106D60000CD0FFE70398092808D0FFE703980A280A
:106D700004D0FFE703980B2801D1FFE708E044F6B1
:106D8000A570C0F6020040F2DB3116F073FCFFE79D
:106D90009DF80B0078B1FFE79DF80B0001280AD0A1
:106DA000FFE79DF80B00022805D0FFE79DF80B00D8
:106DB000032801D1FFE708E044F6A570C0F6020001
:106DC0004FF4777116F056FCFFE79DF80B0018B9E9
:106DD000FFE70020019017E09DF80B00012804D187
:106DE000FFE74FF4807001900DE09DF80B00022842
:106DF00004D1FFE74FF40070019003E04FF44070BE
:106E00000190FFE7FFE7FFE743F61041C4F20201FC
:106E1000086820F440700860019A08681043086010
:106E2000086820F0F8000860039A086840EAC20089
:106E300040F002000860086840F48030086004B048
:106E400080BD000043F60040C4F2020000688005E7
:106E500000281FD5FFE743F60041C4F2020108688D
:106E600020F400700860FFE743F60041C4F202011D
:106E7000086840F400600860086820F4006008605A
:106E8000FFE743F60041C4F20201086840F40070D5
:106E90000860FFE743F60040C4F2020000684005C6
:106EA00000281FD5FFE743F60041C4F2020108683D
:106EB00020F480600860FFE743F60041C4F202015D
:106EC000086840F480500860086820F4805008602A
:106ED000FFE743F60041C4F20201086840F4806015
:106EE0000860FFE77047000080B582B08DF80700AA
:106EF00000919DF8070078B1FFE79DF80700012891
:106F00000AD0FFE79DF80700022805D0FFE79DF8AB
:106F10000700032801D1FFE708E044F6A570C0F69A
:106F200002004FF46F7116F0A5FBFFE700980128EF
:106F300001D1FFE708E044F6A570C0F6020040F278
:106F4000BD3116F097FBFFE743F61041C4F2020192
:106F5000086820F440700860086840F00400086089
:106F60009DF80720086840EA022040F4803008605D
:106F700002B080BD80B582B001908DF803100198F9
:106F8000B0F1006F05D3FFE70198B0F1016F10D3A6
:106F9000FFE7019847F60001C1F6FF71884209D367
:106FA000FFE7019847F60F21C1F6FF71884201D82B
:106FB000FFE708E044F66B70C0F6020040F2BB2128
:106FC00016F058FBFFE743F61041C4F202010868CF
:106FD00020F44070086008680860086840F001000C
:106FE00008609DF803000199087002B080BD0000A0
:106FF00080B584B00390019300920398B0F1006FC4
:1070000005D3FFE70398B0F1016F10D3FFE70398B2
:1070100047F60001C1F6FF71884209D3FFE70398E4
:1070200047F60F21C1F6FF71884201D8FFE708E05B
:1070300044F66B70C0F6020040F2672116F01AFBAE
:10704000FFE743F61041C4F20201086820F44070E3
:107050000860086840F440700860086840F001006B
:107060000860009803990860BFF36F8F0198039937
:10707000486004B080BD000080B582B00190ADF8DA
:1070800002100198B0F1006F05D3FFE70198B0F14D
:10709000016F10D3FFE7019847F60001C1F6FF71B9
:1070A000884209D3FFE7019847F60F21C1F6FF7127
:1070B000884201D8FFE708E044F66B70C0F6020092
:1070C00040F2A22116F0D6FAFFE743F61041C4F2CF
:1070D0000201086820F440700860086840F480707D
:1070E0000860086840F001000860BDF802000199DE
:1070F000088002B080BD000080B582B00190009190
:107100000198B0F1006F05D3FFE70198B0F1016F6E
:1071100010D3FFE7019847F60001C1F6FF718842DE
:1071200009D3FFE7019847F60F21C1F6FF718842A6
:1071300001D8FFE708E044F66B70C0F6020040F2A9
:10714000892116F097FAFFE743F61041C4F20201D5
:10715000086820F440700860086840F40070086017
:10716000086840F00100086000980199086002B0CA
:1071700080BD000043F60C40C4F202000068C00667
:1071800000280FD5FFE742F2B861C2F20001C869DA
:1071900040F01000C86143F60C41C4F20201102017
:1071A0000860FFE743F60C40C4F202000068800666
:1071B00000280FD5FFE742F2B861C2F20001C869AA
:1071C00040F00800C86143F60C41C4F202012020DF
:1071D0000860FFE743F60C40C4F202000068400676
:1071E00000280FD5FFE742F2B861C2F20001C8697A
:1071F00040F00400C86143F60C41C4F20201402093
:107200000860FFE743F60C40C4F202000068000685
:1072100000280FD5FFE742F2B861C2F20001C86949
:1072200040F00200C86143F60C41C4F20201802024
:107230000860FFE743F60C40C4F2020000688007D4
:1072400000280FD5FFE742F2B861C2F20001C86919
:1072500040F02000C86143F60C41C4F20201022054
:107260000860FFE77047000080B584B002900020FE
:10727000019042F2B861C2F20001C86104F0C6F8A0
:107280000190FFE743F60C40C4F202000068C0031F
:10729000002815D5FFE70298013080B1FFE702987A
:1072A00040B1FFE704F0B2F80199401A0299884210
:1072B00004D9FFE703208DF80F0023E0FFE7E1E7A3
:1072C00043F60C40C4F202000068C00738B1FFE783
:1072D00043F60C41C4F2020101200860FFE743F6C7
:1072E0000C40C4F20200006810F0F20F06D0FFE775
:1072F000FFF740FF01208DF80F0003E000208DF81C
:107300000F00FFE79DF80F0004B080BD40F68140FC
:10731000C2F200007047000088B007900691059205
:1073200000200490039005990860FFE704980699EF
:10733000884260D2FFE7FFE70798017800200290BB
:1073400039B1FFE707980078203818BF0120029074
:10735000FFE70298C00720B1FFE7079801300790C8
:10736000EAE7FFE7079801780020019041B1FFE7C5
:10737000079800782038B0FA80F040090190FFE7C4
:107380000198C00720B1FFE7079801300790E9E7AF
:107390000798007868B3FFE70498013004900498D8
:1073A0000699884224D1FFE707980390FFE70798E2
:1073B00001780020009039B1FFE707980078203865
:1073C00018BF01200090FFE70098C00740B1FFE719
:1073D0000599086801300860079801300790E6E7D2
:1073E0000598006818B9FFE700200390FFE702E066
:1073F00000E000E09AE7039808B0704780B586B0D7
:107400000590049103920120029040F22860C2F29C
:1074100000000068002859D1FFE740F22861C2F25D
:10742000000140F2A050C2F200000860FFE740F205
:107430002860C2F200000068002846D0FFE740F252
:107440002860C2F20000006800680068019001989E
:10745000F8F72AFF009005980099405C202805D095
:10746000FFE705980099405C30BBFFE7059801995C
:10747000009AF8F737FFF0B9FFE740F22860C2F250
:1074800000000068006890F90C00002812D4FFE7A3
:10749000059817F007FA40F22861C2F20001096866
:1074A000096891F90C10884203D0FFE70020029090
:1074B000FFE7FFE709E0FFE7FFE740F22861C2F2DC
:1074C0000001086840680860B1E7FFE740F2286003
:1074D000C2F20000006890B1FFE7029878B9FFE7B8
:1074E0000498039A45F2C321C0F60201F8F7D0FED2
:1074F00040F22861C2F200010020086029E040F259
:107500002860C2F200000068B8B1FFE740F22860CE
:10751000C2F2000000680068836804980399059A25
:1075200098470290029838B9FFE740F22861C2F20A
:10753000000100200860FFE70AE00498039A45F282
:107540001B31C0F60201F8F7A3FE00200290FFE70E
:10755000FFE7029806B080BD80B586B0039000209A
:107560000190039858B9FFE74FF0500080F311885D
:10757000BFF36F8FBFF34F8F0490FFE7FEE7082044
:1075800017F0FAFF0290029858B9FFE74FF0500049
:1075900080F31188BFF36F8FBFF34F8F0590FFE724
:1075A000FEE70298B0B1FFE718F0B8FA0398029925
:1075B0000860029900204860029840F22401C2F25B
:1075C00000010A6850600298086018F0D3FA0120A0
:1075D0000190FFE7019806B080BD000080B584B03F
:1075E00047F61020C1F6FF700068039047F614209C
:1075F000C1F6FF700068029047F61820C1F6FF70D0
:10760000006801900199039808440390039888B199
:10761000FFE7039840F26811C2F2000100910231C5
:1076200008220AF089FF00990298123104220AF018
:1076300083FFFFE704B080BD80B58EB006AB049336
:107640000C900B910A920C9820B9FFE7FF208DF85F
:10765000370052E10B9820B9FFE7FF208DF8370083
:107660004BE10A990C980268891A00EE101AB8EEDC
:10767000400A9FEDA41A80EE010A80ED010A0A98E3
:107680000C9908600C980B99097800F0EBF90C98AC
:10769000806890F88E00C00740B1FFE70B9890ED2E
:1076A000010AB1EE400A80ED010A00E0FFE70C9804
:1076B00010300B9991ED010ADFED930ACDED020A2E
:1076C000FDF7C4FE9DED021A0C9890ED052A90ED91
:1076D000430A90ED5E3A33EE022A72EE430AFDF75A
:1076E000F7FE9DED021A049880ED030A0C9890EDC8
:1076F000052A90ED440A90ED5E3A33EE022A72EECE
:10770000430AFDF7E5FE049981ED020A0B98083063
:1077100091ED020AD1ED030AFDF738FF0B9890EDC9
:10772000021A0C9890ED050A30EE010A80ED050A68
:107730000B980430F9F708FC0C98007B0146039184
:1077400040B1FFE7039801281DD0FFE70398022806
:107750005CD074E000208DF81700FFE79DF817005B
:1077600001280FDCFFE70C989DF8171000EB810152
:107770000020C1F85401FFE79DF8170001308DF893
:107780001700EBE75BE00C9901F15800D1ED011A0D
:1077900091ED040AD1ED5A0A9FED5C1A8DED011AA4
:1077A0000CF052FB049A9DED011A82ED010A0C992E
:1077B00001F11C0092ED010AD1ED011AD1ED590A37
:1077C0000CF042FB9DED011A0C9880ED550A0C99C6
:1077D00001F1D000D1ED011A91ED050AD1ED5E0A5B
:1077E0000CF032FB049A9DED011A82ED000A0C990F
:1077F00001F1940092ED000AD1ED011AF0EE410A78
:107800000CF022FB0C9880ED560A18E000208DF851
:107810001600FFE79DF8160001280FDCFFE70C9823
:107820009DF8161000EB81010020C1F85401FFE71C
:107830009DF8160001308DF81600EBE7FFE70020F9
:107840008DF81500FFE79DF8150001281BDCFFE708
:107850000C999DF8152001EB421000F58A7001EBA0
:10786000820191ED550A0AF0DFFE0C989DF8151083
:1078700000EB810080ED550AFFE79DF8150001300F
:107880008DF81500DFE70C98806890F88C00C00731
:1078900040B1FFE70C9890ED550AB1EE400A80ED3B
:1078A000550AFFE70C98806890F88D00C00740B13A
:1078B000FFE70C9890ED560AB1EE400A80ED560AAB
:1078C000FFE70C9890ED550AB5EE400AF1EE10FA7C
:1078D00002DAFFE700BFFFE70C9890ED560AB6EE1C
:1078E000001AB4EE410AF1EE10FA02DDFFE700BF24
:1078F000FFE700208DF83700FFE79DF937000EB055
:1079000080BD00BF00007A44DB0FC94000000000CA
:1079100082B0019000910198D0F85401009908605C
:107920000198D0F858010099486002B070470000F3
:1079300082B0019000910198007B0099087002B01C
:107940007047000080B58AB005AA039202460398EA
:107950000892079180ED010AC0ED000A089820B94D
:10796000FFE7FF208DF8270076E0079808998860E8
:107970000899002008730898806890F88D00C00767
:1079800020B1FFE706A8FDF7F1FDFFE7039890EDB2
:10799000010A089880ED430A089880ED440A089986
:1079A00001F58870896891ED220AB1EE400ADFED99
:1079B0002C0AFDF74BFD039A089901F1580092ED4E
:1079C000000A896801F12002002102910CF0B4FB49
:1079D000039A089901F11C0092ED000A8A680121BE
:1079E00001910CF0A9FB039B0299089A02F1D000C7
:1079F00093ED000A926860320CF09EFB039B0199A4
:107A0000089A02F1940093ED000A926840320CF05B
:107A100093FB02988DF81300FFE79DF813000128EF
:107A200016DCFFE7039A08999DF8130001EB40105C
:107A300000F58A7092ED000A8968D1ED200A0AF0FB
:107A40004FFEFFE79DF8130001308DF81300E4E7C7
:107A500000208DF82700FFE79DF927000AB080BDC0
:107A6000DB0FC94080B584B002908DF807100298F2
:107A700020B9FFE7FF208DF80F0065E09DF80700B3
:107A80000299097B884204D1FFE700208DF80F009E
:107A90005AE000208DF80600FFE79DF80600032855
:107AA00011DCFFE702989DF80610C1EB011100EB15
:107AB00081001C300CF00CFCFFE79DF80600013043
:107AC0008DF80600E9E700208DF80500FFE79DF836
:107AD0000500012812DCFFE702989DF8051000EB75
:107AE000411000F58A709FED1A0A0AF097FEFFE731
:107AF0009DF8050001308DF80500E8E70298103088
:107B0000F9F722FA0298007BB0B9FFE79DF8070069
:107B1000012805D1FFE70299D1F8680108610AE060
:107B20009DF80700022805D1FFE70299D1F87401FA
:107B30000861FFE7FFE7FFE79DF807000299087378
:107B400000208DF80F00FFE79DF90F0004B080BD05
:107B50000000000080B584B002900191029820B925
:107B6000FFE7FF208DF80F002EE0019820B9FFE716
:107B7000FF208DF80F0027E00198406C0299C1F8B2
:107B800074010198406D0299C1F8780102988068EB
:107B900090F88C00C00730B1FFE7029800F5BA708A
:107BA000FDF7E4FCFFE70298806890F88D00C007BD
:107BB00030B1FFE7029800F5BC70FDF7D7FCFFE796
:107BC00000208DF80F00FFE79DF90F0004B080BD85
:107BD00080B586B00490039100200290039800685D
:107BE000122801D8FFE708E045F28E00C0F6020037
:107BF00040F2896115F03EFDFFE70398406830B11F
:107C0000FFE703984068102801D8FFE708E045F235
:107C10008E00C0F6020040F28A6115F02BFDFFE7EE
:107C20000398806818B3FFE70398806801281ED086
:107C3000FFE703988068022819D0FFE7039880685F
:107C4000032814D0FFE70398806804280FD0FFE7CB
:107C50000398806805280AD0FFE703988068062803
:107C600005D0FFE703988068072801D1FFE708E007
:107C700045F28E00C0F6020040F28B6115F0FAFC6E
:107C8000FFE7FFE7049890F83C00012804D1FFE7E4
:107C900002208DF81700F7E00499012081F83C00DC
:107CA000FFE7FFE7039800680A281CD3FFE7039863
:107CB000008800EB4000A0F11E01072000FA01F24D
:107CC00004980168C8689043C86003998868098867
:107CD00001EB41011E3900FA01F204980168C868FD
:107CE0001043C86018E00398008800EB40010720AB
:107CF00000FA01F204980168086990430861039949
:107D00008868098801EB410100FA01F204980168D2
:107D1000086910430861FFE70398406806281BD8EC
:107D2000FFE70398406800EB8000411F1F2000FA26
:107D300001F204980168486B9043486303990888EE
:107D4000496801EB8101053900FA01F204980168E4
:107D5000486B104348633DE0039840680C281CD8EA
:107D6000FFE70398406800EB8000A0F123011F208B
:107D700000FA01F204980168086B904308630399C4
:107D80000888496801EB8101233900FA01F204985F
:107D90000168086B104308631BE00398406800EB20
:107DA0008000A0F141011F2000FA01F2049801684F
:107DB000C86A9043C86203990888496801EB810149
:107DC000413900FA01F204980168C86A1043C86298
:107DD000FFE7FFE742F20030C4F20100019004988F
:107DE000006842F20001C4F2010188420BD1FFE7B2
:107DF00003980068122806D1FFE70199486840F40B
:107E000080004860FFE70498006842F20001C4F275
:107E1000010188422ED1FFE703980068102805D0A1
:107E2000FFE703980068112824D1FFE7019948680B
:107E300040F40000486003980068102819D1FFE75B
:107E400040F22800C2F2000000684DF68361C4F2DF
:107E50001B31A0FB0110800C00EB80004000029061
:107E6000FFE7029820B1FFE7029801380290F8E797
:107E7000FFE7FFE7FFE70499002081F83C00FFE7F8
:107E800000208DF81700FFE79DF8170006B080BDB1
:107E900081B0009000980068C06C01B0704700008D
:107EA00080B584B0029000208DF80700029820B9B8
:107EB000FFE701208DF80F00C7E10298006842F249
:107EC0000001C4F20101884212D0FFE70298006865
:107ED00042F20011C4F20101884209D0FFE7029882
:107EE000006842F20021C4F20101884201D1FFE79B
:107EF00008E045F28E00C0F6020040F2431115F092
:107F0000B9FBFFE70298406890B1FFE7029840682C
:107F1000B0F5803F0CD0FFE702984068B0F5003F15
:107F200006D0FFE702984068B0F5403F01D1FFE777
:107F300008E045F28E00C0F602004FF4A27115F081
:107F400099FBFFE70298806890B1FFE7029880688C
:107F5000B0F1807F0CD0FFE702988068B0F1007F1D
:107F600006D0FFE702988068B0F1407F01D1FFE7BB
:107F700008E045F28E00C0F6020040F2451115F00F
:107F800079FBFFE70298006928B1FFE702980069D2
:107F9000012801D1FFE708E045F28E00C0F602009B
:107FA0004FF4A37115F066FBFFE70298007E28B13D
:107FB000FFE70298007E012801D1FFE708E045F2C3
:107FC0008E00C0F6020040F2471115F053FBFFE7A8
:107FD0000298806A002862D0FFE70298806AB0F1B8
:107FE000807F5CD0FFE70298806AB0F1007F56D0B6
:107FF000FFE70298806AB0F1407F50D0FFE7029817
:10800000806AB0F1806F4AD0FFE70298806AB0F1D1
:10801000A06F44D0FFE70298806AB0F1C06F3ED0F5
:10802000FFE70298806AB0F1E06F38D0FFE702986E
:10803000806AB0F1006F32D0FFE70298806AB0F139
:10804000106F2CD0FFE70298806AB0F1206F26D025
:10805000FFE70298806AB0F1306F20D0FFE7029806
:10806000806AB0F1406F1AD0FFE70298806AB0F1E1
:10807000506F14D0FFE70298806AB0F1606F0ED0A5
:10808000FFE70298806AB0F1706F08D0FFE70298AE
:10809000806A0121C0F60071884201D1FFE708E043
:1080A00045F28E00C0F602004FF4A47115F0E2FA1A
:1080B000FFE70298C06830B1FFE70298C068B0F5EA
:1080C000006F01D1FFE708E045F28E00C0F6020024
:1080D00040F2491115F0CEFAFFE70298C06930B1BD
:1080E000FFE70298C069102801D8FFE708E045F2D1
:1080F0008E00C0F602004FF4A57115F0BBFAFFE741
:10810000029890F8300030B1FFE7029890F8300004
:10811000012801D1FFE708E045F28E00C0F6020019
:1081200040F24B1115F0A6FAFFE7029840690128CA
:1081300009D0FFE70298406928B1FFE7029840693B
:10814000022801D1FFE708E045F28E00C0F60200E8
:108150004FF4A67115F08EFAFFE7029890F8200010
:1081600030B1FFE7029890F82000012801D1FFE725
:1081700008E045F28E00C0F6020040F24D1115F005
:1081800079FAFFE70298806A0121C0F600718842FF
:1081900021D0FFE70298C06A90B1FFE70298C06A59
:1081A000B0F1805F0CD0FFE70298C06AB0F1005FC9
:1081B00006D0FFE70298C06AB0F1405F01D1FFE747
:1081C00008E045F28E00C0F6020040F2511115F0B1
:1081D00051FAFFE7FFE70298006C50B9FFE70298F9
:1081E00000F038F8029900204864029981F83C00B8
:1081F000FFE70298006CC006002817D4FFE702983A
:10820000006C40F0020020F4885002990864029843
:10821000F8F7D0FB0299002048640298006C40F007
:10822000010020F002000299086403E001208DF8AB
:108230000700FFE7FFE70299002081F83C00FFE715
:108240009DF807008DF80F00FFE79DF80F0004B0C0
:1082500080BD000080B58AB009900020089007908A
:108260000690059004900998006842F20001C4F25B
:108270000101884212D1FFE7FFE70020039043F697
:108280004400C4F20200016841F48071016000689A
:1082900000F4807003900398FFE73AE009980068C3
:1082A00042F20021C4F20101884231D1FFE7FFE729
:1082B0000020029043F64400C4F20200016841F439
:1082C00080610160006800F4806002900298FFE71E
:1082D000FFE70020019043F63000C4F2020001687D
:1082E00041F020010160006800F020000190019839
:1082F000FFE74FF480600490032005900020069073
:1083000041F20040C4F2020004A902F089FCFFE738
:10831000FFE70AB080BD000080B584B002900191F3
:10832000002000900298006880684005002816D55B
:10833000FFE7029800688068C00500280FD5FFE7B6
:108340000299086C40F020000864FFE702990020C1
:1083500081F83C00FFE701208DF80F006DE003F08D
:1083600055F80090FFE702980068006800F00200EE
:10837000022829D0FFE70198013020B3FFE70198D8
:1083800040B1FFE703F042F80099401A0199884292
:1083900018D9FFE702980068006800F00200022880
:1083A0000FD0FFE70299086C40F004000864FFE773
:1083B0000299002081F83C00FFE703208DF80F00B0
:1083C0003BE0FFE7FFE7CEE7029801686FF012009D
:1083D00008600299086C40F4007008640298006814
:1083E000806810F0405F24D1FFE70298007E00BB58
:1083F000FFE702980068C06A10F4700F07D0FFE72B
:108400000298006880684005002812D4FFE70299AE
:10841000086C20F4807008640298006CC004002886
:1084200006D4FFE70299086C40F001000864FFE7FA
:10843000FFE700208DF80F00FFE79DF80F0004B064
:1084400080BD000080B584B00290002001900298A9
:10845000007E28B1FFE70298007E012801D1FFE7E6
:1084600008E045F28E00C0F6020040F2D32115F07C
:1084700001F9FFE70298C06A90B1FFE70298C06A6D
:10848000B0F1805F0CD0FFE70298C06AB0F1005FE6
:1084900006D0FFE70298C06AB0F1405F01D1FFE764
:1084A00008E045F28E00C0F602004FF4357115F079
:1084B000E1F8FFE7FFE7029890F83C00012804D1BB
:1084C000FFE702208DF80F00D4E00299012081F827
:1084D0003C00FFE7FFE7029800688068C007F0B93A
:1084E000FFE702980168886840F00100886040F268
:1084F0002800C2F2000000684DF68361C4F21B310F
:10850000A0FB0110800C00EB40000190FFE70198F8
:1085100020B1FFE7019801380190F8E7FFE70298E2
:1085200000688068C007002800F09580FFE7029887
:10853000006C40F4807040F2016188430299086445
:108540000298006840684005002809D5FFE70298B6
:10855000006C40F4805020F4005002990864FFE75A
:108560000298006CC004002806D5FFE70299486C09
:1085700020F00600486403E0029900204864FFE709
:10858000FFE70299002081F83C00FFE742F200304B
:10859000C4F201000090029801686FF022000860A8
:1085A00000984068C006E8BBFFE70298006842F206
:1085B0000001C4F20101884224D0FFE7029800685C
:1085C00042F20011C4F20101884208D1FFE742F2F1
:1085D0000430C4F201000068C00698B1FFE70298B9
:1085E000006842F20021C4F20101884219D1FFE77C
:1085F00042F20430C4F20100006800F01F000F28AE
:108600000FD8FFE702980068806810F0405F07D13C
:10861000FFE702980168886840F080408860FFE7C3
:10862000FFE717E00298006842F20001C4F201017E
:1086300088420ED1FFE702980068806810F0405F22
:1086400007D1FFE702980168886840F080408860A1
:10865000FFE7FFE70AE00299086C40F010000864A9
:108660000299486C40F001004864FFE700208DF853
:108670000F00FFE79DF80F0004B080BD80B584B007
:1086800002900191029890F820008DF80300019863
:1086900048F67F71C0F20301884201D8FFE708E085
:1086A00045F2C600C0F602004FF4D06114F0E2FFBC
:1086B000FFE79DF80300012805D0FFE79DF80300C0
:1086C00002280AD1FFE7019A02980168486910431D
:1086D000486100208DF80F0008E00299486A40F4D4
:1086E0008020486201208DF80F00FFE79DF80F0001
:1086F00004B080BD80B588B00690059104920393C4
:10870000069890F820008DF80700069800688068A9
:1087100000900598806828B1FFE7059880680428D4
:1087200001D1FFE708E045F2C600C0F6020040F2C2
:10873000E94114F09FFFFFE70598C06828B1FFE703
:108740000598C068022801D1FFE708E045F2C6009D
:10875000C0F6020040F2EA4114F08CFFFFE70598F2
:108760000069082801D8FFE708E045F2C600C0F616
:10877000020040F2EB4114F07DFFFFE705988068AE
:1087800090B9FFE7059801680020B0EBD12F01D127
:10879000FFE708E045F2C600C0F6020040F2EE41F5
:1087A00014F068FFFFE711E0059841680020B0EB86
:1087B000517F01D1FFE708E045F2C600C0F6020094
:1087C00040F2F24114F056FFFFE7FFE70598007D05
:1087D00028B1FFE70598007D012801D1FFE708E0F7
:1087E00045F2C600C0F6020040F2F44114F042FF28
:1087F000FFE79DF80700012806D0FFE79DF8070076
:10880000022840F08D80FFE79DF803004007002814
:108810000CD4FFE79DF803000007002806D4FFE70B
:108820009DF80300C006002871D5FFE70098C0F34B
:10883000016002900298032809D3FFE70699486A6D
:1088400040F40000486201208DF81F0071E0029999
:1088500001208840039908600598806868B9FFE79F
:1088600005980168C06840EA415006990968029A73
:1088700001EB0211C1F880010EE005994A68886891
:10888000C96840EAC200084306990968029A01EBE8
:108890000211C1F88001FFE705980069069909688F
:1088A000029A01EB0211C1F884010598007D0128AC
:1088B0000CD1FFE706980068029900EB0111D1F88E
:1088C000840140F48070C1F88401FFE70498406897
:1088D00006990968029A01EB0211C1F88C0104980B
:1088E000006806990968029A01EB0211C1F8880133
:1088F00006980068029900EB0111D1F8800140F060
:108900000100C1F8800100208DF81F0011E00699D8
:10891000486A40F40010486201208DF81F0008E00A
:108920000699486A40F48020486201208DF81F00B3
:10893000FFE79DF81F0008B080BD000080B586B03D
:1089400004900391049800680190049890F8200026
:108950008DF803009DF80300012806D0FFE79DF87D
:108960000300022840F05281FFE70398408808B9CD
:10897000FFE708E045F2C600C0F602004FF454716C
:1089800014F078FEFFE70398C08808B9FFE708E015
:1089900045F2C600C0F6020040F2513114F06AFE02
:1089A000FFE70398408908B9FFE708E045F2C600F1
:1089B000C0F6020040F2523114F05CFEFFE703986B
:1089C000C08908B9FFE708E045F2C600C0F602001A
:1089D00040F2533114F04EFEFFE70398806928B14E
:1089E000FFE703988069012801D1FFE708E045F21D
:1089F000C600C0F602004FF4557114F03BFEFFE7CD
:108A00000398C06928B1FFE70398C069012801D124
:108A1000FFE708E045F2C600C0F6020040F255311B
:108A200014F028FEFFE70398006928B1FFE70398D8
:108A30000069012801D1FFE708E045F2C600C0F651
:108A4000020040F2563114F015FEFFE70398006A69
:108A500028B1FFE70398006A012801D1FFE708E089
:108A600045F2C600C0F6020040F2573114F002FE93
:108A7000FFE746F20040C4F200000190039840690D
:108A80001B2801D8FFE708E045F2C600C0F6020047
:108A900040F2723114F0EEFDFFE70398406A1B28A4
:108AA00001D8FFE708E045F2C600C0F6020040F238
:108AB000733114F0DFFDFFE70199D1F8000240F0B7
:108AC0000100C1F800020199D1F8000220F47C50A5
:108AD000C1F800020398426A0199D1F8000240EA05
:108AE0000220C1F800020398406900F01F01012034
:108AF00088400290029A0199D1F81C029043C1F873
:108B00001C020398C069F0B9FFE7029A0199D1F8F5
:108B10000C029043C1F80C02039A9088D168526904
:108B200040EA0140019901EBC201C1F84002039AF9
:108B300010889168526940EA0140019901EBC20135
:108B4000C1F84402FFE70398C06901281ED1FFE77E
:108B5000029A0199D1F80C021043C1F80C02039A51
:108B600090881168526940EA0140019901EBC20105
:108B7000C1F84002039A90899168526940EA014025
:108B8000019901EBC201C1F84402FFE70398806933
:108B900040B9FFE7029A0199D1F804029043C1F865
:108BA000040207E0029A0199D1F804021043C1F8C7
:108BB0000402FFE70398006940B9FFE7029A0199B0
:108BC000D1F814029043C1F8140207E0029A019907
:108BD000D1F814021043C1F81402FFE70398006AA9
:108BE000012808D1FFE7029A0199D1F81C0210432D
:108BF000C1F81C02FFE70199D1F8000220F0010042
:108C0000C1F8000200208DF8170008E00499486AB6
:108C100040F48020486201208DF81700FFE79DF89E
:108C2000170006B080BD000080B582B001900198A9
:108C3000FAF7C0FD8DF803009DF80300032819D052
:108C4000FFE79DF8030040F2A852C2F2000234216F
:108C500010FB0120006B60B1FFE79DF8030040F2BC
:108C6000A852C2F20002342110FB0120006B8047A1
:108C7000FFE7FFE702B080BD80B586B004900391A6
:108C800002920193049890F820008DF80300039855
:108C900020B1FFE70398012801D1FFE708E045F282
:108CA000C600C0F602004FF4BE6114F0E3FCFFE71B
:108CB0009DF80300012806D0FFE79DF80300022875
:108CC00040F0D780FFE7039880B9FFE70498006879
:108CD000C068800748B9FFE70499486A40F400106B
:108CE000486201208DF81700CCE00FE0049800687E
:108CF0000069800748B9FFE70499486A40F400100A
:108D0000486201208DF81700BCE0FFE70498006876
:108D1000039900EB0110D0F8B00100F004000299B3
:108D200088600298806858B9FFE704980068039942
:108D300000EB0110D0F8B001400D029908600AE084
:108D400004980068039900EB0110D0F8B001C00846
:108D500002994860FFE704980068039900EB01104E
:108D6000D0F8B00100F002000299C86004980068D1
:108D7000039900EB0110D0F8B40100F00F00029944
:108D8000086104980068039900EB0110D0F8B40161
:108D900080B2000A0299886104980068039900EB88
:108DA0000110D0F8B401000C0299486104980068E1
:108DB000039900EB0110D0F8B801019908700498EC
:108DC0000068039900EB0110D0F8B801000A01997E
:108DD000487004980068039900EB0110D0F8B801BE
:108DE000000C0199887004980068039900EB011049
:108DF000D0F8B801000E0199C87004980068039972
:108E000000EB0110D0F8BC010199087104980068CA
:108E1000039900EB0110D0F8BC01000A01994871D8
:108E200004980068039900EB0110D0F8BC01000C15
:108E30000199887104980068039900EB0110D0F83B
:108E4000BC01000E0199C871039838B9FFE7049876
:108E50000168C86840F02000C86006E00498016816
:108E6000086940F020000861FFE700208DF8170036
:108E700008E00499486A40F48020486201208DF897
:108E80001700FFE79DF8170006B080BD80B58AB0D7
:108E90000990002008900998006840690790099897
:108EA00000684068069009980068806805900998F5
:108EB0000068C068049009980068006903900998E8
:108EC0000068806902909DF81C00C007002800F02F
:108ED0009480FFE79DF81400C00758B3FFE7099896
:108EE0000168012088609DF814008007002804D5DF
:108EF000FFE7099800F042FE1BE09DF814004007D0
:108F0000002805D5FFE7089840F4006008900FE0BE
:108F10009DF814000007002805D5FFE7089840F4E5
:108F20008050089003E0099800F000FEFFE7FFE79B
:108F3000FFE7FFE79DF81500C00760B3FFE709985A
:108F400001684FF4807088609DF815008007002844
:108F500004D5FFE7099800F05FFE1BE09DF81500BF
:108F60004007002805D5FFE7089840F40050089016
:108F70000FE09DF815000007002805D5FFE70898C9
:108F800040F48040089003E0099800F01DFEFFE7E0
:108F9000FFE7FFE7FFE79DF81600C00760B3FFE7B4
:108FA000099801684FF4803088609DF816008007AA
:108FB000002804D5FFE7099800F07EFE1BE09DF82D
:108FC00016004007002805D5FFE7089840F4004048
:108FD00008900FE09DF816000007002805D5FFE770
:108FE000089840F48030089003E0099800F03CFEB7
:108FF000FFE7FFE7FFE7FFE7FFE79DF81C0000073B
:10900000002810D5FFE79DF81000C006002809D5FC
:10901000FFE7089840F40070089009980168102054
:10902000C860FFE7FFE79DF81C00400700280FD548
:10903000FFE79DF810000007002808D5FFE7099812
:1090400001680820C860099800F062FCFFE7FFE7AC
:109050009DF81C00800700280BD5FFE709980068E1
:10906000C068800720B1FFE7099800F079FCFFE7AE
:10907000FFE79DF81C004006002810D5FFE79DF88B
:109080000C00C006002809D5FFE7089840F480606E
:1090900008900998016810200861FFE7FFE79DF834
:1090A0001C00800600280FD5FFE79DF80C00000784
:1090B000002808D5FFE70998016808200861099889
:1090C00000F076FCFFE7FFE79DF81C00C0060028D3
:1090D0000BD5FFE7099800680069800720B1FFE71A
:1090E000099800F08DFCFFE7FFE79DF81E00800760
:1090F00000280FD5FFE79DF81800C006002808D506
:10910000FFE70998016810204860099800F0A0FC6A
:10911000FFE7FFE79DF81E00C00778B1FFE79DF865
:1091200018000007002808D5FFE709980168082003
:109130004860099800F0E8FDFFE7FFE79DF81D0093
:109140000006002840F18D80FFE79DF818004007D9
:10915000002840F18180FFE79DF81D00C00750B155
:10916000FFE79DF80800C00728B1FFE7089840F026
:1091700001000890FFE79DF81D00800700280BD52F
:10918000FFE79DF808008007002805D5FFE708984D
:1091900040F002000890FFE79DF81D0040070028FE
:1091A0000BD5FFE79DF808004007002805D5FFE72D
:1091B000089840F004000890FFE79DF81D000007A4
:1091C000002848D5FFE79DF8080010F0700F42D046
:1091D000FFE7029800F0700001460191102814D0BA
:1091E000FFE70198202815D0FFE70198302816D016
:1091F000FFE70198402817D0FFE70198502818D0C2
:10920000FFE70198602819D01DE0089840F0080099
:10921000089019E0089840F01000089014E00898B1
:1092200040F0200008900FE0089840F040000890BF
:109230000AE0089840F08000089005E0089840F4A3
:109240008070089000E0FFE709980168886920F0C5
:1092500070008861FFE7FFE7099801680420486013
:10926000FFE7089848B1FFE7089A0999486A104350
:1092700048620998FFF7D8FCFFE70AB080BD0000FC
:1092800080B584B00290029820B9FFE701208DF8E4
:109290000F0063E20298006846F20041C4F2000148
:1092A000884209D0FFE70298006846F60001C4F240
:1092B0000001884201D1FFE708E045F2C600C0F690
:1092C000020040F21D1114F0D5F9FFE70298007E6C
:1092D00028B1FFE70298007E012801D1FFE708E0EE
:1092E00045F2C600C0F602004FF48F7114F0C2F9C7
:1092F000FFE70298407E28B1FFE70298407E0128F0
:1093000001D1FFE708E045F2C600C0F6020040F2D6
:109310001F1114F0AFF9FFE70298807E28B1FFE734
:109320000298807E012801D1FFE708E045F2C600DF
:10933000C0F602004FF4907114F09CF9FFE7029818
:10934000C07E28B1FFE70298C07E012801D1FFE767
:1093500008E045F2C600C0F6020040F2211114F008
:1093600089F9FFE70298007F28B1FFE70298007FA4
:10937000012801D1FFE708E045F2C600C0F602006F
:109380004FF4917114F076F9FFE70298407F28B10D
:10939000FFE70298407F012801D1FFE708E045F28E
:1093A000C600C0F6020040F2231114F063F9FFE793
:1093B0000298806890B1FFE702988068B0F1804F12
:1093C0000CD0FFE702988068B0F1004F06D0FFE7AD
:1093D00002988068B0F1404F01D1FFE708E045F204
:1093E000C600C0F602004FF4927114F043F9FFE793
:1093F0000298C06890B1FFE70298C068B0F1807F22
:109400000CD0FFE70298C068B0F1007F06D0FFE7FC
:109410000298C068B0F1407F01D1FFE708E045F253
:10942000C600C0F6020040F2251114F023F9FFE750
:109430000298006900285AD0FFE702980069B0F549
:10944000803F54D0FFE702980069B0F5003F4ED04E
:10945000FFE702980069B0F5403F48D0FFE7029867
:109460000069B0F5802F42D0FFE702980069B0F59F
:10947000A02F3CD0FFE702980069B0F5C02F36D08E
:10948000FFE702980069B0F5E02F30D0FFE70298BF
:109490000069B0F5002F2AD0FFE702980069B0F507
:1094A000102F24D0FFE702980069B0F5202F1ED0BE
:1094B000FFE702980069B0F5302F18D0FFE7029857
:1094C0000069B0F5402F12D0FFE702980069B0F5AF
:1094D000502F0CD0FFE702980069B0F5602F06D03E
:1094E000FFE702980069B0F5702F01D1FFE708E0AF
:1094F00045F2C600C0F602004FF4937114F0BAF8BA
:10950000FFE70298406950B3FFE702984069B0F561
:10951000801F24D0FFE702984069B0F5001F1ED0DD
:10952000FFE702984069B0F5401F18D0FFE70298A6
:109530004069B0F5800F12D0FFE702984069B0F59E
:10954000A00F0CD0FFE702984069B0F5C00F06D01D
:10955000FFE702984069B0F5E00F01D1FFE708E0AE
:1095600045F2C600C0F6020040F2271114F082F85E
:10957000FFE70298406838B1FFE702984068B0F50D
:10958000806F01D8FFE708E045F2C600C0F6020090
:109590004FF4947114F06EF8FFE7029890F82000F1
:1095A00020B9FFE7029800F0DDF8FFE702980168B4
:1095B000086820F00200086001F028FF0190FFE732
:1095C0000298006840688007002815D5FFE701F081
:1095D0001DFF0199401A0B280DD3FFE70299486A35
:1095E00040F4003048620299052081F820000120F3
:1095F0008DF80F00B2E0E3E702980168086840F0D8
:109600000100086001F002FF0190FFE70298006886
:109610004068C007A8B9FFE701F0F8FE0199401AB9
:109620000B280DD3FFE70299486A40F400304862E6
:109630000299052081F8200001208DF80F008DE0AF
:10964000E4E70298007E012807D1FFE7029801684D
:10965000086840F08000086006E002980168086829
:1096600020F080000860FFE70298407E012807D1C3
:10967000FFE702980168086840F04000086006E0D3
:1096800002980168086820F040000860FFE702982F
:10969000807E012807D1FFE702980168086840F042
:1096A0002000086006E002980168086820F02000A9
:1096B0000860FFE70298C07E012807D1FFE7029803
:1096C0000168086820F01000086006E00298016850
:1096D000086840F010000860FFE70298007F01284A
:1096E00007D1FFE702980168086840F008000860A9
:1096F00006E002980168086820F008000860FFE7AB
:109700000298407F012807D1FFE7029801680868A6
:1097100040F00400086006E002980168086820F044
:1097200004000860FFE7029B19685A689868D3F83C
:109730000CC040EA0C00D3F810C040EA0C005B6992
:109740001843013A1043C861029900204862029A06
:10975000012182F820108DF80F00FFE79DF80F001F
:1097600004B080BD80B594B0139000201290119089
:1097700010900F900E901398006846F20041C4F2CA
:109780000001884253D1FFE740F26C60C2F2000052
:109790000168013101600068012812D1FFE7FFE78D
:1097A00000200D9043F64000C4F20200016841F031
:1097B00000710160006800F000700D900D98FFE7E7
:1097C000FFE7FFE700200C9043F63000C4F20200F0
:1097D000016841F008010160006800F008000C9089
:1097E0000C98FFE703200E9002210F9100210791B2
:1097F000109111900920129040F60040C4F202002E
:109800000EA901F00DFA079A142005900521069182
:1098100002F018FA059802F0FDF90699079A15204A
:10982000089002F00FFA089802F0F4F96EE013982D
:10983000006846F60001C4F20001884265D1FFE7E6
:10984000FFE700200B9043F64000C4F202000168DD
:1098500041F080610160006800F080600B900B981F
:10986000FFE740F26C60C2F2000001680131016064
:109870000068012812D1FFE7FFE700200A9043F6B5
:109880004000C4F20200016841F00071016000680C
:1098900000F000700A900A98FFE7FFE7FFE700205A
:1098A000099043F63000C4F20200016841F0020161
:1098B0000160006800F0020009900998FFE760204D
:1098C0000E9002200F900020039010900320119022
:1098D0000920129040F20040C4F202000EA901F0EB
:1098E0009FF9039A402001900521029102F0AAF904
:1098F000019802F08FF90299039A4120049002F036
:10990000A1F9049802F086F9FFE7FFE714B080BDE3
:1099100080B582B001900198F9F74CFF8DF80300F3
:109920009DF80300032819D0FFE79DF8030040F2DB
:10993000A852C2F20002342110FB0120C06960B1BC
:10994000FFE79DF8030040F2A852C2F20002342162
:1099500010FB0120C0698047FFE7FFE702B080BD30
:1099600080B582B001900198F9F724FF8DF80300CB
:109970009DF80300032819D0FFE79DF8030040F28B
:10998000A852C2F20002342110FB0120806960B1AC
:10999000FFE79DF8030040F2A852C2F20002342112
:1099A00010FB012080698047FFE7FFE702B080BD20
:1099B00080B582B001900198F9F7FCFE8DF80300A4
:1099C0009DF80300032819D0FFE79DF8030040F23B
:1099D000A852C2F20002342110FB0120406A60B19B
:1099E000FFE79DF8030040F2A852C2F200023421C2
:1099F00010FB0120406A8047FFE7FFE702B080BD0F
:109A000080B582B001900198F9F7D4FE8DF803007B
:109A10009DF80300032819D0FFE79DF8030040F2EA
:109A2000A852C2F20002342110FB0120006A60B18A
:109A3000FFE79DF8030040F2A852C2F20002342171
:109A400010FB0120006A8047FFE7FFE702B080BDFE
:109A500080B582B001900198F9F7ACFE8DF8030053
:109A60009DF80300032819D0FFE79DF8030040F29A
:109A7000A852C2F20002342110FB0120806A60B1BA
:109A8000FFE79DF8030040F2A852C2F20002342121
:109A900010FB0120806A8047FFE7FFE702B080BD2E
:109AA00080B584B00290029890F8200001282FD150
:109AB000FFE70299022081F82000029801680868F7
:109AC00020F00100086001F0A1FC0190FFE702987E
:109AD00000684068C007A8B1FFE701F097FC019952
:109AE000401A0B280DD3FFE70299486A40F4003072
:109AF00048620299052081F8200001208DF80F00AE
:109B00000FE0E4E70299002048628DF80F0008E0BA
:109B10000299486A40F40020486201208DF80F0045
:109B2000FFE79DF80F0004B080BD000080B582B053
:109B300001900198F9F73EFE8DF803009DF80300AF
:109B4000032819D0FFE79DF8030040F2A852C2F2A3
:109B50000002342110FB0120C06860B1FFE79DF8CE
:109B6000030040F2A852C2F20002342110FB01208F
:109B7000C0688047FFE7FFE702B080BD80B582B0D4
:109B800001900198F9F716FE8DF803009DF8030087
:109B9000032817D0FFE79DF803003421414340F22A
:109BA000A850C2F20000405858B1FFE79DF80300EA
:109BB0003421414340F2A850C2F20000405880478F
:109BC000FFE7FFE702B080BD80B582B00190019849
:109BD000F9F7F0FD8DF803009DF80300032819D074
:109BE000FFE79DF8030040F2A852C2F200023421C0
:109BF00010FB0120006960B1FFE79DF8030040F20F
:109C0000A852C2F20002342110FB012000698047F3
:109C1000FFE7FFE702B080BD80B582B001900198F8
:109C2000F9F7C8FD8DF803009DF80300032819D04B
:109C3000FFE79DF8030040F2A852C2F2000234216F
:109C400010FB0120406860B1FFE79DF8030040F27F
:109C5000A852C2F20002342110FB01204068804764
:109C6000FFE7FFE702B080BD80B582B001900198A8
:109C7000F9F7A0FD8DF803009DF80300032819D023
:109C8000FFE79DF8030040F2A852C2F2000234211F
:109C900010FB0120406960B1FFE79DF8030040F22E
:109CA000A852C2F20002342110FB01204069804713
:109CB000FFE7FFE702B080BD80B582B00190019858
:109CC000F9F778FD8DF803009DF80300032819D0FB
:109CD000FFE79DF8030040F2A852C2F200023421CF
:109CE00010FB0120806860B1FFE79DF8030040F29F
:109CF000A852C2F20002342110FB01208068804784
:109D0000FFE7FFE702B080BD80B582B00190019807
:109D1000F9F750FD8DF803009DF80300032819D0D2
:109D2000FFE79DF8030040F2A852C2F2000234217E
:109D300010FB0120C06A60B1FFE79DF8030040F20C
:109D4000A852C2F20002342110FB0120C06A8047F1
:109D5000FFE7FFE702B080BD80B582B000900098B9
:109D600020B9FFE701208DF8070023E00098006884
:109D700043F20001C4F20201884201D1FFE707E08B
:109D800045F2FE00C0F60200682113F073FCFFE705
:109D90000098407938B9FFE70099002008710098D1
:109DA00000F00CF8FFE700990120487100208DF8C1
:109DB0000700FFE79DF8070002B080BD82B0019068
:109DC0000198006843F20001C4F20201884212D1F6
:109DD000FFE7FFE70020009043F63000C4F20200E6
:109DE000016841F480510160006800F480500090E7
:109DF0000098FFE7FFE702B07047000080B584B02D
:109E000002900298806D019001F000FB0090029892
:109E100090F8350002280DD0FFE7029980204865B0
:109E2000FFE70299002081F83400FFE701208DF858
:109E30000F0054E002980168086820F016000860DE
:109E400002980168486920F0800048610298006C1F
:109E500020B9FFE70298806C38B1FFE702980168EB
:109E6000086820F008000860FFE7029801680868A9
:109E700020F001000860FFE7029800680068C00752
:109E8000C0B1FFE701F0C2FA0099401A062810D3CA
:109E9000FFE7029920204865FFE70299002081F83A
:109EA0003400FFE70299032081F835008DF80F0098
:109EB00015E0E1E70298C16D3F2088400199886074
:109EC000FFE70299002081F83400FFE702990120A2
:109ED00081F83500FFE700208DF80F00FFE79DF8BF
:109EE0000F0004B080BD000082B00090009890F890
:109EF0003500022807D0FFE700998020486501203F
:109F00008DF807000EE00099052081F835000098D3
:109F10000168086820F001000860FFE700208DF864
:109F20000700FFE79DF8070002B0704780B586B0D4
:109F300005900020039040F22800C2F20000006863
:109F400048F2B511C1F64E31A0FB0110800A029013
:109F50000598806D01900198006804900498059917
:109F6000C96DC840000700281AD5FFE705980068AA
:109F700000684007002812D5FFE7059801680868C7
:109F800020F0040008600598C16D08208840019900
:109F900088600599486D40F001004865FFE7FFE7DC
:109FA00004980599C96DC840C007A0B1FFE705989E
:109FB00000684069000600280CD5FFE70598C16DD0
:109FC00001208840019988600599486D40F00200A1
:109FD0004865FFE7FFE704980599C96DC840400749
:109FE000002814D5FFE7059800680068800700285E
:109FF0000CD5FFE70598C16D042088400199886061
:10A000000599486D40F004004865FFE7FFE70498B4
:10A010000599C96DC840C006002847D5FFE70598D7
:10A0200000680068000700283FD5FFE70598C16D6C
:10A0300010208840019988600598006800684003F6
:10A0400000281AD5FFE7059800680068000300287B
:10A0500009D4FFE70598006C20B1FFE70598016C73
:10A060008847FFE708E00598806C20B1FFE7059876
:10A07000816C8847FFE7FFE716E0059800680068F5
:10A08000C005002807D4FFE705980168086820F09C
:10A0900008000860FFE70598006C20B1FFE705980D
:10A0A000016C8847FFE7FFE7FFE7FFE704980599A2
:10A0B000C96DC8408006002840F18D80FFE70598F3
:10A0C00000680068C006002840F18480FFE705981A
:10A0D000C16D2020884001998860059890F835006E
:10A0E000052834D1FFE705980168086820F01600BC
:10A0F000086005980168486920F08000486105986B
:10A10000006C20B9FFE70598806C38B1FFE705982F
:10A110000168086820F008000860FFE70598C16D35
:10A120003F20884001998860FFE70599002081F869
:10A130003400FFE70599012081F835000598006D8E
:10A1400020B1FFE70598016D8847FFE77BE00598A0
:10A1500000680068400300281AD5FFE705980068EA
:10A1600000680003002809D4FFE70598406C20B17F
:10A17000FFE70598416C8847FFE708E00598C06B4A
:10A1800020B1FFE70598C16B8847FFE7FFE720E0B4
:10A19000059800680068C005002811D4FFE70598FD
:10A1A0000168086820F010000860FFE705990020AA
:10A1B00081F83400FFE70599012081F83500FFE7B9
:10A1C0000598C06B20B1FFE70598C16B8847FFE792
:10A1D000FFE7FFE7FFE70598406DA0B3FFE70598AD
:10A1E000406DC00730B3FFE70599052081F83500C1
:10A1F00005980168086820F001000860FFE70398EF
:10A20000013003900299884201D9FFE707E0FFE798
:10A21000059800680068C0070028F0D1FFE7FFE755
:10A220000599002081F83400FFE70599012081F8A5
:10A230003500FFE70598C06C20B1FFE70598C16CB9
:10A240008847FFE7FFE706B080BD000080B586B015
:10A2500004900020039001F0D9F80290049820B9EE
:10A26000FFE701208DF8170087E20498006846F2A6
:10A270001001C4F20201884200F08880FFE70498D0
:10A28000006846F22801C4F2020188427ED0FFE74E
:10A290000498006846F24001C4F20201884275D079
:10A2A000FFE70498006846F25801C4F202018842B0
:10A2B0006CD0FFE70498006846F27001C4F2020116
:10A2C000884263D0FFE70498006846F28801C4F230
:10A2D000020188425AD0FFE70498006846F2A001C4
:10A2E000C4F20201884251D0FFE70498006846F2A8
:10A2F000B801C4F20201884248D0FFE70498006820
:10A3000046F21041C4F2020188423FD0FFE70498B0
:10A31000006846F22841C4F20201884236D0FFE7C5
:10A320000498006846F24041C4F2020188422DD0F0
:10A33000FFE70498006846F25841C4F202018842DF
:10A3400024D0FFE70498006846F27041C4F202018D
:10A3500088421BD0FFE70498006846F28841C4F2A7
:10A360000201884212D0FFE70498006846F2A0413B
:10A37000C4F20201884209D0FFE70498006846F25F
:10A38000B841C4F20201884201D1FFE707E045F27B
:10A390001B00C0F60200B82113F06CF9FFE7049827
:10A3A000406850B3FFE704984068B0F1007F24D0C4
:10A3B000FFE704984068B0F1806F1ED0FFE7049873
:10A3C0004068B0F1C06F18D0FFE704984068B0F162
:10A3D000006F12D0FFE704984068B0F1206F0CD0F6
:10A3E000FFE704984068B0F1406F06D0FFE704989B
:10A3F0004068B0F1606F01D1FFE707E045F21B0054
:10A40000C0F60200B92113F035F9FFE7049880681F
:10A4100050B1FFE704988068402805D0FFE7049812
:10A420008068802801D1FFE707E045F21B00C0F6F5
:10A430000200BA2113F01EF9FFE70498C068B0F5D6
:10A44000007F04D0FFE70498C06808B9FFE707E081
:10A4500045F21B00C0F60200BB2113F00BF9FFE729
:10A4600004980069B0F5806F04D0FFE70498006994
:10A4700008B9FFE707E045F21B00C0F60200BC2167
:10A4800013F0F8F8FFE70498406960B1FFE704981B
:10A490004069B0F5006F06D0FFE704984069B0F559
:10A4A000805F01D1FFE707E045F21B00C0F6020024
:10A4B000BD2113F0DFF8FFE70498806960B1FFE782
:10A4C00004988069B0F5005F06D0FFE704988069C2
:10A4D000B0F5804F01D1FFE707E045F21B00C0F661
:10A4E0000200BE2113F0C6F8FFE70498C06958B116
:10A4F000FFE70498C069B0F5807F05D0FFE70498B6
:10A50000C069202801D1FFE707E045F21B00C0F633
:10A510000200BF2113F0AEF8FFE70498006A90B183
:10A52000FFE70498006AB0F5803F0CD0FFE704987D
:10A53000006AB0F5003F06D0FFE70498006AB0F566
:10A54000403F01D1FFE707E045F21B00C0F60200E3
:10A55000C02113F08FF8FFE70498406A28B1FFE7A5
:10A560000498406A042801D1FFE707E045F21B0088
:10A57000C0F60200C12113F07DF8FFE70498406A9D
:10A5800000285BD0FFE70498806A78B1FFE7049861
:10A59000806A01280AD0FFE70498806A022805D063
:10A5A000FFE70498806A032801D1FFE707E045F23E
:10A5B0001B00C0F60200C62113F05CF8FFE7049808
:10A5C000C06A90B1FFE70498C06AB0F5000F0CD0E4
:10A5D000FFE70498C06AB0F1807F06D0FFE70498D7
:10A5E000C06AB0F1C07F01D1FFE707E045F21B0070
:10A5F000C0F60200C72113F03DF8FFE70498006B96
:10A6000090B1FFE70498006BB0F5001F0CD0FFE796
:10A610000498006BB0F5800F06D0FFE70498006B3C
:10A62000B0F5C00F01D1FFE707E045F21B00C0F60F
:10A630000200C82113F01EF8FFE7FFE7FFE70499C7
:10A64000002081F83400FFE70499022081F83500EA
:10A6500004980168086820F001000860FFE704988A
:10A6600000680068C00790B1FFE700F0CFFE0299D4
:10A67000401A06280AD3FFE7049920204865049968
:10A68000032081F835008DF8170076E0E7E704989D
:10A69000006800680390039848F23F01CFF2100170
:10A6A00008400390049900914868D1F808C0CB682D
:10A6B0000A6940EA0C00184310434A6910438A694A
:10A6C0001043CA691043096A014303980843039081
:10A6D0000498406A042808D1FFE70499C86A096B06
:10A6E0000143039808430390FFE70398049909681E
:10A6F00008600498006840690390039820F0070000
:10A7000003900498416A0398084303900498406AB0
:10A7100004281AD1FFE70498816A0398084303903C
:10A720000498C06A80B1FFE70498FCF777F850B14D
:10A73000FFE70499402048650499012081F835001D
:10A740008DF8170019E0FFE7FFE7039804990968FF
:10A7500048610498FCF736F801900498C16D3F20D9
:10A76000884001998860049900204865049A012175
:10A7700082F835108DF81700FFE79DF8170006B036
:10A7800080BD000080B588B00690059104920393C7
:10A7900000208DF80B000698806D0190039828B179
:10A7A000FFE7BDF80E0008B9FFE708E045F21B001F
:10A7B000C0F602004FF4E67112F05CFFFFE7FFE71E
:10A7C000069890F83400012804D1FFE702208DF8A4
:10A7D0001F0045E00699012081F83400FFE7FFE7FC
:10A7E000069890F8350001282BD1FFE70699022042
:10A7F00081F8350006990020486506980599049A65
:10A80000039BFCF783F80698C16D3F2088400199AF
:10A81000886006980168086840F01600086006988D
:10A82000006C38B1FFE706980168086840F008003E
:10A830000860FFE706980168086840F001000860BA
:10A8400009E0FFE70699002081F83400FFE70220C5
:10A850008DF80B00FFE79DF80B008DF81F00FFE758
:10A860009DF81F0008B080BD80B584B0039000F053
:10A87000CDFD0290039801900198013048B1FFE7A7
:10A8800040F29050C2F20000017801980844019013
:10A89000FFE7FFE700F0BAFD0299401A01998842EC
:10A8A00001D2FFE7F6E704B080BD000080B586B0B6
:10A8B0000490039101208DF80B0000200190FFE728
:10A8C00042F2B860C2F20000007E012804D1FFE726
:10A8D00002208DF8170094E042F2B861C2F2000144
:10A8E00001200876FFE7FFE70498006828B1FFE73A
:10A8F00004980068012801D1FFE707E044F6A5703D
:10A90000C0F60200AB2112F0B5FEFFE74CF250306A
:10A91000FCF7AAFC8DF80B009DF80B00002863D112
:10A92000FFE703994FF0FF300860049800680128A2
:10A9300014D1FFE70499087C4968FCF7D5FA4CF27A
:10A940005030FCF791FC8DF80B0043F61041C4F237
:10A950000201086820F00400086042E00498816861
:10A96000C068084440B1FFE704988168C0680844A3
:10A970000C2801D8FFE707E044F6A570C0F60200F6
:10A98000C32112F077FEFFE7049880680190FFE78B
:10A99000019804998A68C9681144884220D2FFE767
:10A9A00001980499097CFCF7B3F94CF25030FCF79C
:10A9B0005BFC8DF80B0043F61041C4F202010868FD
:10A9C00020F0FA0008609DF80B0020B1FFE7019825
:10A9D0000399086004E0FFE7019801300190D7E790
:10A9E000FFE7FCF72FFAFFE7FFE742F2B861C2F298
:10A9F000000100200876FFE79DF80B008DF8170096
:10AA0000FFE79DF8170006B080BD000043F6104137
:10AA1000C4F20201086840F000400860002070475E
:10AA200080B588B0069005910393029201208DF8BD
:10AA30000700FFE742F2B860C2F20000007E012882
:10AA400004D1FFE702208DF81F0069E042F2B861EF
:10AA5000C2F2000101200876FFE7FFE7069860B127
:10AA6000FFE70698012808D0FFE70698022804D0DF
:10AA7000FFE70698032801D1FFE707E044F66B7073
:10AA8000C0F60200A42112F0F5FDFFE74CF25030B1
:10AA9000FCF7EAFB8DF807009DF8070098BBFFE77D
:10AAA000069830B9FFE705989DF80810FCF762FAA0
:10AAB0001AE00698012806D1FFE70598BDF80810AE
:10AAC000FCF7DAFA0FE00698022805D1FFE70598AF
:10AAD0000299FCF711FB05E00598029A039BFCF72D
:10AAE00087FAFFE7FFE7FFE74CF25030FCF7BCFBCB
:10AAF0008DF8070043F61041C4F20201086820F007
:10AB000001000860FFE7FFE742F2B861C2F200010E
:10AB100000200876FFE79DF807008DF81F00FFE78B
:10AB20009DF81F0008B080BD81B000208DF80300A3
:10AB300043F61040C4F202000068C00FD8B1FFE72E
:10AB400043F60441C4F2020140F22310C4F26750FC
:10AB5000086048F6AB10CCF6EF50086043F61040A2
:10AB6000C4F202000068C00F20B1FFE701208DF899
:10AB70000300FFE7FFE79DF8030001B07047000006
:10AB800080B582B0ADF8060000208DF80500FFE723
:10AB90009DF805000F2824DCFFE7BDF806009DF8AE
:10ABA0000510C840C007A8B1FFE79DF8051040F2A6
:10ABB0002C60C2F2000050F8210050B1FFE79DF870
:10ABC000051040F22C60C2F2000050F821008047CE
:10ABD000FFE7FFE7FFE79DF8050001308DF805006E
:10ABE000D6E702B080BD000080B582B0ADF80600A7
:10ABF00043F61440C4F201000068BDF80610084294
:10AC00000CD0FFE7BDF8060043F61441C4F2010181
:10AC10000860BDF80600FFF7B3FFFFE702B080BD94
:10AC200080B58EB00D900C9100200A90099008908C
:10AC30000D980021C4F20201884240D0FFE70D9830
:10AC400040F20041C4F20201884238D0FFE70D987B
:10AC500040F60001C4F20201884230D0FFE70D98AF
:10AC600040F60041C4F20201884228D0FFE70D9867
:10AC700041F20001C4F20201884220D0FFE70D98A2
:10AC800041F20041C4F20201884218D0FFE70D985A
:10AC900041F60001C4F20201884210D0FFE70D988E
:10ACA00041F60041C4F20201884208D0FFE70D9846
:10ACB00042F20001C4F20201884201D1FFE707E03D
:10ACC00044F6E270C0F60200AC2112F0D3FCFFE7BC
:10ACD0000C98008828B1FFE70C98408808B9FFE776
:10ACE00007E044F6E270C0F60200AD2112F0C2FCAB
:10ACF000FFE70C984068002849D0FFE70C984068AF
:10AD0000012844D0FFE70C98406811283FD0FFE7A6
:10AD10000C98406802283AD0FFE70C984068122847
:10AD200035D0FFE70C9840680021C1F2110188423C
:10AD30002DD0FFE70C9840680021C1F22101884224
:10AD400025D0FFE70C9840680021C1F2310188420C
:10AD50001DD0FFE70C9840680021C1F21201884223
:10AD600015D0FFE70C9840680021C1F2220188420B
:10AD70000DD0FFE70C9840680021C1F232018842F3
:10AD800005D0FFE70C984068032801D1FFE707E0F2
:10AD900044F6E270C0F60200AE2112F06BFCFFE751
:10ADA0000C98806850B1FFE70C988068012805D0A6
:10ADB000FFE70C988068022801D1FFE707E044F61E
:10ADC000E270C0F60200AF2112F054FCFFE7002051
:10ADD0000B90FFE70B980F2800F2B082FFE70B996A
:10ADE000012088400A900C9800680A990840099050
:10ADF00009980A99884240F09C82FFE70C984068C5
:10AE000000F00300012807D0FFE70C98406800F02D
:10AE1000030002284BD1FFE70C98C06878B1FFE728
:10AE20000C98C06801280AD0FFE70C98C068022877
:10AE300005D0FFE70C98C068032801D1FFE707E0C1
:10AE400044F6E270C0F60200C12112F013FCFFE7E5
:10AE50000D98806808900B984100032000FA01F1DA
:10AE60000898884308900C98C0680B99490000FA2C
:10AE700001F108980843089008980D9988600D988A
:10AE8000406808900B99012000FA01F10898884366
:10AE900008900C984068C0F300100B9900FA01F17B
:10AEA00008980843089008980D994860FFE70C98A7
:10AEB000406800F00300032818D0FFE70D98C06831
:10AEC00008900B984100032000FA01F1089888438C
:10AED00008900C9880680B99490000FA01F10898D5
:10AEE0000843089008980D99C860FFE70C984068DF
:10AEF00000F00300022840F0EE80FFE70C980069A4
:10AF0000002800F0B980FFE70C980069092800F0DC
:10AF1000B380FFE70C980069002800F0AD80FFE7E0
:10AF20000C980069002800F0A780FFE70C980069E2
:10AF3000002800F0A180FFE70C980069002800F0CD
:10AF40009B80FFE70C980069012800F09580FFE7DF
:10AF50000C980069012800F08F80FFE70C980069C9
:10AF6000022800F08980FFE70C980069022800F0B1
:10AF70008380FFE70C98006902287DD0FFE70C98DA
:10AF80000069032878D0FFE70C980069042873D083
:10AF9000FFE70C98006904286ED0FFE70C98006961
:10AFA000042869D0FFE70C980069052864D0FFE702
:10AFB0000C98006905285FD0FFE70C980069092804
:10AFC0005AD0FFE70C980069062855D0FFE70C9887
:10AFD0000069092850D0FFE70C98006907284BD07A
:10AFE000FFE70C980069072846D0FFE70C98006936
:10AFF000072841D0FFE70C98006908283CD0FFE7FC
:10B000000C980069082837D0FFE70C9800690828D9
:10B0100032D0FFE70C98006909282DD0FFE70C9883
:10B020000069092828D0FFE70C9800690A2823D076
:10B03000FFE70C9800690A281ED0FFE70C9800690A
:10B040000B2819D0FFE70C9800690C2814D0FFE7F3
:10B050000C9800690C280FD0FFE70C9800690D28A8
:10B060000AD0FFE70C9800690C2805D0FFE70C9880
:10B0700000690F2801D1FFE707E044F6E270C0F64F
:10B080000200DC2112F0F6FAFFE70D980B996FF041
:10B09000030202EA51010844006A08900B9800F08C
:10B0A000070081000F2000FA01F1089888430890FA
:10B0B0000C9800690B9901F00701890000FA01F171
:10B0C00008980843089008980D990B9B02EA5302D0
:10B0D00011440862FFE70D98006808900B98410042
:10B0E000032000FA01F10898884308900C98406802
:10B0F00000F003000B99490000FA01F10898084399
:10B10000089008980D9908600C98C079C00600282E
:10B1100040F10E81FFE7FFE70020079043F644006F
:10B12000C4F20200016841F480410160006800F44B
:10B13000804007900798FFE70B9820F0030043F644
:10B140000801C4F20101405808900B9800F0030078
:10B1500081000F2000FA01F10898884308900D98AB
:10B160000021C4F20201884203D1FFE700200690CB
:10B170005EE00D9840F20041C4F20201884203D122
:10B18000FFE70120059050E00D9840F60001C4F261
:10B190000201884203D1FFE70220049042E00D98AB
:10B1A00040F60041C4F20201884203D1FFE70320C8
:10B1B000039034E00D9841F20001C4F2020188428C
:10B1C00003D1FFE70420029026E00D9841F20041F0
:10B1D000C4F20201884203D1FFE70520019018E084
:10B1E0000D9841F60001C4F20201884203D1FFE745
:10B1F000062000900AE00D9941F60042C4F20202D6
:10B200000820914208BF07200090FFE700980190B6
:10B21000FFE701980290FFE702980390FFE7039889
:10B220000490FFE704980590FFE705980690FFE774
:10B230000698C0B20B9901F00301890000FA01F1F0
:10B2400008980843089008980B9921F0030143F6E9
:10B250000802C4F20102885043F60040C4F2010023
:10B260000068089009990898884308900C9880799C
:10B27000C00728B1FFE70999089808430890FFE73D
:10B28000089843F60041C4F20101086043F6044007
:10B29000C4F2010000680890099908988843089052
:10B2A0000C9880798007002805D5FFE70999089850
:10B2B00008430890FFE7089843F60441C4F20101EF
:10B2C000086043F60840C4F201000068089009993C
:10B2D0000898884308900C988079C006002805D506
:10B2E000FFE70999089808430890FFE7089843F694
:10B2F0000841C4F20101086043F60C40C4F20100A9
:10B300000068089009990898884308900C988079FB
:10B310008006002805D5FFE709990898084308909A
:10B32000FFE7089843F60C41C4F201010860FFE70B
:10B33000FFE7FFE70B9801300B904BE50EB080BDA7
:10B3400080B582B00190ADF80210BDF8020020B1C6
:10B35000FFE7002008B9FFE708E044F6E270C0F616
:10B3600002004FF4BD7112F085F9FFE70198006902
:10B37000BDF80210084204D0FFE701208DF801005B
:10B3800003E000208DF80100FFE79DF8010002B006
:10B3900080BD000080B582B00190ADF802108DF83C
:10B3A0000120BDF8020020B1FFE7002008B9FFE747
:10B3B00008E044F6E270C0F6020040F29B1112F081
:10B3C00059F9FFE79DF8010028B1FFE79DF801005A
:10B3D000012801D1FFE708E044F6E270C0F6020060
:10B3E0004FF4CE7112F046F9FFE79DF8010028B145
:10B3F000FFE7BDF802000199886105E0BDF8020091
:10B40000000401998861FFE702B080BD49F69410FD
:10B41000C2F200000068704780B58EB00C900C98A6
:10B4200020B9FFE701208DF8370002E20C98006890
:10B4300045F20041C4F20001884212D0FFE70C98A7
:10B44000006845F60001C4F20001884209D0FFE718
:10B450000C98006845F60041C4F20001884201D111
:10B46000FFE708E045F23610C0F6020040F2BF11D7
:10B4700012F000F9FFE70C98406850B1FFE70C9814
:10B48000406841F68021C0F20601884201D8FFE7FA
:10B4900008E045F23610C0F602004FF4E07112F0F9
:10B4A000E9F8FFE70C98806830B1FFE70C988068F6
:10B4B000B0F5804F01D1FFE708E045F23610C0F645
:10B4C000020040F2C11112F0D5F8FFE70C98C068F5
:10B4D000800A08B9FFE708E045F23610C0F602001E
:10B4E0004FF4E17112F0C6F8FFE70C980069B0F56F
:10B4F000804F06D0FFE70C980069B0F5404F01D1AE
:10B50000FFE708E045F23610C0F6020040F2C31132
:10B5100012F0B0F8FFE70C98406928B1FFE70C98EB
:10B520004069012801D1FFE708E045F23610C0F676
:10B5300002004FF4E27112F09DF8FFE70C98806969
:10B540006FF0FE01084201D1FFE708E045F2361036
:10B55000C0F6020040F2C51112F08CF8FFE70C981B
:10B56000C06928B1FFE70C98C069402801D1FFE706
:10B5700008E045F23610C0F602004FF4E37112F015
:10B5800079F8FFE70C98006A28B1FFE70C98006A89
:10B59000802801D1FFE708E045F23610C0F602002E
:10B5A00040F2C71112F066F8FFE70C9890F83D00E2
:10B5B00040B9FFE70C99002081F83C000C9800F09E
:10B5C0003DF9FFE70C99242081F83D000C980168B3
:10B5D000086820F0010008600C980168086840F4D1
:10B5E000004008600C980168086820F4004008607A
:10B5F00001F054FE0A900C98406848F2A061C0F235
:10B60000010188420BD8FFE70A9948F28042C0F254
:10B610001E020020914238BF012009900AE00A99D9
:10B6200040F60012C0F23D020020914238BF0120D6
:10B630000990FFE70998012804D1FFE701208DF860
:10B640003700F6E00A984DF68361C4F21B31A0FB87
:10B650000110800C0B900C980068406820F03F00AF
:10B660000B9908430C99096848600C980068006AB7
:10B6700020F03F0008900C98406848F2A061C0F2AA
:10B680000101884204D8FFE70B98013007900EE0D3
:10B690000B984FF49671484344F6D351C1F26201BE
:10B6A000A0FB0101012000EB91100790FFE7089833
:10B6B000079908430C99096808620C980068C069EA
:10B6C0004CF6FF71884306900C98406848F2A061E0
:10B6D000C0F2010188421FD8FFE70A9801380C998F
:10B6E00049684900B0FBF1F001306FF31F300328C7
:10B6F00003D8FFE7042005900BE00A9801380C9965
:10B7000049684900B0FBF1F001306FF31F3005903C
:10B71000FFE7059804904CE00C98806868B9FFE753
:10B720000A9801380C99496801EB4101B0FBF1F02E
:10B7300001306FF31F3003900DE00A9801380C9927
:10B74000496819225143B0FBF1F00130042161F343
:10B750001F300390FFE70398000518B9FFE70120A9
:10B76000029023E00C98806868B9FFE70A980138D6
:10B770000C99496801EB4101B0FBF1F001306FF326
:10B780001F3001900DE00A9801380C994968192280
:10B790005143B0FBF1F00130042161F31F300190FF
:10B7A000FFE7019840F400400290FFE70298049000
:10B7B000FFE70698049908430C990968C8610C983A
:10B7C0000068006820F0C0000C9B1968DA691B6AE9
:10B7D0001A43104308600C980068806848F2FF31F3
:10B7E00088430C9A1168D36812691A431043886021
:10B7F0000C980068C06820F0FF000C9B19685A691B
:10B800009B691A431043C8600C980168086840F0AF
:10B81000010008600C99002008640C9A202182F82D
:10B820003D100C9908630C9981F83E008DF83700A3
:10B83000FFE79DF837000EB080BD000080B594B0E2
:10B84000139000201290119010900F900E9013986A
:10B85000006845F20041C4F20001884235D1FFE79B
:10B86000FFE700200D9043F63000C4F202000168AB
:10B8700041F002010160006800F002000D900D9897
:10B88000FFE74FF440700E9012200F9001201090AF
:10B89000032011900420129040F20040C4F20200F4
:10B8A0000EA9FFF7BDF9FFE700200C9043F640001A
:10B8B000C4F20200016841F400110160006800F464
:10B8C00000100C900C98FFE7FBE01398006845F619
:10B8D0000001C4F2000188425FD1FFE7FFE70020CA
:10B8E0000B9043F63000C4F20200016841F02001E1
:10B8F0000160006800F020000B900B98FFE7032028
:10B900000E9012210F91012110911190042012909C
:10B9100041F20040C4F202000EA9FFF781F9FFE7EF
:10B9200000200A9043F64000C4F20200016841F48E
:10B9300080010160006800F480000A900A98FFE727
:10B9400041F65820C2F20000069046F2B801C4F257
:10B95000020101604FF0606141604021816000217F
:10B96000C1604FF48062026141618161C1614FF445
:10B97000003202624162FEF769FC18B1FFE7FBF793
:10B98000C3F9FFE7FFE7139841F65821C2F200011F
:10B99000416313988863FFE792E01398006845F6C7
:10B9A0000041C4F20001884240F08980FFE7FFE7D0
:10B9B0000020099043F63000C4F20200016841F013
:10B9C00004010160006800F0040009900998FFE795
:10B9D000FFE70020089043F63000C4F2020001683F
:10B9E00041F001010160006800F001000890089832
:10B9F000FFE74FF400700E90122001900F9001208D
:10BA00000290109003200390119004200490129053
:10BA100040F60000C4F202000EA90591FFF700F9FC
:10BA2000DDF804C0029B039A049805994FF4807EC8
:10BA3000CDF838E0CDF83CC0109311921290002060
:10BA4000C4F20200FFF7ECF8FFE70020079043F68E
:10BA50004000C4F20200016841F400010160006886
:10BA600000F4000007900798FFE741F6B820C2F203
:10BA70000000009046F24001C4F2020101604FF064
:10BA8000C061416000218160C1604FF48062026149
:10BA900041618161C16101624162FEF7D7FB18B16A
:10BAA000FFE7FBF731F9FFE7FFE7139841F6B8210D
:10BAB000C2F20001816313988863FFE7FFE7FFE7A5
:10BAC000FFE714B080BD000040F29050C2F20000C9
:10BAD000027849F69411C2F2000108681044086027
:10BAE0007047000080B543F60041C4F202010868C7
:10BAF00040F400700860086840F4806008600868DE
:10BB000040F480700860032000F0D0F80F2000F0AF
:10BB100005F800F03BF8002080BD000080B582B041
:10BB2000009040F22800C2F20000006840F29051FC
:10BB3000C2F200010A784FF47A71B1FBF2F1B0FB66
:10BB4000F1F003F005FB20B1FFE701208DF80700BD
:10BB500018E000980F280DD8FFE700994FF0FF304C
:10BB6000002200F06FF8009840F29451C2F20001F8
:10BB7000086003E001208DF8070003E000208DF845
:10BB80000700FFE79DF8070002B080BD80B582B0D6
:10BB9000FFE70020019043F64400C4F20200016870
:10BBA00041F480410160006800F4804001900198F8
:10BBB000FFE7FFE70020009043F64000C4F20200D8
:10BBC000016841F080510160006800F080500090F1
:10BBD0000098FFE76FF001000F21002200F032F81B
:10BBE00002B080BD80B582B08DF807009DF90700D6
:10BBF000002801D4FFE707E045F25300C0F6020039
:10BC0000CE2111F037FDFFE79DF9070011F094FCFC
:10BC100002B080BD80B582B08DF807009DF90700A5
:10BC2000002801D4FFE707E045F25300C0F6020008
:10BC3000BE2111F01FFDFFE79DF9070011F098FCF0
:10BC400002B080BD80B586B08DF8170004910392D4
:10BC50000020029003980F2801D8FFE707E045F283
:10BC60005300C0F60200AA2111F004FDFFE704987A
:10BC70000F2801D8FFE707E045F25300C0F60200A5
:10BC8000AB2111F0F7FCFFE711F08AFC02909DF95F
:10BC90001700019002980499039A07F0C5FE014627
:10BCA000019811F085FC06B080BD000080B582B01F
:10BCB00001900198072810D0FFE7019806280CD0C2
:10BCC000FFE70198052808D0FFE70198042804D071
:10BCD000FFE70198032801D1FFE707E045F2530091
:10BCE000C0F60200922111F0C5FCFFE7019811F0A7
:10BCF000A3FC02B080BD000082B001908DF803105B
:10BD000002B0704782B00190ADF80210BDF8020099
:10BD1000019909684862002002B0704784B003901E
:10BD20008DF80B10ADF8082003980068406A009069
:10BD30009DF80B0048B9FFE7BDF80810009840EAED
:10BD4000014003990968886233E003980068816ABA
:10BD5000009800EB1140009000208DF80700FFE7ED
:10BD60009DF807009DF80B100139884213D2FFE7B8
:10BD7000039800689DF8071000EB8100D0F80411CB
:10BD8000009800EB11400090FFE79DF8070001309C
:10BD90008DF80700E4E7BDF80810009840EA01407C
:10BDA000039909689DF80B2001EB8201C1F800019D
:10BDB000FFE7002004B0704780B582B00190019881
:10BDC000D0F804040FF01CFB02B080BD80B582B037
:10BDD00001908DF80310019AD2F804049DF8031025
:10BDE000C1EBC10302EB8302926C0FF0E7F902B0E2
:10BDF00080BD000080B582B001908DF80310019ADB
:10BE0000D2F804049DF80310C1EBC10302EB8302D6
:10BE1000D2F808220FF078FA02B080BD80B582B067
:10BE200001900198D0F804040FF0F0FA02B080BD40
:10BE300080B584B002908DF807109DF807000006C9
:10BE400000280FD5FFE702989DF8071001F00F01B9
:10BE5000C1EBC10100EB81003C3000900099012052
:10BE600048700FE002989DF8071001F00F01C1EB38
:10BE7000C10100EB810000F5FE70009000990020E8
:10BE80004870FFE79DF8070000F00F000099087068
:10BE9000FFE7029890F8BC03012804D1FFE70220D5
:10BEA0008DF80F0014E00299012081F8BC03FFE730
:10BEB000FFE702980068009910F06CFAFFE702991A
:10BEC000002081F8BC03FFE700208DF80F00FFE79A
:10BED0009DF80F0004B080BD80B584B002908DF84D
:10BEE00007109DF8070000F00F000299496888428A
:10BEF00004D9FFE701208DF80F004DE09DF8070001
:10BF0000000600280FD5FFE702989DF8071001F002
:10BF10000F01C1EBC10100EB81003C3000900099A2
:10BF2000012048700FE002989DF8071001F00F0102
:10BF3000C1EBC10100EB810000F5FE70009000999B
:10BF400000204870FFE70099002088709DF80700E6
:10BF500000F00F0000990870FFE7029890F8BC030A
:10BF6000012804D1FFE702208DF80F0014E00299A8
:10BF7000012081F8BC03FFE7FFE702980068009901
:10BF800010F08CFDFFE70299002081F8BC03FFE769
:10BF900000208DF80F00FFE79DF80F0004B080BD72
:10BFA00082B001908DF8031001989DF8031001F004
:10BFB0000F01C1EBC10100EB8100D0F8140202B007
:10BFC0007047000080B586B004908DF80F10ADF872
:10BFD0000C208DF80B3000208DF80A009DF80F0022
:10BFE000000600280FD5FFE704989DF80F1001F018
:10BFF0000F01C1EBC10100EB81003C3001900199C0
:10C00000012048700FE004989DF80F1001F00F0117
:10C01000C1EBC10100EB810000F5FE7001900199B8
:10C0200000204870FFE79DF80F0000F00F00019915
:10C030000870BDF80C00019988609DF80B0001990B
:10C04000C8700198407820B1FFE701990878C8804E
:10C05000FFE79DF80B00022804D1FFE701990020BB
:10C060000871FFE7FFE7049890F8BC03012804D1AA
:10C07000FFE702208DF8170015E00499012081F8F0
:10C08000BC03FFE7FFE704980068019910F03EF851
:10C09000FFE70499002081F8BC03FFE79DF80A0040
:10C0A0008DF81700FFE79DF8170006B080BD00006F
:10C0B00080B586B005908DF8131003920293059811
:10C0C0009DF8131001F00F01C1EBC10100EB8100DD
:10C0D00000F5FE70019003980199C86002980199DB
:10C0E0004861019900208861019948709DF813000A
:10C0F00000F00F000199087005980069012804D12B
:10C10000FFE7039801990861FFE79DF81300000716
:10C1100038B9FFE7059A10680199127C10F076FB98
:10C1200006E0059A10680199127C10F05BFDFFE7AC
:10C13000002006B080BD000080B584B002908DF86C
:10C1400007109DF8070000F00F0002994968884227
:10C1500004D9FFE701208DF80F0058E09DF8070093
:10C16000000600280FD5FFE702989DF8071001F0A0
:10C170000F01C1EBC10100EB81003C300090009940
:10C18000012048700DE002989DF80710C1EBC10135
:10C1900000EB810000F5FE700090009900204870CF
:10C1A000FFE70099012088709DF8070000F00F005C
:10C1B00000990870FFE7029890F8BC03012804D1A9
:10C1C000FFE702208DF80F0021E00299012081F89D
:10C1D000BC03FFE7FFE702980068009910F0AEFC8F
:10C1E0009DF80700000740B9FFE7029A1068117C2C
:10C1F00002F5717210F002FCFFE7FFE702990020E0
:10C2000081F8BC03FFE700208DF80F00FFE79DF8E1
:10C210000F0004B080BD000080B586B005908DF899
:10C2200013100392029305989DF8131001F00F016B
:10C23000C1EBC10100EB81003C30019003980199F2
:10C24000C8600298019948610199002088610199AC
:10C25000012048709DF8130000F00F00019908704C
:10C2600005980069012804D1FFE703980199086146
:10C27000FFE79DF81300000738B9FFE7059A10683B
:10C280000199127C10F0C2FA06E0059A1068019933
:10C29000127C10F0A7FCFFE7002006B080BD000074
:10C2A00080B58CB00B900B9800680A900A980990A2
:10C2B0000B98006810F0C8FE002840F01A83FFE7D2
:10C2C0000B98006810F02CFF08B9FFE711E30B98FA
:10C2D000006810F025FF8007002807D5FFE70B98BE
:10C2E0000168486900F002004861FFE70B980068A8
:10C2F00010F016FFC006002862D5FFE70B98016812
:10C30000886920F0100088610A98006A03900B98F1
:10C31000039901F00F01C1EBC10100EB810000F5B1
:10C32000FE700290039800F4F0110220B0EB514F20
:10C3300023D1FFE7BDF80C0047F6F07108421BD08F
:10C34000FFE70A980299C968039AC2F30A1210F02B
:10C35000F5FE039847F6F07100EA0103029AD068EF
:10C3600000EB1310D060039800EA0102029988697B
:10C3700000EB12108861FFE71BE0039800F4F01156
:10C380000620B0EB514F12D1FFE70A980B9901F547
:10C390007171082210F0D2FE039847F6F07100EA9E
:10C3A00001020299886900EB1210886100E0FFE742
:10C3B000FFE70B980168886940F010008861FFE78B
:10C3C0000B98006810F0ACFE0003002870D5FFE762
:10C3D000002005900B98006810F050FE0790FFE7D2
:10C3E0000798002863D0FFE79DF81C00C0070028CD
:10C3F00056D0FFE70B9800689DF8141010F078FEF7
:10C4000006909DF81800C00760B1FFE709980599EC
:10C4100000EB41110120C1F8080B0B98059907F0BA
:10C4200087FBFFE79DF81800000700280CD5FFE701
:10C430000998059900EB41110820C1F8080B0B98E9
:10C44000059907F02FFBFFE79DF81800C0060028AC
:10C4500008D5FFE70998059900EB41111020C1F8B4
:10C46000080BFFE79DF818008006002808D5FFE7B5
:10C470000998059900EB41112020C1F8080BFFE74E
:10C480009DF819008006002809D5FFE7099805994D
:10C4900000EB41114FF40050C1F8080BFFE7FFE734
:10C4A00005980130059007984008079098E7FFE746
:10C4B0000B98006810F034FE4003002840F1AC8077
:10C4C000FFE70B98006810F0C7FD0790002005906B
:10C4D000FFE70798002800F09E80FFE79DF81C000A
:10C4E000C007002800F09080FFE70B9800689DF8D7
:10C4F000141010F0D5FD06909DF81800C007002814
:10C500003ED0FFE7059800F00F01012000FA01F18D
:10C510000491049B099AD2F834189943C2F834184C
:10C520000999059A01EB4211C1F808090B980069B5
:10C5300001281FD1FFE70B980599C1EBC10100EB62
:10C5400081014A6C886C10448864059888B9FFE7BB
:10C550000B980599C1EBC10100EB8100006D40B95A
:10C56000FFE70B99086801F57172012110F046FA96
:10C57000FFE7FFE70B989DF81410FFF727FCFFE794
:10C580009DF818000007002808D5FFE709980599CD
:10C5900000EB41110820C1F80809FFE79DF81800D9
:10C5A000C006002808D5FFE70998059900EB41115E
:10C5B0001020C1F80809FFE79DF818004006002880
:10C5C00008D5FFE70998059900EB41114020C1F813
:10C5D0000809FFE79DF818008007002808D5FFE745
:10C5E0000998059900EB41110220C1F80809FFE7FD
:10C5F0009DF818000006002805D5FFE70B9805995F
:10C6000007F088FBFFE7FFE70598013005900798E2
:10C61000400807905DE7FFE70B98006810F080FD89
:10C62000C00F00B3FFE70999D1F8040820F001001A
:10C63000C1F804080B9890F8F403012808D1FFE72B
:10C640000B98002180F8F4130B98FFF755FB03E0DB
:10C650000B9800F061FBFFE70B980168486900F058
:10C6600000404861FFE70B98006810F059FD000595
:10C67000002811D5FFE70998D0F80808C00720B1B5
:10C68000FFE70B9800F0D6FBFFE70B9801684869BD
:10C6900000F400604861FFE70B98006810F040FD6F
:10C6A000C004002840F19080FFE70999D1F8040800
:10C6B00020F00100C1F804080B980068102110F068
:10C6C00073FC00200890FFE708980B99496888429E
:10C6D0003BD2FFE70998089900EB41114FF67F30F4
:10C6E000C1F808090999089A01EB4212D2F8001919
:10C6F00021F40011C2F800190999089A01EB4212BD
:10C70000D2F8001941F00061C2F800190999089A9D
:10C7100001EB4211C1F8080B0998089900EB41118F
:10C72000D1F8000B20F40010C1F8000B099808990B
:10C7300000EB4111D1F8000B40F00060C1F8000B94
:10C74000FFE7089801300890BEE70999D1F81C0866
:10C7500040F00110C1F81C080B98006B78B1FFE79E
:10C760000999D1F8840840F00B00C1F884080999B0
:10C77000D1F8440840F00B00C1F844080FE00999D3
:10C78000D1F8140842F22B021043C1F81408099999
:10C79000D1F8100840F00B00C1F81008FFE7099924
:10C7A000D1F8000820F4FE60C1F800080B9A106868
:10C7B000117C02F5717210F021F90B98016848693B
:10C7C00000F480504861FFE70B98006810F0A8FC67
:10C7D000800400281FD5FFE70B9800680FF006FDC6
:10C7E0000B98006810F00AFC0B99C8600B98006861
:10C7F000019000F04DFD014601980B9A127B10F05C
:10C8000023FD0B9800F05EFA0B980168486900F46C
:10C8100000504861FFE70B98006810F081FC0007AA
:10C8200000280AD5FFE70B9800F080FA0B98016802
:10C83000486900F008004861FFE70B98006810F0B5
:10C840006FFCC00200280ED5FFE7002005900B9872
:10C850009DF8141000F050F80B980168486900F436
:10C8600080104861FFE70B98006810F059FC8002C7
:10C8700000280ED5FFE7002005900B989DF81410B6
:10C8800000F048F80B980168486900F4001048610E
:10C89000FFE70B98006810F043FC400000280AD521
:10C8A000FFE70B98FFF788FA0B980168486900F0DA
:10C8B00080404861FFE70B98006810F031FC4007AA
:10C8C000002815D5FFE70B980068406803909DF895
:10C8D0000C004007002804D5FFE70B98FFF79EFAED
:10C8E000FFE7039A0B980168486810434860FFE728
:10C8F000FFE70CB080BD000080B582B001908DF8DC
:10C9000003100198D0F804049DF803100EF010FEF7
:10C9100002B080BD80B582B001908DF803100198FF
:10C92000D0F804049DF803100EF02EFE02B080BD76
:10C930002DE9F04F97B01590159820B9FFE7012029
:10C940008DF85B0060E115980068B0F1A04F08D049
:10C95000FFE7159800680021C4F20401884201D164
:10C96000FFE707E044F6FB60C0F60200872110F005
:10C9700081FEFFE7159800681490159890F8BD03A4
:10C9800040B9FFE71599002081F8BC03159800F025
:10C9900041F9FFE71599032081F8BD031498C06B96
:10C9A000C005002804D4FFE7159900200861FFE7BF
:10C9B000159800680FF020FF1598109001681191EC
:10C9C00041688268C368D0F810C044698569C66947
:10C9D000076AD0F82480D0F82890D0F82CA0D0F89E
:10C9E00030B0D0F834E068461290C0F824E01198D6
:10C9F000DDF848E0CEF820B0CEF81CA0CEF81890B4
:10CA0000CEF81480CEF81070CEF80C60CEF8085036
:10CA1000CEF80440CEF800C00FF0FEFB40B1FFE7B7
:10CA20001599022081F8BD0301208DF85B00EBE031
:10CA30001598006800210F9110F0A8FB0F988DF851
:10CA40004F00FFE79DF84F0015994968884245D28D
:10CA5000FFE715989DF84F10C1EBC10100EB810174
:10CA6000012081F83D009DF84F001599C0EBC002F0
:10CA700001EB820181F83C009DF84F001599C0EB55
:10CA8000C00201EB8201A1F8420015989DF84F10F9
:10CA9000C1EBC10100EB8101002081F83F00159935
:10CAA0009DF84F20C2EBC20201EB82014864159948
:10CAB0009DF84F20C2EBC20201EB820188641599F8
:10CAC0009DF84F20C2EBC20201EB82010865FFE72F
:10CAD0009DF84F0001308DF84F00B3E700208DF82E
:10CAE0004F00FFE79DF84F001599496888423ED2F4
:10CAF000FFE715989DF84F10C1EBC10100EB8101D4
:10CB0000002081F8FD019DF84F10159AC1EBC1037B
:10CB100002EB830282F8FC1115999DF84F20C2EBBD
:10CB2000C20201EB820181F8FF0115999DF84F20A7
:10CB3000C2EBC20201EB8201C1F8040215999DF813
:10CB40004F20C2EBC20201EB8201C1F80802159925
:10CB50009DF84F20C2EBC20201EB8201C1F8100226
:10CB6000FFE79DF84F0001308DF84F00BAE71598A8
:10CB70000C9001680D9141688268C368D0F810C0BC
:10CB800044698569C669076AD0F82480D0F828907E
:10CB9000D0F82CA0D0F830B0D0F834E068460E9031
:10CBA000C0F824E00D98DDF838E0CEF820B0CEF8DB
:10CBB0001CA0CEF81890CEF81480CEF81070CEF8E5
:10CBC0000C60CEF80850CEF80440CEF800C00FF04C
:10CBD000B1FC40B1FFE71599022081F8BD030120A7
:10CBE0008DF85B0010E0159900200B9081F838005B
:10CBF0001599012081F8BD03159800680FF084FC99
:10CC00000B988DF85B00FFE79DF85B0017B0BDE85F
:10CC1000F08F000080B58AB009900020089007903E
:10CC200006900590049009980068B0F1A04F47D194
:10CC3000FFE7FFE70020039043F63000C4F2020054
:10CC4000016841F001010160006800F001000390FB
:10CC50000398FFE74FF4C050049002200590002095
:10CC60000690032007900A2008900020C4F20200DA
:10CC700004A9FDF7D5FFFFE743F63401C4F2020132
:10CC8000086840F080000860FFE70020029043F64B
:10CC90004400C4F20200016841F480410160006870
:10CCA00000F4804002900298FFE7FFE743200190E4
:10CCB00005210022FEF7C6FF0198FEF7ABFFFFE754
:10CCC0000AB080BD80B582B0019001208DF80300CC
:10CCD0000198C06820B9FFE700208DF803000CE040
:10CCE0000198C068022804D1FFE701208DF80300F5
:10CCF00002E0FAF709F8FFE7FFE70198D0F804042B
:10CD00009DF803100EF03EFD0198D0F804040EF0DB
:10CD1000AFFC02B080BD000080B582B001900198E8
:10CD2000D0F804040EF0F4FC02B080BD80B582B0EF
:10CD300001900198D0F804040EF0FCFC02B080BD14
:10CD400080B584B002908DF80710FFE7029890F844
:10CD5000BC03012804D1FFE702208DF80F001AE080
:10CD60000299012081F8BC03FFE7FFE79DF8070067
:10CD7000029981F83800029800689DF8071010F0B9
:10CD800035FAFFE70299002081F8BC03FFE7002095
:10CD90008DF80F00FFE79DF80F0004B080BD000084
:10CDA00080B582B001900199D1F8040401F5717148
:10CDB0000EF012FD02B080BD80B584B002900298E2
:10CDC00000680190FFE7029890F8BC03012804D1A5
:10CDD000FFE702208DF80F0027E00299012081F87B
:10CDE000BC03FFE7FFE70298806A01280BD1FFE749
:10CDF00002988069012806D0FFE70199886B40F40A
:10CE000080308863FFE70298006810F09DF8029870
:10CE100000680FF063FBFFE70299002081F8BC0374
:10CE2000FFE700208DF80F00FFE79DF80F0004B02A
:10CE300080BD000080B582B001900198D0F8040454
:10CE40000EF04CFD01980168D1F8000E40F0010091
:10CE5000C1F8000E0198006A48B1FFE74EF6105184
:10CE6000CEF20001086840F006000860FFE702B05B
:10CE700080BD000080B584B002900191029820B975
:10CE8000FFE701208DF80F00FDE10298006830B146
:10CE9000FFE7029800680F2801D8FFE708E044F692
:10CEA0003370C0F602004FF4177110F0E3FBFFE798
:10CEB0000198E0B1FFE70198012818D0FFE7019839
:10CEC000022814D0FFE70198032810D0FFE701984B
:10CED00004280CD0FFE70198052808D0FFE7019847
:10CEE000062804D0FFE70198072801D1FFE708E0F2
:10CEF00044F63370C0F6020040F25D2110F0BAFB38
:10CF0000FFE7019843F60041C4F20201096801F00D
:10CF10000701884212D9FFE7019943F60040C4F2A5
:10CF200002000170006800F007000199884204D0F7
:10CF3000FFE701208DF80F00A5E1FFE702980078D8
:10CF40008007002860D5FFE7029800784007002896
:10CF500009D5FFE743F60801C4F20201086840F46E
:10CF6000E0500860FFE7029800780007002809D524
:10CF7000FFE743F60801C4F20201086840F460408C
:10CF80000860FFE70298806840B3FFE70298806876
:10CF9000802823D0FFE70298806890281ED0FFE702
:10CFA00002988068A02819D0FFE702988068B0280E
:10CFB00014D0FFE702988068C0280FD0FFE70298DE
:10CFC0008068D0280AD0FFE702988068E02805D062
:10CFD000FFE702988068F02801D1FFE708E044F6F7
:10CFE0003370C0F602004FF4207110F043FBFFE7EE
:10CFF00043F60801C4F20201086820F0F000029A2A
:10D00000926810430860FFE702980078C007002884
:10D0100000F08C80FFE70298406878B1FFE7029843
:10D02000406801280AD0FFE702984068022805D02E
:10D03000FFE702984068032801D1FFE708E044F6C3
:10D040003370C0F6020040F2872110F013FBFFE7B7
:10D0500002984068012811D1FFE743F60000C4F2AE
:10D060000200006800F400310020B0EB514F04D101
:10D07000FFE701208DF80F0005E12CE002984068E1
:10D08000022805D0FFE702984068032811D1FFE786
:10D0900043F60000C4F20200006800F000710020B6
:10D0A000B0EB516F04D1FFE701208DF80F00EAE0EB
:10D0B00010E043F60000C4F20200006800F0020134
:10D0C0000020B0EB510F04D1FFE701208DF80F00D5
:10D0D000D9E0FFE7FFE743F60801C4F20201086860
:10D0E00020F00300029A526810430860FEF78EF9A0
:10D0F0000090FFE743F60800C4F20200006800F069
:10D100000C0002994968B0EB810F0ED0FFE7FEF7E3
:10D110007DF90099401A41F28931884204D3FFE732
:10D1200003208DF80F00AEE0E4E7FFE7019843F637
:10D130000041C4F20201096801F00701884212D2DD
:10D14000FFE7019943F60040C4F202000170006855
:10D1500000F007000199884204D0FFE701208DF814
:10D160000F0090E0FFE7029800784007002832D5D2
:10D17000FFE70298C068C0B1FFE70298C068B0F549
:10D18000805F12D0FFE70298C068B0F5A05F0CD0B6
:10D19000FFE70298C068B0F5C05F06D0FFE70298CD
:10D1A000C068B0F5E05F01D1FFE708E044F63370F6
:10D1B000C0F6020040F2C52110F05CFAFFE743F62A
:10D1C0000801C4F20201086820F4E050029AD26813
:10D1D00010430860FFE7029800780007002833D565
:10D1E000FFE702980069C0B1FFE702980069B0F557
:10D1F000805F12D0FFE702980069B0F5A05F0CD005
:10D20000FFE702980069B0F5C05F06D0FFE702981B
:10D210000069B0F5E05F01D1FFE708E044F6337044
:10D22000C0F602004FF4337110F024FAFFE743F622
:10D230000801C4F20201086820F46040029A1269F1
:10D2400040EAC2000860FFE700F04CF843F608012E
:10D25000C4F202010968C9B20A0944F20071C0F6B9
:10D260000201895CC84040F22801C2F20001086056
:10D2700040F29450C2F200000068FEF74FFC00201C
:10D280008DF80F00FFE79DF80F0004B080BD00008F
:10D2900040F22800C2F200000068704780B5FFF736
:10D2A000F7FF43F60801C4F202010968C1F38222C4
:10D2B00044F21071C0F60201895CC84080BD0000D4
:10D2C00080B5FFF7E5FF43F60801C4F202010968E3
:10D2D00089B24A0B44F21071C0F60201895CC84061
:10D2E00080BD000080B586B00020059004900390BA
:10D2F000029043F60800C4F20200006800F00C003F
:10D300000146019140B1FFE7019804280AD0FFE7E8
:10D31000019808280CD04FE042F20040C0F2F4001F
:10D3200002904FE041F60030C0F2B700029049E0B1
:10D3300043F60400C4F20200016801F03F010591C8
:10D3400000684002002813D5FFE743F60400C4F24A
:10D3500002000068C0F3881041F60031C0F2B70146
:10D36000A0FB0101059A0023F2F72AFF049012E0C6
:10D3700043F60400C4F202000068C0F3881042F2D1
:10D380000041C0F2F401A0FB0101059A0023F2F76D
:10D3900017FF0490FFE743F60400C4F202000068A0
:10D3A00000F44031022000EBD1300390049803993F
:10D3B000B0FBF1F0029005E042F20040C0F2F40050
:10D3C0000290FFE7029806B080BD000080B586B0ED
:10D3D0000490049828B9FFE701208DF8170000F0A9
:10D3E00048BC049800680F2801D8FFE707E044F61E
:10D3F0003370C0F60200E82110F03CF9FFE7049812
:10D400000078C007002800F0BE80FFE7049840685D
:10D4100060B1FFE704984068B0F5803F06D0FFE7B1
:10D4200004984068B0F5A02F01D1FFE707E044F66B
:10D430003370C0F60200ED2110F01CF9FFE743F64F
:10D440000800C4F20200006800F00C00042813D0A9
:10D45000FFE743F60800C4F20200006800F00C0089
:10D4600008281ED1FFE743F60400C4F2020000685A
:10D470004002002815D5FFE743F60000C4F2020081
:10D48000006800F400310020B0EB514F08D0FFE7F6
:10D490000498406820B9FFE701208DF81700E8E301
:10D4A00070E0FFE704984068B0F5803F09D1FFE7DE
:10D4B00043F60001C4F20201086840F480300860BD
:10D4C00020E004984068B0F5A02F0DD1FFE743F6A7
:10D4D0000001C4F20201086840F480200860086876
:10D4E00040F4803008600CE043F60001C4F2020111
:10D4F000086820F480300860086820F48020086004
:10D50000FFE7FFE7FFE704984068E8B1FFE7FDF7B2
:10D510007DFF0390FFE743F60000C4F202000068BD
:10D5200000F400310020B0EB514F0CD1FFE7FDF7C4
:10D530006DFF0399401A652804D3FFE703208DF897
:10D54000170096E3E7E71CE0FDF760FF0390FFE7B5
:10D5500043F60000C4F20200006800F4003100202D
:10D56000B0EB514F0CD0FFE7FDF750FF0399401A85
:10D57000652804D3FFE703208DF8170079E3E7E778
:10D58000FFE7FFE7FFE7049800788007002840F1F5
:10D59000B880FFE70498C06828B1FFE70498C06826
:10D5A000012801D1FFE708E044F63370C0F602001D
:10D5B00040F21F1110F05EF8FFE7049800691F2881
:10D5C00001D8FFE708E044F63370C0F602004FF4DC
:10D5D000907110F04FF8FFE743F60800C4F2020024
:10D5E000006810F00C0F13D0FFE743F60800C4F2F8
:10D5F0000200006800F00C0008282CD1FFE743F679
:10D600000400C4F2020000684002002823D4FFE7AF
:10D6100043F60000C4F20200006800F0020100209E
:10D62000B0EB510F09D0FFE70498C068012804D07F
:10D63000FFE701208DF817001BE343F60001C4F259
:10D640000201086820F0F800049A126940EAC2005A
:10D650000860FFE754E00498C06870B3FFE700215A
:10D66000C4F2472101200860FDF7D0FE0390FFE7D8
:10D6700043F60000C4F20200006800F0020100203E
:10D68000B0EB510F0CD1FFE7FDF7C0FE0399401A34
:10D69000032804D3FFE703208DF81700E9E2E7E74A
:10D6A00043F60001C4F20201086820F0F800049A71
:10D6B000126940EAC200086021E00021C4F247215B
:10D6C00000200860FDF7A2FE0390FFE743F600008C
:10D6D000C4F20200006800F002010020B0EB510F1C
:10D6E0000CD0FFE7FDF792FE0399401A032804D3FC
:10D6F000FFE703208DF81700BBE2E7E7FFE7FFE74E
:10D70000FFE704980078000700285ED5FFE704983B
:10D71000406928B1FFE704984069012801D1FFE77B
:10D7200008E044F63370C0F602004FF4B0710FF019
:10D73000A1FFFFE70498406918B3FFE740F6806156
:10D74000C4F2472101200860FDF760FE0390FFE767
:10D7500043F67400C4F20200006800F002010020E9
:10D76000B0EB510F0CD1FFE7FDF750FE0399401AC3
:10D77000032804D3FFE703208DF8170079E2E7E7D9
:10D7800022E040F68061C4F2472100200860FDF7E6
:10D790003DFE0390FFE743F67400C4F20200006808
:10D7A00000F002010020B0EB510F0CD0FFE7FDF7B5
:10D7B0002DFE0399401A032804D3FFE703208DF8B8
:10D7C000170056E2E7E7FFE7FFE704980078400715
:10D7D000002840F1E680FFE700208DF8070004985C
:10D7E000806850B1FFE704988068012805D0FFE702
:10D7F00004988068052801D1FFE708E044F63370FB
:10D80000C0F602004FF4C6710FF034FFFFE743F695
:10D810004000C4F202000068C000002815D4FFE7F1
:10D82000FFE70020009043F64000C4F202000168C8
:10D8300041F080510160006800F080500090009835
:10D84000FFE701208DF80700FFE747F20000C4F270
:10D8500000000068C005002822D4FFE747F200015D
:10D86000C4F20001086840F480700860FDF7CEFD46
:10D870000390FFE747F20000C4F200000068C00513
:10D8800000280CD4FFE7FDF7C1FD0399401A0328D7
:10D8900004D3FFE703208DF81700EAE1EAE7FFE78A
:10D8A000FFE704988068012809D1FFE743F670017B
:10D8B000C4F20201086840F0010008601FE004980B
:10D8C000806805280DD1FFE743F67001C4F202011C
:10D8D000086840F004000860086840F00100086033
:10D8E0000CE043F67001C4F20201086820F0010068
:10D8F0000860086820F004000860FFE7FFE7FFE722
:10D9000004988068F8B1FFE7FDF780FD0390FFE71A
:10D9100043F67000C4F20200006800F0020100202B
:10D92000B0EB510F0ED1FFE7FDF770FD0399401AE0
:10D9300041F28931884204D3FFE703208DF81700B4
:10D9400097E1E5E71EE0FDF761FD0390FFE743F691
:10D950007000C4F20200006800F002010020B0EB89
:10D96000510F0ED0FFE7FDF751FD0399401A41F228
:10D970008931884204D3FFE703208DF8170078E14E
:10D98000E5E7FFE79DF80700012809D1FFE743F627
:10D990004001C4F20201086820F080500860FFE7EF
:10D9A000FFE70498806950B1FFE704988069012877
:10D9B00005D0FFE704988069022801D1FFE708E05D
:10D9C00044F63370C0F6020040F2CF110FF052FE61
:10D9D000FFE704988069002800F04781FFE743F6DD
:10D9E0000800C4F20200006800F00C00082800F0F3
:10D9F000F080FFE704988069022840F0C780FFE7C5
:10DA00000498C06930B1FFE70498C069B0F5800F91
:10DA100001D1FFE708E044F63370C0F602004FF48E
:10DA2000EC710FF027FEFFE70498006A3F2801D849
:10DA3000FFE708E044F63370C0F6020040F2D91167
:10DA40000FF018FEFFE70498406A322807D3FFE77B
:10DA50000498406AB0F5D87F01D8FFE708E044F6A3
:10DA60003370C0F602004FF4ED710FF003FEFFE7D4
:10DA70000498806A02280FD0FFE70498806A04287F
:10DA80000AD0FFE70498806A062805D0FFE70498CB
:10DA9000806A082801D1FFE708E044F63370C0F639
:10DAA000020040F2DB110FF0E5FDFFE70498C06AC9
:10DAB000022806D3FFE70498C06A0F2801D8FFE7C1
:10DAC00008E044F63370C0F602004FF4EE710FF038
:10DAD000D1FDFFE76021C4F2472100200860FDF777
:10DAE00095FC0390FFE743F60000C4F202000068D3
:10DAF00000F000710020B0EB516F0CD0FFE7FDF794
:10DB000085FC0399401A032804D3FFE703208DF80E
:10DB10001700AEE0E7E70499C869D1F820C04B6A66
:10DB20008A6A40EA0C0040EA8310D2034FF6FF7382
:10DB30009A43A2F580321043C96A40EA016043F675
:10DB40000401C4F2020108606021C4F247210120EF
:10DB50000860FDF75BFC0390FFE743F60000C4F2AA
:10DB60000200006800F000710020B0EB516F0CD192
:10DB7000FFE7FDF74BFC0399401A032804D3FFE7A6
:10DB800003208DF8170074E0E7E721E06021C4F27C
:10DB9000472100200860FDF739FC0390FFE743F6BA
:10DBA0000000C4F20200006800F000710020B0EB39
:10DBB000516F0CD0FFE7FDF729FC0399401A0328A9
:10DBC00004D3FFE703208DF8170052E0E7E7FFE7F3
:10DBD0004AE004988069012804D1FFE701208DF80C
:10DBE000170046E043F60400C4F202000068029009
:10DBF00004988069012831D0FFE7029800F4800082
:10DC00000499C969884229D1FFE7029800F03F00D2
:10DC10000499096A884221D1FFE7029847F6C0714A
:10DC200008400499496AB0EB811F17D1FFE70298B9
:10DC300000F440300499896AC9034FF6FF7291439A
:10DC4000A1F58031884209D1FFE7029800F07060A9
:10DC50000499C96AB0EB016F04D0FFE701208DF889
:10DC6000170006E0FFE7FFE7FFE700208DF8170049
:10DC7000FFE79DF8170006B080BD000080B582B0B8
:10DC80000090009820B9FFE701208DF807002EE0F2
:10DC90000098006840F60001C5F20601884201D1F3
:10DCA000FFE707E045F26E10C0F60200A3210FF077
:10DCB000E1FCFFE70098407938B9FFE700990020C0
:10DCC0000871009800F018F8FFE7009902204871E9
:10DCD00000980168086840F004000860009901207D
:10DCE00048710099002088608DF80700FFE79DF8D3
:10DCF000070002B080BD000082B00190019800686A
:10DD000040F60001C5F20601884212D1FFE7FFE7A5
:10DD10000020009043F63400C4F20200016841F094
:10DD200040010160006800F0400000900098FFE7AB
:10DD3000FFE702B07047000080B582B00190019803
:10DD400008F03EFC8DF803009DF8030003281BD06B
:10DD5000FFE7019808F034FC014640F2F060C2F29F
:10DD6000000000EB4110806968B1FFE7019808F0FE
:10DD700027FC014640F2F060C2F2000000EB4110C7
:10DD800080698047FFE7FFE702B080BD80B584B0BF
:10DD90000290029820B9FFE701208DF80F00D2E130
:10DDA0000298006843F20001C4F20101884212D0D7
:10DDB000FFE70298006843F60001C4F200018842C0
:10DDC00009D0FFE70298006843F60041C4F2000161
:10DDD000884201D1FFE708E045F2A610C0F6020034
:10DDE0004FF4A1710FF046FCFFE70298406830B194
:10DDF000FFE702984068B0F5827F01D1FFE708E0B5
:10DE000045F2A610C0F6020040F243110FF032FCBA
:10DE1000FFE70298806860B1FFE702988068B0F57C
:10DE2000806F06D0FFE702988068B0F5004F01D1FF
:10DE3000FFE708E045F2A610C0F602004FF4A27119
:10DE40000FF018FCFFE70298C068B0F5006F04D02F
:10DE5000FFE70298C06808B9FFE708E045F2A6109E
:10DE6000C0F6020040F245110FF004FCFFE70298F3
:10DE70008069B0F5007F0AD0FFE70298806930B171
:10DE8000FFE702988069B0F5802F01D1FFE708E035
:10DE900045F2A610C0F602004FF4A3710FF0EAFBA2
:10DEA000FFE70298C06918B3FFE70298C069082825
:10DEB0001ED0FFE70298C069102819D0FFE702982A
:10DEC000C069182814D0FFE70298C06920280FD035
:10DED000FFE70298C06928280AD0FFE70298C069C6
:10DEE000302805D0FFE70298C069382801D1FFE744
:10DEF00008E045F2A610C0F6020040F247110FF00C
:10DF0000B9FBFFE70298006A28B1FFE70298006AB0
:10DF1000802801D1FFE708E045F2A610C0F6020014
:10DF20004FF4A4710FF0A6FBFFE70298406A28B1F6
:10DF3000FFE70298406A102801D1FFE708E045F2A8
:10DF4000A610C0F6020040F249110FF093FBFFE764
:10DF50000298406A002863D1FFE70298006928B15F
:10DF6000FFE702980069022801D1FFE708E045F2C7
:10DF7000A610C0F602004FF4A6710FF07BFBFFE77E
:10DF80000298406928B1FFE702984069012801D151
:10DF9000FFE708E045F2A610C0F6020040F24D117E
:10DFA0000FF068FBFFE702984068B0F5827F32D13E
:10DFB000FFE70298C06918B3FFE70298C069082814
:10DFC0001ED0FFE70298C069102819D0FFE7029819
:10DFD000C069182814D0FFE70298C06920280FD024
:10DFE000FFE70298C06928280AD0FFE70298C069B5
:10DFF000302805D0FFE70298C069382801D1FFE733
:10E0000008E045F2A610C0F6020040F251110FF0F0
:10E0100031FBFFE703E002990020C861FFE736E02B
:10E020000298C06918B3FFE70298C06908281ED09B
:10E03000FFE70298C069102819D0FFE70298C0696D
:10E04000182814D0FFE70298C06920280FD0FFE7F6
:10E050000298C06928280AD0FFE70298C0693028D2
:10E0600005D0FFE70298C069382801D1FFE708E032
:10E0700045F2A610C0F6020040F25B110FF0FAFA6A
:10E08000FFE702990020086102994861FFE70299C1
:10E0900000208862029890F8510040B9FFE7029989
:10E0A000002081F85000029800F052F8FFE7029932
:10E0B000022081F8510002980168086820F04000B1
:10E0C0000860029A019211685068D2F808C0D368BB
:10E0D00000F482700CF4044C604403F400631844B0
:10E0E000136903F002031844536903F00103184451
:10E0F000936903F400731844D36903F03803184498
:10E10000136A03F080031843926A02F4005210432A
:10E110000860029A508B00F004001168526A02F005
:10E1200010021044486002980168C86920F4006039
:10E13000C861029900204865029A012182F85110B5
:10E140008DF80F00FFE79DF80F0004B080BD0000C0
:10E1500080B592B01190002010900F900E900D900D
:10E160000C901198006843F20001C4F2010188424A
:10E1700040F0B680FFE7FFE700200B9043F6440035
:10E18000C4F20200016841F480510160006800F4AB
:10E1900080500B900B98FFE7FFE700200A9043F6B2
:10E1A0003000C4F20200016841F002010160006821
:10E1B00000F002000A900A98FFE7FFE700200990AC
:10E1C00043F63000C4F20200016841F00101016031
:10E1D000006800F0010009900998FFE718200C90F2
:10E1E000022001900D90012002900E9003200390D8
:10E1F0000F9005200490109040F20040C4F20200FD
:10E200000CA90591FCF70CFDDDF804C0029B039AF4
:10E21000049805994FF0800ECDF830E0CDF834C069
:10E220000E930F9210900020C4F20200FCF7F8FC4D
:10E2300041F61830C2F20000069046F24041C4F2A6
:10E24000020101604FF0C061416000218160C16046
:10E250004FF48062026141618161C1614FF44032DB
:10E2600002624162FBF7F2FF18B1FFE7F8F74CFDDD
:10E27000FFE7FFE7119841F61831C2F20001C164CF
:10E2800011988863FFE741F67830C2F200000090F1
:10E2900046F25841C4F2020101604FF0C061416092
:10E2A000402181600021C1604FF4806202614161C0
:10E2B0008161C1614FF4003202624162FBF7C6FF27
:10E2C00018B1FFE7F8F720FDFFE7FFE7119841F6E7
:10E2D0007831C2F20001816411988863FFE73EE063
:10E2E0001198006843F60001C4F20001884235D15C
:10E2F000FFE7FFE70020089043F64000C4F2020069
:10E30000016841F480410160006800F48040089099
:10E310000898FFE7FFE70020079043F63000C4F2BB
:10E320000200016841F002010160006800F0020093
:10E3300007900798FFE74FF460400C9002200D9083
:10E3400001200E9003200F900520109040F2004015
:10E35000C4F202000CA9FCF763FCFFE7FFE712B070
:10E3600080BD000080B588B006900591ADF8122000
:10E37000039300208DF8070006984068B0F5827F6F
:10E3800016D1FFE70698806890B9FFE70699042048
:10E3900081F851000698059ABDF812300399EC46B1
:10E3A000CCF80010114600F089FB8DF81F00EDE05D
:10E3B000FFE7069890F85000012804D1FFE70220FB
:10E3C0008DF81F00E2E00699012081F85000FFE778
:10E3D000FFE7FDF71BF80290069890F8510001281E
:10E3E00004D0FFE702208DF80700C0E0059820B1B7
:10E3F000FFE7BDF8120020B9FFE701208DF8070004
:10E40000B5E00699042081F851000699002048657E
:10E410000599069A9163BDF81210069A9187BDF886
:10E420001210069AD187069908630699888606997C
:10E43000C886069908640699486406988068B0F50D
:10E44000004F0DD1FFE706980168086820F04000F2
:10E45000086006980168086820F480400860FFE7BB
:10E4600006980068006800F04000402807D0FFE7E9
:10E4700006980168086840F040000860FFE70698C9
:10E48000C06880BBFFE7FFE70698C08F50B3FFE787
:10E49000069800688068C00778B1FFE706980068B2
:10E4A000007B0699896B08700699886B0130886338
:10E4B0000699C88F0138C88713E0FCF7A7FF0299B7
:10E4C000401A0399884204D3FFE70398013018B932
:10E4D000FFE7039820B9FFE703208DF8070046E027
:10E4E000FFE7D1E72FE0FFE70698C08F50B3FFE7C3
:10E4F000069800688068C00778B1FFE70698006852
:10E50000C0680699896B08800699886B0230886319
:10E510000699C88F0138C88713E0FCF777FF029986
:10E52000401A0399884204D3FFE70398013018B9D1
:10E53000FFE7039820B9FFE703208DF8070016E0F6
:10E54000FFE7D1E7FFE706980399029A07F074FF07
:10E5500020B1FFE7069920204865FFE70698406D47
:10E5600020B1FFE701208DF80700FFE7FFE70699DC
:10E57000012081F85100FFE70699002081F8500042
:10E58000FFE79DF807008DF81F00FFE79DF81F00CB
:10E5900008B080BD80B584B002900191ADF8022032
:10E5A00000208DF801000298C06C08B1FFE708E078
:10E5B00045F2A610C0F6020040F2CA610FF05AF808
:10E5C000FFE70298806810BBFFE702984068B0F54B
:10E5D000827F1CD1FFE70299042081F85100029844
:10E5E000806C08B1FFE708E045F2A610C0F6020013
:10E5F00040F2D1610FF03EF8FFE70298019ABDF8B2
:10E600000230114600F01CFC8DF80F00A8E0FFE777
:10E61000029890F85000012804D1FFE702208DF8FD
:10E620000F009DE00299012081F85000FFE7FFE70D
:10E63000029890F85100012804D0FFE702208DF8DD
:10E64000010082E0019820B1FFE7BDF8020020B987
:10E65000FFE701208DF8010077E00299042081F89E
:10E6600051000299002048650199029A9163BDF812
:10E670000210029A9187BDF80210029AD18702997E
:10E68000086402994864029988860299C8860298AB
:10E690008068B0F5004F0DD1FFE702980168086867
:10E6A00020F04000086002980168086820F480406B
:10E6B0000860FFE70298C16C46F2DD20C0F6010059
:10E6C00008640298C16C46F20D30C0F60100C863C0
:10E6D0000298C16C46F2A920C0F60100C8640298F5
:10E6E000C16C00200865029B19689A6BD86C0C31CC
:10E6F000DB8FFCF747F860B1FFE70299486D40F007
:10E700001000486501208DF80100029981F8510040
:10E710001BE002980068006800F04000402807D025
:10E72000FFE702980168086840F040000860FFE7D2
:10E7300002980168486840F020004860029801682B
:10E74000486840F001004860FFE7FFE702990020B9
:10E7500081F85000FFE79DF801008DF80F00FFE7FA
:10E760009DF80F0004B080BD80B582B00190019883
:10E7700007F026FF8DF803009DF8030003281BD047
:10E78000FFE7019807F01CFF014640F2F060C2F27B
:10E79000000000EB4110406868B1FFE7019807F006
:10E7A0000FFF014640F2F060C2F2000000EB4110A2
:10E7B00040688047FFE7FFE702B080BD80B582B0C8
:10E7C0000190019807F0FCFE8DF803009DF803000E
:10E7D00003281BD0FFE7019807F0F2FE014640F244
:10E7E000F060C2F2000000EB4110006968B1FFE781
:10E7F000019807F0E5FE014640F2F060C2F2000029
:10E8000000EB411000698047FFE7FFE702B080BDE1
:10E8100080B588B006900591ADF8122003930020D2
:10E820008DF807000698806830B1FFE70698806889
:10E83000B0F5004F01D1FFE708E045F2A610C0F6A1
:10E84000020040F20A310EF015FFFFE7FFE70698DD
:10E8500090F85000012804D1FFE702208DF81F0036
:10E8600028E10699012081F85000FFE7FFE7FCF757
:10E87000CDFD0290BDF81200ADF80400069890F8A6
:10E880005100012804D0FFE702208DF8070002E1C3
:10E89000059820B1FFE7BDF8120020B9FFE701207D
:10E8A0008DF80700F7E00699032081F851000699DA
:10E8B000002048650599069A1163BDF81210069A62
:10E8C0009186BDF81210069AD1860699886306993A
:10E8D00088870699C8870699486406990864069847
:10E8E0008068B0F5004F0DD1FFE706980168086811
:10E8F00020F04000086006980168086840F48040F5
:10E900000860FFE706980068006800F040004028B3
:10E9100007D0FFE706980168086840F040000860EB
:10E92000FFE70698C068B0F5006F47D1FFE706988B
:10E93000406828B1FFE7BDF8040001280ED1FFE7C9
:10E9400006980168006B0088C8600699086B023061
:10E9500008630699C88E0138C886FFE7FFE7069866
:10E96000C08E50B3FFE706980068806880070028D3
:10E970000ED5FFE706980168006B0088C86006990D
:10E98000086B023008630699C88E0138C88613E008
:10E99000FCF73CFD0299401A0399884204D3FFE733
:10E9A0000398013018B9FFE7039820B9FFE7032067
:10E9B0008DF807006FE0FFE7D1E746E00698406872
:10E9C00028B1FFE7BDF8040001280ED1FFE7069843
:10E9D0000168006B007808730699086B01300863C2
:10E9E0000699C88E0138C886FFE7FFE70698C08EF3
:10E9F00050B3FFE7069800688068800700280ED5AE
:10EA0000FFE706980168006B007808730699086BA9
:10EA1000013008630699C88E0138C88613E0FCF7F8
:10EA2000F5FC0299401A0399884204D3FFE7039842
:10EA3000013018B9FFE7039820B9FFE703208DF8EC
:10EA4000070028E0FFE7D1E7FFE706980399029A5D
:10EA500007F064FD20B1FFE7069920204865FFE735
:10EA60000698806870B9FFE7FFE7002000900698DD
:10EA70000068C06800900698006880680090009860
:10EA8000FFE7FFE70698406D20B1FFE701208DF812
:10EA90000700FFE7FFE70699012081F85100FFE733
:10EAA0000699002081F85000FFE79DF807008DF8D7
:10EAB0001F00FFE79DF81F0008B080BD80B58EB035
:10EAC000DDF840C00C900B910A92ADF82630012081
:10EAD000059000208DF813000C98806808B9FFE7B6
:10EAE00008E045F2A610C0F6020040F27E410EF0AA
:10EAF000C1FDFFE7FFE70C9890F85000012804D112
:10EB0000FFE702208DF8370095E10C99012081F88C
:10EB10005000FFE7FFE7FCF779FC06900C9890F8AF
:10EB200051008DF81F000C9840680890BDF8260031
:10EB3000ADF824009DF81F00012812D0FFE70898C7
:10EB4000B0F5827F09D1FFE70C98806828B9FFE70C
:10EB50009DF81F00042804D0FFE702208DF8130061
:10EB60005AE10B9838B1FFE70A9820B1FFE7BDF8EA
:10EB7000260020B9FFE701208DF813004CE10C9826
:10EB800090F85100042805D0FFE70C99052081F882
:10EB90005100FFE70C99002048650A990C9A91638F
:10EBA000BDF826100C9AD187BDF826100C9A9187D3
:10EBB0000B990C9A1163BDF826100C9AD186BDF8FA
:10EBC00026100C9A91860C9908640C9948640C984C
:10EBD0000068006800F04000402807D0FFE70C986C
:10EBE0000168086840F040000860FFE70C98C068C2
:10EBF000B0F5006F76D1FFE70C98406828B1FFE7C9
:10EC0000BDF8240001280ED1FFE70C980168006BC5
:10EC10000088C8600C99086B023008630C99C88E94
:10EC20000138C886FFE7FFE70C98C18E01200290EB
:10EC300039B9FFE70C98C08F002818BF0120029057
:10EC4000FFE70298C00700284BD0FFE70C98006848
:10EC500080688007002818D5FFE70C98C08EA0B107
:10EC6000FFE70598012810D1FFE70C980168006BB9
:10EC70000088C8600C99086B023008630C99C88E34
:10EC80000138C88600200590FFE70C98006880686E
:10EC9000C007A8B1FFE70C98C08F88B1FFE70C98B8
:10ECA0000068C0680C99896B08800C99886B0230E9
:10ECB00088630C99C88F0138C88701200590FFE749
:10ECC000FCF7A4FB0699401A1099884208D3FFE785
:10ECD0001098013020B1FFE703208DF813009BE06E
:10ECE000A2E778E00C98406828B1FFE7BDF824005F
:10ECF00001280ED1FFE70C980168006B00780873BB
:10ED00000C99086B013008630C99C88E0138C886CD
:10ED1000FFE7FFE70C98C18E0120019039B9FFE7AA
:10ED20000C98C08F002818BF01200190FFE70198C0
:10ED3000C00700284ED0FFE70C9800688068800765
:10ED4000002818D5FFE70C98C08EA0B1FFE7059802
:10ED5000012810D1FFE70C980168006B0078087358
:10ED60000C99086B013008630C99C88E0138C8866D
:10ED700000200590FFE70C9800688068C007A8B1E4
:10ED8000FFE70C98C08F88B1FFE70C980068C06857
:10ED90000C99896B08700C99886B013088630C9909
:10EDA000C88F0138C88701200590FFE7FCF72EFBCC
:10EDB0000699401A1099884204D3FFE71098013051
:10EDC00018B9FFE7109820B9FFE703208DF813006A
:10EDD00022E09FE7FFE70C981099069A07F09EFB48
:10EDE00038B1FFE701208DF813000C992020486509
:10EDF00012E00C98806870B9FFE7FFE700200390ED
:10EE00000C980068C06803900C98006880680390B4
:10EE10000398FFE7FFE7FFE70C99012081F8510015
:10EE2000FFE70C99002081F85000FFE79DF81300E0
:10EE30008DF83700FFE79DF837000EB080BD000069
:10EE400080B588B0069005910492ADF80E30002090
:10EE50008DF806000698C06C08B1FFE708E045F29F
:10EE6000A610C0F602004FF4E8610EF003FCFFE7C5
:10EE70000698806C08B1FFE708E045F2A610C0F6DE
:10EE8000020040F241710EF0F5FBFFE70698806842
:10EE900008B9FFE708E045F2A610C0F6020040F20C
:10EEA00044710EF0E7FBFFE7FFE7069890F850008B
:10EEB000012804D1FFE702208DF81F00EFE006993A
:10EEC000012081F85000FFE7FFE7069890F8510015
:10EED0008DF807000698406802909DF80700012809
:10EEE00012D0FFE70298B0F5827F09D1FFE70698BC
:10EEF000806828B9FFE79DF80700042804D0FFE7E1
:10EF000002208DF80600BFE0059838B1FFE70498AD
:10EF100020B1FFE7BDF80E0020B9FFE701208DF812
:10EF20000600B1E0069890F85100042805D0FFE7EC
:10EF30000699052081F85100FFE7069900204865F1
:10EF40000599069A1163BDF80E10069A9186BDF8D0
:10EF50000E10069AD1860499069A9163BDF80E1098
:10EF6000069A9187BDF80E10069AD1870699086413
:10EF700006994864069890F8510004280FD1FFE7DD
:10EF80000698C16C46F2DD20C0F6010008640698C0
:10EF9000C16C46F20D30C0F60100C8630EE0069861
:10EFA000C16C46F2F520C0F6010008640698C16CF9
:10EFB00046F2B130C0F60100C863FFE70698C16CA5
:10EFC00046F2A920C0F60100C8640698C16C002072
:10EFD0000865069B19689A6BD86C0C31DB8FFBF7C0
:10EFE000D1FB60B1FFE70699486D40F0100048651D
:10EFF00001208DF80600069981F8510044E006983A
:10F000000168486840F0010048600698816C002063
:10F0100008640699896CC8630699896CC864069966
:10F02000896C0865069B1A68196B986C0C32DB8E2C
:10F03000FBF7A8FB60B1FFE70699486D40F01000B0
:10F04000486501208DF80600069981F851001BE003
:10F0500006980068006800F04000402807D0FFE7ED
:10F0600006980168086840F040000860FFE70698CD
:10F070000168486840F020004860069801684868C8
:10F0800040F002004860FFE7FFE70699002081F8A2
:10F090005000FFE79DF806008DF81F00FFE79DF880
:10F0A0001F0008B080BD000080B582B001900198BB
:10F0B00007F086FA8DF803009DF8030003281BD0A3
:10F0C000FFE7019807F07CFA014640F2F060C2F2D7
:10F0D000000000EB4110806868B1FFE7019807F07D
:10F0E0006FFA014640F2F060C2F2000000EB4110FE
:10F0F00080688047FFE7FFE702B080BD80B582B03F
:10F100000190019807F05CFA8DF803009DF8030068
:10F1100003281BD0FFE7019807F052FA014640F29E
:10F12000F060C2F2000000EB4110406968B1FFE7F7
:10F13000019807F045FA014640F2F060C2F2000083
:10F1400000EB411040698047FFE7FFE702B080BD58
:10F1500080B582B00190019807F0E0FF02B080BD59
:10F1600081B0009001B0704781B0009001B070474D
:10F1700080B584B002900191002000900298006850
:10F180000021C4F20101884209D0FFE7029800681B
:10F1900040F20041C4F20101884201D1FFE708E0DA
:10F1A00045F21620C0F6020040F2B4710EF062FA89
:10F1B000FFE701980068B0F5006F04D0FFE7019801
:10F1C000006808B9FFE708E045F21620C0F6020023
:10F1D00040F2B5710EF04EFAFFE701984068B0F5C5
:10F1E000806F04D0FFE70198406808B9FFE708E0A6
:10F1F00045F21620C0F6020040F2B6710EF03AFA5F
:10F20000FFE70198806890B1FFE701988068B0F54A
:10F21000807F0CD0FFE701988068B0F5007F06D0B2
:10F22000FFE701988068B0F5407F01D1FFE708E073
:10F2300045F21620C0F6020040F2B7710EF01AFA3D
:10F24000FFE70198C068FF2801D8FFE708E045F212
:10F250001620C0F602004FF4F7610EF00BFAFFE73C
:10F2600001980069B0F5805F04D0FFE7019800695C
:10F2700008B9FFE708E045F21620C0F6020040F2A8
:10F28000B9710EF0F7F9FFE70198406930B1FFE777
:10F2900001984069B0F5005F01D1FFE708E045F251
:10F2A0001620C0F6020040F2BA710EF0E3F9FFE753
:10F2B0000198C069B0F5804F04D0FFE70198C0699C
:10F2C00008B9FFE708E045F21620C0F6020040F258
:10F2D000BB710EF0CFF9FFE7FFE7029890F83C0012
:10F2E000012804D1FFE702208DF80F0044E00299C5
:10F2F000012081F83C00FFE7FFE7009820F0FF00C5
:10F300000199C96808430090009820F44070019961
:10F31000896808430090009820F48060019949684A
:10F3200008430090009820F40060019909680843A0
:10F330000090009820F480500199096908430090DA
:10F34000009820F400500199496908430090009802
:10F3500020F480400199C9690843009000980299FF
:10F3600009684864FFE70299002081F83C00FFE744
:10F3700000208DF80F00FFE79DF80F0004B080BD5E
:10F3800080B586B004900391049800680021C4F20F
:10F39000010188423CD0FFE704980068B0F1804F3B
:10F3A00036D0FFE70498006840F20041C4F2000143
:10F3B00088422DD0FFE70498006840F60001C4F2AF
:10F3C0000001884224D0FFE70498006840F600411D
:10F3D000C4F2000188421BD0FFE70498006841F2A4
:10F3E0000001C4F20001884212D0FFE704980068CF
:10F3F00041F20041C4F20001884209D0FFE70498BD
:10F40000006840F20041C4F20101884201D1FFE7E7
:10F4100008E045F21620C0F6020040F277710EF0C7
:10F4200029F9FFE70398006818B3FFE7039800681D
:10F4300010281ED0FFE703980068202819D0FFE7A6
:10F4400003980068302814D0FFE70398006840282C
:10F450000FD0FFE70398006850280AD0FFE7039811
:10F460000068602805D0FFE703980068702801D184
:10F47000FFE708E045F21620C0F602004FF4EF6106
:10F480000EF0F8F8FFE703984068802804D0FFE703
:10F490000398406808B9FFE708E045F21620C0F677
:10F4A000020040F279710EF0E5F8FFE7FFE70498FB
:10F4B00090F83C00012804D1FFE702208DF81700E6
:10F4C0007EE00499012081F83C00FFE7FFE7049902
:10F4D000022081F83D00049800684068029004987A
:10F4E000006880680190029820F0700002900398F4
:10F4F00001680298084302900298049909684860DC
:10F50000049800680021C4F2010188423CD0FFE762
:10F5100004980068B0F1804F36D0FFE70498006887
:10F5200040F20041C4F2000188422DD0FFE7049868
:10F53000006840F60001C4F20001884224D0FFE7D1
:10F540000498006840F60041C4F2000188421BD0D4
:10F55000FFE70498006840F20041C4F201018842CC
:10F5600012D0FFE70498006844F20001C4F20101E0
:10F57000884209D0FFE70498006841F60001C4F210
:10F58000000188420ED1FFE7019820F08000019031
:10F59000039841680198084301900198049909680B
:10F5A0008860FFE70499012081F83D00FFE7049996
:10F5B000002081F83C00FFE700208DF81700FFE7EE
:10F5C0009DF8170006B080BD80B582B0009000980D
:10F5D00020B9FFE701208DF8070012E100980068CC
:10F5E0000021C4F20101884272D0FFE70098006850
:10F5F000B0F1804F6CD0FFE70098006840F2004106
:10F60000C4F20001884263D0FFE70098006840F62A
:10F610000001C4F2000188425AD0FFE70098006858
:10F6200040F60041C4F20001884251D0FFE7009843
:10F63000006841F20001C4F20001884248D0FFE7AF
:10F640000098006841F20041C4F2000188423FD0B6
:10F65000FFE70098006840F20041C4F201018842CF
:10F6600036D0FFE70098006844F20001C4F20101BF
:10F6700088422DD0FFE70098006844F20041C4F2B0
:10F680000101884224D0FFE70098006844F6000199
:10F69000C4F2010188421BD0FFE70098006841F6E0
:10F6A0000001C4F20001884212D0FFE70098006810
:10F6B00041F60041C4F20001884209D0FFE70098FA
:10F6C000006842F20001C4F20001884201D1FFE764
:10F6D00008E045F2DE10C0F6020040F213110DF012
:10F6E000C9FFFFE700988068A0B1FFE70098806835
:10F6F00010280FD0FFE70098806820280AD0FFE785
:10F7000000988068402805D0FFE70098806860284E
:10F7100001D1FFE708E045F2DE10C0F602004FF429
:10F720008A710DF0A7FFFFE70098006960B1FFE75D
:10F7300000980069B0F5807F06D0FFE70098006967
:10F74000B0F5007F01D1FFE708E045F2DE10C0F61A
:10F75000020040F215110DF08DFFFFE7009880695F
:10F7600028B1FFE700988069802801D1FFE708E011
:10F7700045F2DE10C0F602004FF48B710DF07AFFF7
:10F78000FFE7009890F83D0040B9FFE7009900209E
:10F7900081F83C00009800F039F8FFE7009902205A
:10F7A00081F83D00009951F8040B07F06BFD0099BA
:10F7B000012081F84600FFE70099012081F83E0012
:10F7C000009981F83F00009981F84000009981F884
:10F7D0004100FFE7FFE70099012081F8420000990E
:10F7E00081F84300009981F84400009981F84500B0
:10F7F000FFE70099012081F83D0000208DF8070007
:10F80000FFE79DF8070002B080BD000080B58AB018
:10F810000990099800680021C4F2010188421BD1B7
:10F82000FFE7FFE70020089043F64400C4F202001F
:10F83000016841F001010160006800F001000890DA
:10F840000898FFE71820019005210022FCF7FAF93B
:10F850000198FCF7DFF9B0E00998006840F2004138
:10F86000C4F20001884212D1FFE7FFE700200790B1
:10F8700043F64000C4F20200016841F00201016059
:10F88000006800F0020007900798FFE794E00998ED
:10F89000006840F60001C4F20001884212D1FFE77F
:10F8A000FFE70020069043F64000C4F20200016822
:10F8B00041F004010160006800F004000690069821
:10F8C000FFE778E00998006840F60041C4F20001C3
:10F8D000884212D1FFE7FFE70020059043F6400081
:10F8E000C4F20200016841F008010160006800F004
:10F8F000080005900598FFE75CE00998006841F270
:10F900000041C4F2000188421BD1FFE7FFE700205D
:10F91000049043F64000C4F20200016841F0200167
:10F920000160006800F0200004900498FFE7372091
:10F93000009005210022FCF785F90098FCF76AF990
:10F9400037E00998006840F20041C4F201018842A2
:10F9500012D1FFE7FFE70020039043F64400C4F212
:10F960000200016841F002010160006800F002003D
:10F9700003900398FFE71BE00998006844F20041F8
:10F98000C4F20101884212D1FFE7FFE70020029094
:10F9900043F64400C4F20200016841F40031016002
:10F9A000006800F4003002900298FFE7FFE7FFE7ED
:10F9B000FFE7FFE7FFE7FFE7FFE70AB080BD0000D2
:10F9C00080B584B00290029800680021C4F2010161
:10F9D000884272D0FFE702980068B0F1804F6CD087
:10F9E000FFE70298006840F20041C4F2000188423B
:10F9F00063D0FFE70298006840F60001C4F20001FE
:10FA000088425AD0FFE70298006840F60041C4F2ED
:10FA10000001884251D0FFE70298006841F20001DE
:10FA2000C4F20001884248D0FFE70298006841F222
:10FA30000041C4F2000188423FD0FFE7029800680D
:10FA400040F20041C4F20101884236D0FFE702983B
:10FA5000006844F20001C4F2010188422DD0FFE7A2
:10FA60000298006844F20041C4F20101884224D0A7
:10FA7000FFE70298006844F60001C4F201018842E1
:10FA80001BD0FFE70298006841F60001C4F20001B4
:10FA9000884212D0FFE70298006841F60041C4F2A4
:10FAA0000001884209D0FFE70298006842F2000195
:10FAB000C4F20001884201D1FFE708E045F2DE1000
:10FAC000C0F6020040F2CF110DF0D4FDFFE702981E
:10FAD00090F83D00012804D0FFE701208DF80F00C9
:10FAE0006AE00299022081F83D0002980168C86826
:10FAF00040F00100C860029800680021C4F20101D2
:10FB000088423CD0FFE702980068B0F1804F36D0C1
:10FB1000FFE70298006840F20041C4F20001884209
:10FB20002DD0FFE70298006840F60001C4F2000102
:10FB3000884224D0FFE70298006840F60041C4F2F2
:10FB4000000188421BD0FFE70298006840F20041A4
:10FB5000C4F20101884212D0FFE70298006844F223
:10FB60000001C4F20101884209D0FFE70298006851
:10FB700041F60001C4F20001884212D1FFE7029869
:10FB80000068806800F0070001900198062807D0FF
:10FB9000FFE702980168086840F001000860FFE78D
:10FBA00006E002980168086840F001000860FFE77D
:10FBB00000208DF80F00FFE79DF80F0004B080BD16
:10FBC00080B586B004900391FFE7049890F83C005C
:10FBD000012805D1FFE702208DF8170000F069BC6D
:10FBE0000499012081F83C00FFE7FFE70499022017
:10FBF00081F83D0003980068B0F5805F2DD0FFE7E5
:10FC000003980068B0F5005F27D0FFE7039800680D
:10FC100018B3FFE70398006810281ED0FFE7039889
:10FC20000068202819D0FFE703980068302814D016
:10FC3000FFE70398006840280FD0FFE703980068AB
:10FC400050280AD0FFE703980068602805D0FFE736
:10FC500003980068702801D1FFE708E045F2DE1044
:10FC6000C0F6020041F222410DF004FDFFE70498C6
:10FC7000006880680290029820F077000290029855
:10FC800020F47F40029002980499096888600398E4
:10FC900000680190002800F0A883FFE70198102871
:10FCA00000F0A383FFE70198202800F09E83FFE780
:10FCB0000198302800F09983FFE70198402800F070
:10FCC0000883FFE70198502800F0EB81FFE70198D7
:10FCD000602800F07282FFE70198702800F09180A0
:10FCE000FFE70198B0F5805F06D0FFE70198B0F517
:10FCF000005F00F03A81CDE3049800680021C4F26F
:10FD00000101884272D0FFE704980068B0F1804F8B
:10FD10006CD0FFE70498006840F20041C4F2000193
:10FD2000884263D0FFE70498006840F60001C4F2FF
:10FD3000000188425AD0FFE70498006840F600416D
:10FD4000C4F20001884251D0FFE70498006841F2F4
:10FD50000001C4F20001884248D0FFE7049800681F
:10FD600041F20041C4F2000188423FD0FFE704980D
:10FD7000006840F20041C4F20101884236D0FFE73A
:10FD80000498006844F20001C4F2010188422DD0B9
:10FD9000FFE70498006844F20041C4F20101884280
:10FDA00024D0FFE70498006844F60001C4F2010182
:10FDB00088421BD0FFE70498006841F60001C4F2B6
:10FDC0000001884212D0FFE70498006841F6004124
:10FDD000C4F20001884209D0FFE70498006842F2AB
:10FDE0000001C4F20001884201D1FFE708E045F2BA
:10FDF000DE10C0F6020041F22E410DF03BFCFFE7A1
:10FE000049E3049800680021C4F2010188423CD013
:10FE1000FFE704980068B0F1804F36D0FFE7049800
:10FE2000006840F20041C4F2000188422DD0FFE793
:10FE30000498006840F60001C4F20001884224D012
:10FE4000FFE70498006840F60041C4F200018842D0
:10FE50001BD0FFE70498006840F20041C4F20101A2
:10FE6000884212D0FFE70498006844F20001C4F20F
:10FE70000101884209D0FFE70498006841F60001BB
:10FE8000C4F20001884201D1FFE708E045F2DE102C
:10FE9000C0F6020041F235410DF0ECFBFFE703989C
:10FEA000806890B1FFE703988068B0F5805F0CD060
:10FEB000FFE703988068B0F5005F06D0FFE703987E
:10FEC0008068B0F5405F01D1FFE708E045F2DE1041
:10FED000C0F6020041F238410DF0CCFBFFE7039879
:10FEE0004068B0F5004F12D0FFE70398406870B14A
:10FEF000FFE70398406850B1FFE703984068022885
:10FF000005D0FFE7039840680A2801D1FFE708E021
:10FF100045F2DE10C0F6020041F239410DF0AAFBB5
:10FF2000FFE70398C0680F2801D8FFE708E045F213
:10FF3000DE10C0F6020041F23A410DF09BFBFFE7F4
:10FF400004980068039B5A689968DB6807F008FB0F
:10FF50000498006880680290029840F07700029050
:10FF6000029804990968886095E204980068002165
:10FF7000C4F2010188422AD0FFE704980068B0F17A
:10FF8000804F24D0FFE70498006840F20041C4F29B
:10FF9000000188421BD0FFE70498006840F600018A
:10FFA000C4F20001884212D0FFE70498006840F6CE
:10FFB0000041C4F20001884209D0FFE704980068BC
:10FFC00040F20041C4F20101884201D1FFE708E09C
:10FFD00045F2DE10C0F6020041F24D410DF04AFB41
:10FFE000FFE70398806890B1FFE703988068B0F559
:10FFF000805F0CD0FFE703988068B0F5005F06D003
:020000040801F1
:10000000FFE703988068B0F5405F01D1FFE708E0A3
:1000100045F2DE10C0F6020041F250410DF02AFB1D
:10002000FFE703984068B0F5004F12D0FFE7039850
:10003000406870B1FFE70398406850B1FFE703984C
:100040004068022805D0FFE7039840680A2801D1DC
:10005000FFE708E045F2DE10C0F6020041F2514130
:100060000DF008FBFFE70398C0680F2801D8FFE7F1
:1000700008E045F2DE10C0F6020041F252410DF0F8
:10008000F9FAFFE704980068039B5A689968DB68EF
:1000900007F066FA04980168886840F48040886038
:1000A000F9E1049800680021C4F2010188423CD0C3
:1000B000FFE704980068B0F1804F36D0FFE704985E
:1000C000006840F20041C4F2000188422DD0FFE7F1
:1000D0000498006840F60001C4F20001884224D070
:1000E000FFE70498006840F60041C4F2000188422E
:1000F0001BD0FFE70498006840F20041C4F2010100
:10010000884212D0FFE70498006844F20001C4F26C
:100110000101884209D0FFE70498006841F6000118
:10012000C4F20001884201D1FFE708E045F2DE1089
:10013000C0F6020041F261410DF09CFAFFE703981E
:100140004068B0F5004F12D0FFE70398406870B1E7
:10015000FFE70398406850B1FFE703984068022822
:1001600005D0FFE7039840680A2801D1FFE708E0BF
:1001700045F2DE10C0F6020041F264410DF07AFA59
:10018000FFE70398C0680F2801D8FFE708E045F2B1
:10019000DE10C0F6020041F265410DF06BFAFFE798
:1001A00004980068039A5168D26807F08FFC04989D
:1001B0000068502107F0EEF96DE104980068002115
:1001C000C4F2010188423CD0FFE704980068B0F116
:1001D000804F36D0FFE70498006840F20041C4F237
:1001E000000188422DD0FFE70498006840F6000126
:1001F000C4F20001884224D0FFE70498006840F66A
:100200000041C4F2000188421BD0FFE70498006857
:1002100040F20041C4F20101884212D0FFE7049885
:10022000006844F20001C4F20101884209D0FFE7EE
:100230000498006841F60001C4F20001884201D12F
:10024000FFE708E045F2DE10C0F6020041F271411E
:100250000DF010FAFFE703984068B0F5004F12D098
:10026000FFE70398406870B1FFE70398406850B11A
:10027000FFE703984068022805D0FFE7039840682D
:100280000A2801D1FFE708E045F2DE10C0F60200BF
:1002900041F274410DF0EEF9FFE70398C0680F28B2
:1002A00001D8FFE708E045F2DE10C0F6020041F297
:1002B00075410DF0DFF9FFE704980068039A516873
:1002C000D26807F02BFC04980068602107F062F9FF
:1002D000E1E0049800680021C4F2010188423CD0AA
:1002E000FFE704980068B0F1804F36D0FFE704982C
:1002F000006840F20041C4F2000188422DD0FFE7BF
:100300000498006840F60001C4F20001884224D03D
:10031000FFE70498006840F60041C4F200018842FB
:100320001BD0FFE70498006840F20041C4F20101CD
:10033000884212D0FFE70498006844F20001C4F23A
:100340000101884209D0FFE70498006841F60001E6
:10035000C4F20001884201D1FFE708E045F2DE1057
:10036000C0F6020041F281410DF084F9FFE70398E5
:100370004068B0F5004F12D0FFE70398406870B1B5
:10038000FFE70398406850B1FFE7039840680228F0
:1003900005D0FFE7039840680A2801D1FFE708E08D
:1003A00045F2DE10C0F6020041F284410DF062F920
:1003B000FFE70398C0680F2801D8FFE708E045F27F
:1003C000DE10C0F6020041F285410DF053F9FFE75F
:1003D00004980068039A5168D26807F077FB049884
:1003E0000068402107F0D6F855E004980068002125
:1003F000C4F2010188423CD0FFE704980068B0F1E4
:10040000804F36D0FFE70498006840F20041C4F204
:10041000000188422DD0FFE70498006840F60001F3
:10042000C4F20001884224D0FFE70498006840F637
:100430000041C4F2000188421BD0FFE70498006825
:1004400040F20041C4F20101884212D0FFE7049853
:10045000006844F20001C4F20101884209D0FFE7BC
:100460000498006841F60001C4F20001884201D1FD
:10047000FFE708E045F2DE10C0F6020041F29441C9
:100480000DF0F8F8FFE7049800680399096807F091
:1004900081F800E0FFE70499012081F83D00FFE7C3
:1004A0000499002081F83C00FFE700208DF8170038
:1004B000FFE79DF8170006B080BD000081B00090F6
:1004C00001B0704780B582B0019001980068006962
:1004D00000F002010020B0EB510F28D0FFE7019897
:1004E0000068C06800F002010020B0EB510F1DD081
:1004F000FFE7019801686FF002000861019901208F
:100500000877019800688069800720B1FFE70198AB
:10051000FFF7D4FF06E0019800F04CFA019800F0D4
:10052000A3FDFFE7019900200877FFE7FFE70198A7
:100530000068006900F004010020B0EB910F29D0A1
:10054000FFE701980068C06800F004010020B0EBEC
:10055000910F1ED0FFE7019801686FF00400086159
:1005600001990220087701980068806910F4407FA3
:1005700004D0FFE70198FFF7A1FF06E0019800F023
:1005800019FA019800F070FDFFE701990020087743
:10059000FFE7FFE701980068006900F0080100200C
:1005A000B0EBD10F28D0FFE701980068C06800F0D9
:1005B00008010020B0EBD10F1DD0FFE701980168C2
:1005C0006FF008000861019904200877019800681D
:1005D000C069800720B1FFE70198FFF76FFF06E0D1
:1005E000019800F0E7F9019800F03EFDFFE701995E
:1005F00000200877FFE7FFE701980068006900F036
:1006000010010020B0EB111F29D0FFE7019800680E
:10061000C06800F010010020B0EB111F1ED0FFE7F2
:10062000019801686FF010000861019908200877AF
:1006300001980068C06910F4407F04D0FFE701987A
:10064000FFF73CFF06E0019800F0B4F9019800F0D4
:100650000BFDFFE7019900200877FFE7FFE701980E
:1006600000680069C00780B1FFE701980068C068B2
:10067000C00748B1FFE7019801686FF00100086109
:10068000019801F057F8FFE7FFE70198006800695B
:10069000C1B20020B0EBD11F13D0FFE70198006872
:1006A000C068C1B20020B0EBD11F09D0FFE70198AC
:1006B00001686FF0800008610198FEF751FDFFE7C7
:1006C000FFE701980068006900F040010020B0EBEE
:1006D000911F14D0FFE701980068C06800F0400146
:1006E0000020B0EB911F09D0FFE7019801686FF07F
:1006F00040000861019801F033F8FFE7FFE7019837
:100700000068006900F020010020B0EB511F14D0F8
:10071000FFE701980068C06800F020010020B0EBFE
:10072000511F09D0FFE7019801686FF020000861B0
:100730000198FEF719FDFFE7FFE702B080BD00005A
:1007400080B592B01190002010900F900E900D90F7
:100750000C90119800680021C4F20101884222D156
:10076000FFE7FFE700200B9043F63000C4F20200E1
:10077000016841F010010160006800F010000B906A
:100780000B98FFE74FF4D4400C9002210D9101200B
:100790000E900F91109041F20000C4F202000CA9DB
:1007A000FAF73EFA03E11198006840F20041C4F202
:1007B0000001884222D1FFE7FFE700200A9043F6BC
:1007C0003000C4F20200016841F0040101600068D9
:1007D00000F004000A900A98FFE74FF480700C9034
:1007E00002200D9001210E910F90109040F6000014
:1007F000C4F202000CA9FAF713FAD7E011980068C6
:1008000040F60001C4F20001884223D1FFE7FFE770
:100810000020099043F63000C4F20200016841F064
:1008200008010160006800F0080009900998FFE7DE
:100830004FF480400C9002200D9001210E91032175
:100840000F91109040F60040C4F202000CA9FAF794
:10085000E7F9AAE01198006840F60041C4F20001EF
:10086000884222D1FFE7FFE70020089043F63000DE
:10087000C4F20200016841F080010160006800F0EC
:10088000800008900898FFE74FF4E0500C90022099
:100890000D9001210E910F90109041F60040C4F28E
:1008A00002000CA9FAF7BCF97EE01198006840F24A
:1008B0000041C4F2010188424AD1FFE7FFE700206E
:1008C000079043F63000C4F20200016841F48071E1
:1008D0000160006800F4807007900798FFE7FFE769
:1008E0000020069043F63000C4F20200016841F097
:1008F00004010160006800F0040006900698FFE71C
:10090000402000900C90022002900D900121019156
:100910000E910F9003200390109042F20000C4F259
:1009200002000CA90491FAF77BF9DDF800C0019BE5
:10093000029A03980499CDF830C00D920E930F924D
:10094000109040F60000C4F20200FAF769F92AE0BC
:100950001198006844F20041C4F20101884221D19B
:10096000FFE7FFE70020059043F63000C4F20200E5
:10097000016841F020010160006800F0200005904E
:100980000598FFE740200C9002200D900E900F90EC
:100990000320109041F20040C4F202000CA9FAF7C3
:1009A0003FF9FFE7FFE7FFE7FFE7FFE7FFE712B0E9
:1009B00080BD000081B0009001B0704780B586B066
:1009C000049003910292029880B1FFE702980428F4
:1009D0000CD0FFE70298082808D0FFE702980C28FF
:1009E00004D0FFE702983C2801D1FFE708E045F278
:1009F000DE10C0F6020041F217010CF03BFEFFE7EB
:100A000003980068602805D0FFE703980068702805
:100A100001D1FFE708E045F2DE10C0F6020041F226
:100A200018010CF027FEFFE70398806828B1FFE764
:100A300003988068022801D1FFE708E045F2DE1044
:100A4000C0F6020041F219010CF014FEFFE7039812
:100A5000006928B1FFE703980069042801D1FFE786
:100A600008E045F2DE10C0F6020041F21A010CF077
:100A700001FEFFE7FFE7049890F83C00012804D14D
:100A8000FFE702208DF81700C3E10499012081F8E7
:100A90003C00FFE7FFE7029801900C2800F2AE81CE
:100AA0000199DFE811F00D00AB01AB01AB0198003B
:100AB000AB01AB01AB010001AB01AB01AB015501D7
:100AC000049800680021C4F20101884260D0FFE769
:100AD00004980068B0F1804F5AD0FFE7049800688E
:100AE00040F20041C4F20001884251D0FFE704986F
:100AF000006840F60001C4F20001884248D0FFE7D8
:100B00000498006840F60041C4F2000188423FD0DA
:100B1000FFE70498006840F20041C4F201018842F6
:100B200036D0FFE70498006844F20001C4F20101E6
:100B300088422DD0FFE70498006844F20041C4F2D7
:100B40000101884224D0FFE70498006844F60001C0
:100B5000C4F2010188421BD0FFE70498006841F607
:100B60000001C4F20001884212D0FFE70498006837
:100B700041F60041C4F20001884209D0FFE7049821
:100B8000006842F20001C4F20001884201D1FFE78F
:100B900008E045F2DE10C0F6020041F224010CF03C
:100BA00069FDFFE704980068039906F009FD0498C1
:100BB0000168886940F008008861049801688869C4
:100BC00020F004008861039802690498016888692C
:100BD0001043886113E1049800680021C4F2010108
:100BE00088423CD0FFE704980068B0F1804F36D0CF
:100BF000FFE70498006840F20041C4F20001884217
:100C00002DD0FFE70498006840F60001C4F200010F
:100C1000884224D0FFE70498006840F60041C4F2FF
:100C2000000188421BD0FFE70498006840F20041B1
:100C3000C4F20101884212D0FFE70498006844F230
:100C40000001C4F20101884209D0FFE7049800685E
:100C500041F60001C4F20001884201D1FFE708E03B
:100C600045F2DE10C0F6020041F235010CF002FD43
:100C7000FFE704980068039906F054FD04980168A2
:100C8000886940F40060886104980168886920F4EC
:100C9000806088610398026904980168886940EA65
:100CA00002208861ABE0049800680021C4F20101D1
:100CB00088422AD0FFE704980068B0F1804F24D022
:100CC000FFE70498006840F20041C4F20001884246
:100CD0001BD0FFE70498006840F60001C4F2000151
:100CE000884212D0FFE70498006840F60041C4F241
:100CF0000001884209D0FFE70498006840F20041F3
:100D0000C4F20101884201D1FFE708E045F2DE109C
:100D1000C0F6020041F246010CF0ACFCFFE704987B
:100D20000068039906F0B4FD04980168C86940F0B2
:100D30000800C86104980168C86920F00400C8610F
:100D40000398026904980168C8691043C86156E0B5
:100D5000049800680021C4F2010188422AD0FFE70C
:100D600004980068B0F1804F24D0FFE70498006831
:100D700040F20041C4F2000188421BD0FFE7049812
:100D8000006840F60001C4F20001884212D0FFE77B
:100D90000498006840F60041C4F20001884209D07E
:100DA000FFE70498006840F20041C4F20101884264
:100DB00001D1FFE708E045F2DE10C0F6020041F283
:100DC00057010CF057FCFFE704980068039906F000
:100DD00015FE04980168C86940F40060C861049871
:100DE0000168C86920F48060C861039802690498AA
:100DF0000168C86940EA0220C86100E0FFE7FFE738
:100E00000499002081F83C00FFE700208DF81700CE
:100E1000FFE79DF8170006B080BD000080B582B0E6
:100E20000090009820B9FFE701208DF8070012E13B
:100E3000009800680021C4F20101884272D0FFE7E7
:100E400000980068B0F1804F6CD0FFE70098006810
:100E500040F20041C4F20001884263D0FFE70098ED
:100E6000006840F60001C4F2000188425AD0FFE752
:100E70000098006840F60041C4F20001884251D059
:100E8000FFE70098006841F20001C4F200018842C7
:100E900048D0FFE70098006841F20041C4F2000129
:100EA00088423FD0FFE70098006840F20041C4F25A
:100EB0000101884236D0FFE70098006844F2000143
:100EC000C4F2010188422DD0FFE70098006844F287
:100ED0000041C4F20101884224D0FFE70098006875
:100EE00044F60001C4F2010188421BD0FFE70098DC
:100EF000006841F60001C4F20001884212D0FFE709
:100F00000098006841F60041C4F20001884209D00F
:100F1000FFE70098006842F20001C4F20001884235
:100F200001D1FFE708E045F2DE10C0F6020040F212
:100F30000E510CF09FFBFFE700988068A0B1FFE71F
:100F40000098806810280FD0FFE70098806820285C
:100F50000AD0FFE700988068402805D0FFE7009896
:100F60008068602801D1FFE708E045F2DE10C0F696
:100F7000020040F20F510CF07DFBFFE70098006982
:100F800060B1FFE700980069B0F5807F06D0FFE709
:100F900000980069B0F5007F01D1FFE708E045F255
:100FA000DE10C0F602004FF4A2610CF063FBFFE715
:100FB0000098806928B1FFE700988069802801D1F6
:100FC000FFE708E045F2DE10C0F6020040F21151E2
:100FD0000CF050FBFFE7009890F83D0040B9FFE7A8
:100FE0000099002081F83C00009800F039F8FFE7F4
:100FF0000099022081F83D00009951F8040B06F099
:1010000041F90099012081F84600FFE7009901208D
:1010100081F83E00009981F83F00009981F8400076
:10102000009981F84100FFE7FFE70099012081F86E
:101030004200009981F84300009981F8440000992A
:1010400081F84500FFE70099012081F83D0000206C
:101050008DF80700FFE79DF8070002B080BD000093
:1010600081B0009001B0704781B0009001B070472E
:1010700080B58CB00A9009910A9800680021C4F2EA
:101080000101884214D1FFE70998002800F0E780A9
:10109000FFE70998042800F0E280FFE70998082894
:1010A00000F0DD80FFE709980C2800F0D880FFE70A
:1010B0000A980068B0F1804F14D1FFE70998002822
:1010C00000F0CD80FFE70998042800F0C880FFE712
:1010D0000998082800F0C380FFE709980C2800F061
:1010E000BE80FFE70A98006840F20041C4F20001A8
:1010F000884214D1FFE70998002800F0B080FFE78C
:101100000998042800F0AB80FFE70998082800F050
:10111000A680FFE709980C2800F0A180FFE70A9855
:10112000006840F60001C4F20001884214D1FFE7D4
:101130000998002800F09380FFE70998042800F040
:101140008E80FFE70998082800F08980FFE709985A
:101150000C2800F08480FFE70A98006840F6004100
:10116000C4F20001884210D1FFE70998002876D028
:10117000FFE70998042872D0FFE7099808286ED085
:10118000FFE709980C286AD0FFE70A98006840F248
:101190000041C4F20101884210D1FFE709980028FC
:1011A0005DD0FFE70998042859D0FFE7099808287F
:1011B00055D0FFE709980C2851D0FFE70A9800683E
:1011C00044F20001C4F20101884208D1FFE7099806
:1011D000002844D0FFE70998042840D0FFE70A9888
:1011E000006844F20041C4F20101884203D1FFE7E4
:1011F0000998A0B3FFE70A98006844F60001C4F21A
:101200000101884203D1FFE7099840B3FFE70A983C
:10121000006841F60001C4F20001884207D1FFE7EF
:101220000998E0B1FFE70998042818D0FFE70A9869
:10123000006841F60041C4F20001884203D1FFE793
:10124000099860B1FFE70A98006842F20001C4F211
:101250000001884204D1FFE7099808B9FFE708E0D8
:1012600045F2DE10C0F6020040F294510CF002FA92
:10127000FFE7099828B9FFE70A9890F83E00079021
:101280001CE00998042805D1FFE70A9890F83F0070
:10129000069010E00998082805D1FFE70A9890F811
:1012A0004000059004E00A9890F841000590FFE79F
:1012B00005980690FFE706980790FFE70798012832
:1012C00004D0FFE701208DF82F00AFE0099828B97E
:1012D000FFE70A99022081F83E001EE009980428E1
:1012E00006D1FFE70A99022081F83F00049012E03E
:1012F0000998082806D1FFE70A99022081F84000E2
:10130000039005E00A99022081F841000390FFE76D
:1013100003980490FFE70498FFE70A98006809998A
:101320000122019206F07CF801980A9909680022CE
:10133000C4F20102914202900CD0FFE70A980068C3
:101340004FF60041CBF6FE710844B0FA80F0400938
:101350000290FFE70298C00738B1FFE70A980168DA
:10136000486C40F400404864FFE70A980068002198
:10137000C4F2010188423CD0FFE70A980068B0F14E
:10138000804F36D0FFE70A98006840F20041C4F26F
:10139000000188422DD0FFE70A98006840F600015E
:1013A000C4F20001884224D0FFE70A98006840F6A2
:1013B0000041C4F2000188421BD0FFE70A98006890
:1013C00040F20041C4F20101884212D0FFE70A98BE
:1013D000006844F20001C4F20101884209D0FFE72D
:1013E0000A98006841F60001C4F20001884212D157
:1013F000FFE70A980068806800F0070008900898E6
:10140000062807D0FFE70A980168086840F0010045
:101410000860FFE706E00A980168086840F00100EC
:101420000860FFE700208DF82F00FFE79DF82F00F0
:101430000CB080BD80B586B0059004910598006819
:101440000021C4F20101884214D1FFE7049800286A
:1014500000F0E780FFE70498042800F0E280FFE74F
:101460000498082800F0DD80FFE704980C2800F0BD
:10147000D880FFE705980068B0F1804F14D1FFE7EE
:101480000498002800F0CD80FFE70498042800F0BD
:10149000C880FFE70498082800F0C380FFE704989D
:1014A0000C2800F0BE80FFE70598006840F200417C
:1014B000C4F20001884214D1FFE70498002800F02C
:1014C000B080FFE70498042800F0AB80FFE70498A1
:1014D000082800F0A680FFE704980C2800F0A180FF
:1014E000FFE70598006840F60001C4F20001884259
:1014F00014D1FFE70498002800F09380FFE70498D8
:10150000042800F08E80FFE70498082800F0898006
:10151000FFE704980C2800F08480FFE70598006836
:1015200040F60041C4F20001884210D1FFE7049860
:10153000002876D0FFE70498042872D0FFE70498CB
:1015400008286ED0FFE704980C286AD0FFE70598BA
:10155000006840F20041C4F20101884210D1FFE767
:10156000049800285DD0FFE70498042859D0FFE7CD
:101570000498082855D0FFE704980C2851D0FFE7BD
:101580000598006844F20001C4F20101884208D1C4
:10159000FFE70498002844D0FFE70498042840D0CF
:1015A000FFE70598006844F20041C4F20101884257
:1015B00003D1FFE70498A0B3FFE70598006844F65D
:1015C0000001C4F20101884203D1FFE7049840B34F
:1015D000FFE70598006841F60001C4F20001884267
:1015E00007D1FFE70498E0B1FFE70498042818D07A
:1015F000FFE70598006841F60041C4F20001884207
:1016000003D1FFE7049860B1FFE70598006842F254
:101610000001C4F20001884204D1FFE7049808B930
:10162000FFE708E045F2DE10C0F602004FF4B961B2
:101630000CF020F8FFE7059800680499002205F0F7
:10164000EFFE0598016801200022C4F201029142D8
:1016500003900CD0FFE7059800684FF60041CBF6E9
:10166000FE710844B0FA80F040090390FFE7039848
:10167000C007D8B1FFE7FFE705980068006A41F2AC
:101680001111084210D1FFE705980068006A40F286
:101690004441084207D1FFE705980168486C20F4EF
:1016A00000404864FFE7FFE7FFE7FFE7FFE7059833
:1016B0000068006A41F21111084210D1FFE7059855
:1016C0000068006A40F24441084207D1FFE70598EC
:1016D0000168086820F001000860FFE7FFE7FFE706
:1016E000049828B9FFE70599012081F83E001EE023
:1016F0000498042806D1FFE70599012081F83F00EE
:10170000029012E00498082806D1FFE7059901200D
:1017100081F84000019005E00599012081F8410021
:101720000190FFE701980290FFE70298FFE7002091
:1017300006B080BD81B000900098006841F2004181
:10174000C4F20001884208D1FFE741F6B461C2F259
:101750000001086801300860FFE701B07047000031
:1017600081B0009001B0704782B00190ADF80210D6
:1017700002B0704780B582B00190019807F068FE12
:101780008DF803009DF8030004281BD0FFE79DF8A7
:10179000030000EBC00140F27070C2F2000000EBE9
:1017A0008100C06968B1FFE79DF8030000EBC0014C
:1017B00040F27070C2F2000000EB8100C069804707
:1017C000FFE7FFE702B080BD80B582B001900198CD
:1017D0000168C86820F49070C86001980168486981
:1017E00020F0010048610198006B012807D1FFE754
:1017F00001980168C86820F01000C860FFE70198F0
:1018000000684069400600282BD5FFE70198016871
:10181000486920F0400048610198806B98B1FFE76B
:101820000198816B49F23D30C0F6010008650198CE
:10183000806BF8F759FB28B1FFE70198806B016DC9
:101840008847FFE70CE001990020C885019A202114
:1018500082F83E10019908630198FFF78BFFFFE7BC
:101860000CE001990020C885019A202182F83E10E1
:10187000019908630198FFF77DFFFFE7002002B0A0
:1018800080BD000080B582B00190019807F0E0FDB6
:101890008DF803009DF8030004281BD0FFE79DF896
:1018A000030000EBC00140F27070C2F2000000EBD8
:1018B0008100006968B1FFE79DF8030000EBC001FB
:1018C00040F27070C2F2000000EB810000698047B6
:1018D000FFE7FFE702B080BD80B588B007900798AA
:1018E00000680068069007980068C068059007982F
:1018F000006840690490002003900290069800F070
:101900000F000390039888B9FFE79DF81800800640
:1019100000280AD5FFE79DF814008006002804D5AA
:10192000FFE7079807F0C6FD78E1FFE70398002876
:1019300000F0B480FFE79DF81000C00738B9FFE75A
:10194000BDF8140010F4907F00F0A880FFE79DF828
:101950001800C00758B1FFE79DF81500C00730B167
:10196000FFE70799086C40F001000864FFE79DF865
:101970001800400700280BD5FFE79DF81000C007AE
:1019800030B1FFE70799086C40F002000864FFE7F8
:101990009DF81800800700280BD5FFE79DF8100080
:1019A000C00730B1FFE70799086C40F004000864F5
:1019B000FFE79DF818000007002811D5FFE79DF804
:1019C00014008006002805D4FFE79DF81000C0072A
:1019D00030B1FFE70799086C40F008000864FFE7A2
:1019E0000798006C002858D0FFE79DF81800800683
:1019F00000280AD5FFE79DF814008006002804D5CA
:101A0000FFE7079807F056FDFFE707980068406971
:101A1000C0F3801002900798006C0007002803D4E0
:101A2000FFE7029888B3FFE7079807F0CBFC079819
:101A3000006840694006002822D5FFE70798016842
:101A4000486920F0400048610798806B98B1FFE733
:101A50000798816B49F2E910C0F601000865079804
:101A6000806BF8F741FA28B1FFE70798806B016DAA
:101A70008847FFE703E00798FFF704FFFFE703E06D
:101A80000798FFF7FFFEFFE706E00798FFF7FAFE6B
:101A9000079900200864FFE7FFE7BFE00798006BA5
:101AA000012840F09B80FFE79DF81800C006002841
:101AB00040F19480FFE79DF81400C006002840F133
:101AC0008D80FFE7FFE7002001900798006800681D
:101AD000019007980068406801900198FFE7079817
:101AE00000684069400600284AD5FFE70798806BE8
:101AF00000684068ADF80200BDF8020000283ED042
:101B0000FFE7BDF802000799898D884237DAFFE7C1
:101B1000BDF802000799C8850798806BC069B0F5C9
:101B2000807F24D0FFE707980168C86820F48070A0
:101B3000C86007980168486920F00100486107986B
:101B40000168486920F0400048610799202081F829
:101B50003E0007990020086307980168C86820F0D4
:101B60001000C8600798806BF8F748F9FFE70798FE
:101B7000818DC28D891A89B2FFF7F6FDFFE74DE02E
:101B80000799888DC98D401AADF800000798C08D5F
:101B900018B3FFE7BDF80000F8B1FFE70798016848
:101BA000C86820F49070C86007980168486920F000
:101BB000010048610799202081F83E000799002024
:101BC000086307980168C86820F01000C86007988B
:101BD000BDF80010FFF7C8FDFFE71FE09DF81800F3
:101BE000000600280AD5FFE79DF81400000600282B
:101BF00004D5FFE7079807F03FFE0FE09DF81800B7
